:100000000C943F2B0C94442E0C946F2E0C949A2E2F
:100010000C94C52E0C94F02E0C941B2F0C94462F90
:100020000C94712F0C94702B0C94702B0C94702BDF
:100030000C94702B0C94702B0C94702B0C94702BD4
:100040000C94702B0C94EFBF0C94702B0C94702BB1
:100050000C94702B0C94702B0C94D4B20C94722BC7
:100060000C94702B0C943D9F0C94E99F0C94702B76
:100070000C94702B0C94702B0C94702B0C94702B94
:100080000C94702B0C94702B0C94702B0C94702B84
:100090000C94702B0C94702B0C94702B0C94702B74
:1000A0000C94702B0C94702B0C94702B0C94702B64
:1000B0000C94702B0C94702B0C94702B0C94702B54
:1000C0000C94702B0C94702B0C94702B0C94702B44
:1000D0000C94702B0C94702B0C94702B0C94702B34
:1000E0000C94702BBA2CBF2CC42CCE2CD82C512D98
:1000F000E22CEA2CF22CFC2C062D102D1F2D292D84
:10010000512D332D3D2D472D752D782D672D6B2DC0
:10011000712DAF2D7C2D802D862D8A2D8E2D942D29
:10012000982D9C2DAF2DA22DA62DAA2D7D615D6150
:1001300063616061666169616C6178616F618A6148
:1001400072617561839C819CA59CA29CA09CD79C9C
:10015000D49CD29C309DFE9CFB9CF99C709F769F0A
:10016000879F929F9A9FAF9F9E9FAF9FA29FA69FA0
:10017000AF9FAC9F084AD73B3BCE016E84BCBFFD0E
:10018000C12F3D6C74319ABD56833DDA3D00C77F67
:1001900011BED9E4BB4C3E916BAAAABE0000008000
:1001A0003F05A84CCDB2D44EB93836A9020C50B98F
:1001B000918688083CA6AAAA2ABE000000803F00BB
:1001C0000D94A21D0D94A22A0D94D4274E414E49A0
:1001D0004E495459494E46CDCCCC3D0AD7233C1705
:1001E000B7D13877CC2B329595E6241FB14F0A0052
:1001F0000020410000C84200401C4620BCBE4CCA42
:100200001B0E5AAEC59D7400407A10F35A00A072BE
:100210004E18090010A5D4E80000E8764817000041
:10022000E40B54020000CA9A3B000000E1F505000F
:100230000080969800000040420F000000A0860158
:10024000000000102700000000E803000000006428
:1002500000000000000A0000000000010000000093
:10026000002C76D888DC674F0823DFC1DFAE59E168
:10027000B1B796E5E3E453C63AE651997696E8E6D7
:10028000C28426EB898C9B62ED407C6FFCEFBC9CAA
:100290009F40F2BAA56FA5F490055A2AF75C936BBC
:1002A0006CF9676DC11BFCE0E40D47FEF520E6B577
:1002B00000D0ED902E0300943577050080841E0851
:1002C0000000204E0A000000C80C333333330F986F
:1002D0006E12831141EF8D2114893BE65516CFFE36
:1002E000E6DB18D1844B381BF77C1D901DA4BBE4C2
:1002F00024203284725E228100C9F124ECA1E53D04
:100300002700000A0B02090C0D0E08070304010068
:1003100000000000000000000000000000000000DD
:10032000000000000000000000000000001211109A
:1003300000000000000000000000000000000000BD
:10034000000000000000000102102020080810201A
:100350004010204080020102010804020101020451
:100360000810204080804020100804020180040210
:100370000180402010080402010804020101020467
:100380000810204080010204081020408005050567
:1003900005070508080808020202020A0A080804FC
:1003A000040404010101010101010103030303032A
:1003B000030303040707070C0C0C0C0C0C0C0C02B9
:1003C00002020206060606060606060B0B0B0B0BC0
:1003D0000B0B0B000020002300260029002C002F0F
:1003E00000320000010000030106010901000022A3
:1003F00000250028002B002E0031003400020100EF
:1004000000050108010B0100002100240027002A3B
:10041000002D003000330001010000040107010A33
:100420000101060D00FE09016602D620FFFE0BFE4B
:100430000AFE0D0060221969808080808080800023
:1004400080183363A0A0A00357675050F850F850AD
:10045000500259692078A0A0702828F0200259691C
:1004600048A85010204050A89002586840A0A040D2
:10047000A0989068281363808080113B6B204040D7
:100480008080808080404020113B6B804040202055
:1004900020202040408006556520A870A8200455E3
:1004A000652020F82020113363604080065161F8F8
:1004B00011336340E04002596908081010204040A1
:1004C0008080025969205088888888885020025985
:1004D000692060A02020202020F8025969708888B7
:1004E0000810204080F8025969F8081020700808A8
:1004F0008870025969101030505090F8101002594D
:1005000069F88080B0C808088870025969708880CE
:1005100080F088888870025969F8081010202040FF
:1005200040400259697088888870888888700259AC
:100530006970888888780808887011386840E040B9
:10054000000040E04011386840E04000006040801A
:10055000025969081020408040201008045464F8B3
:100560000000F802596980402010081020408002E5
:100570005969708888081020200020025969708805
:100580008898A8A8B080780259692050888888F88F
:10059000888888025969F048484870484848F002FD
:1005A0005969708880808080808870025969F0481D
:1005B000484848484848F0025969F8808080F080EF
:1005C0008080F8025969F8808080F0808080800205
:1005D00059697088808080988888700259698888F5
:1005E0008888F888888888123969E040404040400F
:1005F0004040E0025969381010101010109060024D
:100600005969888890A0C0A0908888025969808024
:10061000808080808080F80259698888D8A8A8885E
:1006200088888802596988C8C8A8A89898888802C4
:100630005969708888888888888870025969F08824
:100640008888F080808080015A6A708888888888CD
:1006500088A87008025969F0888888F0A090888876
:10066000025969708880807008088870025969F89A
:10067000202020202020202002596988888888880E
:10068000888888700259698888888850505020204E
:1006900002596988888888A8A8A8A850025969883A
:1006A00088505020505088880259698888505020BE
:1006B00020202020025969F808101020404080F8BE
:1006C000113B6BE0808080808080808080E00259D8
:1006D00069808040402010100808113B6BE020200A
:1006E00020202020202020E0085363205088015142
:1006F00061F82A22628040025666700878889868FD
:10070000025969808080F088888888F00256667077
:1007100088808088700259690808087888888888E5
:10072000780256667088F8808870025969304840AF
:1007300040F04040404000586870888888780888B9
:1007400070025969808080B0C888888888123868AB
:100750004000C040404040E0004A6A1000301010A5
:10076000101090906002596980808090A0C0A09085
:1007700088123969C040404040404040E00256661F
:10078000D0A8A8A8A888025666B0C8888888880219
:100790005666708888888870005868F0888888F065
:1007A0008080800058687888888878080808025611
:1007B00066B0C8808080800256667088601088703D
:1007C0000258684040F040404048300256668888F1
:1007D0008888986802566688888850502002566635
:1007E0008888A8A8A8500256668850202050880003
:1007F00058688888889868088870025666F81020BB
:100800004080F8015B6B1820202020C02020202091
:1008100018221969808080808080808080015B6BD5
:10082000C0202020201820202020C008536348A882
:1008300090FFFFFFFFFFFFFFFFFFFFFFFFFFFFFF37
:10084000FFFFFFFFFFFFFFFFFFFFFFFFFFFFFFFFB8
:10085000FFFF0D0060221969800080808080808009
:10086000800358682070A8A0A0A8702002596930A1
:10087000484040E0404048B0035666887050507091
:100880008802596988885050F820F8202022196978
:10089000808080800080808080124A6A60908060C2
:1008A0009090601090601A3262A0A003596970881D
:1008B000A8D8C8D8A88870045767700878887800C6
:1008C000F80356662850A0A05028045363F808087F
:1008D000163161E00359697088E8D8D8E8D8887083
:1008E0000A5161F8174464609090600357672020B4
:1008F000F8202000F807356540A02040E007356566
:1009000040A04020C02A2262408000586888888821
:100910008898E8808002596978E8E8E8E86828283B
:1009200028262161C0202262408007356540C040F2
:1009300040E0045767708888887000F8035666A006
:1009400050282850A0025A6A40C04040E0081828A9
:100950003808025A6A40C04040E0102808103802A7
:100960005A6A40A04020A048182838080259692037
:100970000020204080888870025A6A402000205061
:100980008888F88888025A6A10200020508888F8E1
:100990008888025A6A30480020508888F88888027F
:1009A0005A6A28500020508888F88888025A6A506D
:1009B000500020508888F88888025A6A20502020E9
:1009C000508888F8888802596958A0A0A0B0E0A093
:1009D000A0B8005B6B708880808080808870204029
:1009E000025A6A402000F88080F08080F8025A6A3B
:1009F000102000F88080F08080F8025A6A304800A9
:100A0000F88080F08080F8025A6A505000F88080A8
:100A1000F08080F8123A6A804000E0404040404058
:100A2000E0123A6A204000E04040404040E0124A74
:100A30006A609000E04040404040E0123A6AA0A066
:100A400000E04040404040E0025969F0484848E832
:100A5000484848F0025A6A2850008888C8A89888F0
:100A600088025A6A40200070888888888870025AF4
:100A70006A10200070888888888870025A6A304816
:100A80000070888888888870025A6A2850007088A8
:100A90008888888870025A6A5050007088888888D0
:100AA00088700355658850205088015B6B087098EA
:100AB00098A8A8A8C8C87080025A6A4020008888F0
:100AC0008888888870025A6A1020008888888888F8
:100AD0008870025A6A30480088888888888870023E
:100AE0005A6A50500088888888888870025A6A102C
:100AF00020008888502020202002596980F08888B2
:100B000088F0808080025969609090A0A0908888C9
:100B1000B0025969402000700878889868025969C5
:100B20001020007008788898680259693048007071
:100B30000878889868025969285000700878889861
:100B400068025969505000700878889868025A6A9B
:100B500030483000700878889868025666702870AF
:100B6000A0A8500058687088808088702040025982
:100B7000694020007088F880887002596910200050
:100B80007088F88088700259693048007088F88051
:100B900088700259695050007088F8808870123946
:100BA00069804000C040404040E012396920400068
:100BB000C040404040E0124969609000C040404061
:100BC00040E0123969A0A000C040404040E0025A15
:100BD0006A5020601070888888887002596928508F
:100BE00000B0C888888888025969402000708888C9
:100BF000888870025969102000708888888870027F
:100C0000596930480070888888887002596928506E
:100C100000708888888870025969505000708888F0
:100C2000888870035767202000F80020200158684A
:100C3000087098A8A8C87080025969402000888868
:100C40008888986802596910200088888888986880
:100C50000259693048008888888898680259695024
:100C60005000888888889868005B6B10200088880E
:100C7000889868088870005A6A8080B0C88888C8D8
:100C8000B08080005B6B5050008888889868088826
:100C90007001050700FE0500FB01F220FFFE05FEC6
:100CA00005FE02004002152580808000800532424A
:100CB000A0A002556550F850F8500146562070C06B
:100CC00030E0200255659010204048025565608054
:100CD000689068051222808002253540808080401F
:100CE0000225358040404080043343A040A00333B8
:100CF0004340E0400122324080043141E0021121B2
:100D00008002556508102040800245556090909003
:100D100060022535C040404040024555E0106080EB
:100D2000F0024555E0106010E00245552060A0F04B
:100D300020024555F080E010E00245556080E090CB
:100D400060024555F010204040024555609060908B
:100D5000600245556090701060031323800080028C
:100D600014248000808002354520408040200333D9
:100D700043E000E00235458040204080024555E0D8
:100D8000106000400255657088B8A8700245556033
:100D90009090F090024555E090E090E0023545607B
:100DA00080808060024555E0909090E0023545E0FB
:100DB00080E080E0023545E080E0808002455570AB
:100DC00080B090700245559090F09090023545E0CB
:100DD000404040E00245553010109060024555906B
:100DE000A0C0A09002354580808080E002556588D3
:100DF000D8A8888802455590D0B09090024555609B
:100E000090909060024555E09090E08001465660D9
:100E10009090906010024555E09090E0900245550A
:100E200070806010E0023545E0404040400245558A
:100E300090909090600245559090A0A0400255651A
:100E400088A8A8A8500245559090609090024555FA
:100E50009090701060023545E0204080E00225351A
:100E6000C0808080C0025565804020100802253572
:100E7000C0404040C005324240A0024151F005222E
:100E80003280400244547090907002455580E0904A
:100E900090E002344460808060024555107090906C
:100EA0007002445460B0C0600235452040E04040CC
:100EB00000465670909070106002455580E090900A
:100EC0009002152580008080800027374000404038
:100ED0004040800245558090A0E09002152580801A
:100EE000808080025464F0A8A8A8024454E0909046
:100EF0009002445460909060004656E09090E080EC
:100F000080004656709090701010023444A0C0804B
:100F10008002445470C030E002354540E04040203B
:100F2000024454909090700244549090A040025417
:100F300064A8A85050023444A04040A000465690F7
:100F40009090701060024454F02040F002354560EB
:100F5000408040600215258080808080023545C039
:100F6000402040C005425250A0FFFFFFFFFFFFFF9F
:100F7000FFFFFFFFFFFFFFFFFFFFFFFFFFFFFFFF81
:100F8000FFFFFFFFFFFFFFFFFFFF020040FFFFFF2C
:100F9000FFFFFFFFFFFFFFFFFFFFFFFFFFFFFFFF61
:100FA000FFFFFFFFFFFFFFFFFFFFFFFFFFFFFFFF51
:100FB000FFFFFFFFFFFFFFFFFFFFFFFFFFFFFFFF41
:100FC000FFFFFFFFFFFFFFFFFFFFFFFFFFFFFFFF31
:100FD000FFFFFFFFFFFFFFFFFFFFFFFFFFFFFFFF21
:100FE000FFFFFFFFFFFFFFFFFFFFFFFF01050800FF
:100FF000FF060121023520FFFF07FF06FF09005011
:10100000221656808080800080153353A0A0A00255
:1010100057575050F850F850500257572070A07052
:1010200028702013355580A040A02002475740A0CB
:10103000A040A0A0502513538080801226564080E7
:1010400080808040122656804040404080024555B6
:101050009060F060900255552020F8202011335305
:10106000604080044151F011335340E04002465645
:1010700010102040808012365640A0A0A0A0401240
:10108000365640C0404040E00246566090106080B6
:10109000F0024656F020601090600246562060A094
:1010A000F02020024656F080E01090600246566024
:1010B00080E0909060024656F010202040400246AA
:1010C00056609060909060024656609090701060FC
:1010D000122555C0C000C0C0113656606000604087
:1010E00080123656204080804020034353F000F0A9
:1010F00012365680402020408012365640A02040B4
:101100000040015858304898A8A8904030024656F0
:10111000609090F09090024656E090E09090E0024F
:101120004656609080809060024656E09090909085
:10113000E0024656F080E08080F0024656F080E003
:10114000808080024656609080B090600246569043
:1011500090F0909090123656E040404040E00246B9
:101160005670202020A04002465690A0C0A0A0901B
:101170000246568080808080F002465690F0F090C3
:10118000909002465690D0F0B0B0900246566090D3
:1011900090909060024656E09090E0808001475722
:1011A000609090D0B06010024656E09090E0909031
:1011B000024656609040209060123656E040404013
:1011C0004040024656909090909060024656909013
:1011D00090906060024656909090F0F090024656D3
:1011E000909060609090025656888850202020028F
:1011F0004656F010204080F0123656E08080808005
:10120000E0024656808040201010123656E0202022
:101210002020E016325240A0014151F016225280A7
:1012200040024454709090700246568080E0909046
:10123000E012345460808060024656101070909026
:101240007002445460B0C060024656205040E040F6
:101250004001455560907010600246568080E090D5
:1012600090901236564000C04040E01137572000A1
:10127000202020A040024656808090E090901236B8
:1012800056C040404040E0025454D0A8A8A80244B0
:1012900054E090909002445460909060014555E075
:1012A00090E080800145557090701010024454A069
:1012B000D0808012345460C020C00246564040E0C6
:1012C00040502002445490909070123454A0A0A03A
:1012D0004002545488A8A850024454906060900181
:1012E00045559090709060024454F02040F00247C1
:1012F00057304020C02040302216568080808080A9
:1013000080024757C02040304020C006425250A0C3
:10131000FFFFFFFFFFFFFFFFFFFFFFFFFFFFFFFFDD
:10132000FFFFFFFFFFFFFFFFFFFFFFFFFFFFFFFFCD
:10133000FF090050221656800080808080014656AA
:101340002070A0A070200246562050E04050A0021D
:10135000555588705070880256568850F820F820ED
:10136000221757808080008080800247577080E07D
:10137000907010E0173151A002565670A8C8C8A846
:101380007014355560A06000E003435350A0501224
:101390003353E02020143151E002565670E8D8E86B
:1013A000D870173151E015335340A04012355540E5
:1013B000E04000E014355540A02040E0143555C011
:1013C00020C020C01622524080014555909090E0E8
:1013D0008002565678E8E8682828241151801122A6
:1013E00052408014355540C04040E014355540A06F
:1013F0004000E0034353A050A0024757808080A0E4
:1014000060F0200247578080A0D01020700247571C
:1014100080408060A0F02012365640004080A040FE
:1014200002475740206090F090900247572040605C
:1014300090F0909002475760906090F09090024733
:101440005750A06090F0909002475790006090F045
:10145000909002475760906090F0909002465670CE
:10146000A0A0F0A0B001475760908080906040023B
:1014700047574020F080E080F00247572040F0803E
:10148000E080F00247576090F080E080F00247571C
:101490009000F080E080F01237578040E0404040FC
:1014A000E01237572040E0404040E012375740A05C
:1014B000E0404040E0123757A000E0404040E002EA
:1014C00056567048E848487002475750A090D0B030
:1014D00090900247574020609090906002475720BC
:1014E000406090909060024757609060909090604C
:1014F00002475750A060909090600247579000605C
:1015000090909060123353A040A002465670B0B045
:10151000D0D0E0024757402090909090600247570B
:1015200020409090909060024757609090909090EB
:10153000600247579000909090906002575710209B
:10154000885020202002465680E09090E08002469D
:10155000566090A0A090A002475740200070909045
:1015600070024757204000709090700247572050FB
:10157000007090907002475750A0007090907002D9
:10158000465650007090907002475760906070907F
:101590009070025454F068B07811355560808060C6
:1015A0004002475740200060B0C0600247572040CB
:1015B0000060B0C06002475760900060B0C0600239
:1015C0004656500060B0C060123757804000C0409F
:1015D00040E0123757204000C04040E012375740EB
:1015E000A000C04040E0123656A000C04040E002DB
:1015F0004757A040A01070906002475750A000E0ED
:1016000090909002475740200060909060024757AA
:10161000204000609090600247576090006090907A
:101620006002475750A000609090600246569000BC
:10163000609090601235554000E0004002445470C4
:10164000B0D0E0024757402000909090700247577A
:1016500020400090909070024757609000909090CA
:1016600070024656900090909070014858204000BB
:1016700090907090600147578080E090E0808001FA
:1016800047579000909070906025753A25303275DC
:1016900000253032753A25303275002575642025D5
:1016A0003032753A25303275003FFFF03800703126
:1016B00086302387102787902F87D02F03D02030A4
:1016C000102078102078102030102F03D02F87D0D2
:1016D0002787902387103186303800703FFFF03F16
:1016E000FFF038007030FC3020FC102078102030E3
:1016F000102C00D02E31D02F7BD02F7BD02E31D08C
:101700002C00D020301020781020FC1030FC303815
:1017100000703FFFF004104002082002082004106F
:101720004008208010410010410008208004104033
:101730000000001FFFF81FFFF81FFFF81FFFF81F32
:10174000E020102010201010201020201020103039
:10175000300840048003001FE03FF03FF03FF01FDF
:10176000E01FE03FF03FF03FF00FC007800300456F
:1017700072723A207574663820666F6E74206E6FD0
:101780007420696E697469616C697A65642E0045BC
:1017900072723A207574663820666F6E74206E6FB0
:1017A0007420696E697469616C697A65642E00459C
:1017B00072723A207574663820666F6E74206E6F90
:1017C0007420696E697469616C697A65642E005071
:1017D0006C65617365205265736574005052494EA3
:1017E0005445522048414C54454400687474703A42
:1017F0002F2F6D61726C696E66772E6F7267003283
:101800002E302E302E31373000000C0D00FE070236
:101810002603BC017FFE08FE08FE0508080600003E
:1018200040F0C88888987810050808060000C0F8BD
:101830008888888888F80505050600012030F8307A
:10184000200508080600002070F820202020E00570
:1018500009090600FF2070A8A8B88888702005062E
:1018600006060001E08CEA8C8A0A0509090600FFD9
:10187000F8A88888888888A8F8050A0A0600FE2043
:101880005050505088A8A8887003030306000340F6
:10189000A040FFFFFFFFFFFFFFFFFFFFFFFFFFFF76
:1018A000FFFFFFFFFFFFFFFF0000000605FF01072E
:1018B0000706020080808080800080030303060109
:1018C00005A0A0A005060606000050F85050F850EC
:1018D0000509090600FF2070A8A07028A87020053F
:1018E0000707060000C8C81020409898050707069B
:1018F000000040A0A040A8906801030306020580F4
:1019000080800309090601FF20404080808040401C
:10191000200309090601FF8040402020204040802C
:1019200005070706000020A8702070A820050505FF
:101930000600012020F820200203030601FFC0401A
:1019400080050101060003F8020202060100C0C082
:101950000507070600000810102040408005070713
:10196000060000708898A8C8887003070706010061
:1019700040C040404040E00507070600007088086E
:10198000102040F8050707060000F8081030088806
:101990007005070706000010305090F8101005077A
:1019A00007060000F880F0080888700507070600A1
:1019B00000304080F0888870050707060000F808AE
:1019C0001010202020050707060000708888708806
:1019D0008870050707060000708888780810600284
:1019E0000505060100C0C000C0C00206060601FFD2
:1019F000C0C000C0408003050506010120408040B2
:101A000020050303060002F800F80305050601019E
:101A100080402040800507070600007088102020C5
:101A200000200507070600007088B8A8B880700578
:101A30000707060000708888F88888880507070669
:101A40000000F04848704848F0050707060000709D
:101A5000888080808870050707060000F0484848A5
:101A60004848F0050707060000F88080F08080F8FD
:101A7000050707060000F88080F0808080050707D2
:101A800006000070888080988870050707060000AF
:101A9000888888F8888888030707060100E04040A6
:101AA000404040E005070706000038101010109075
:101AB000600507070600008890A0C0A09088050771
:101AC00007060000808080808080F80507070600F8
:101AD0000088D8A8888888880507070600008888B5
:101AE000C8A8988888050707060000708888888835
:101AF0008870050707060000F08888F08080800560
:101B0000070706000070888888A890680507070600
:101B10000000F08888F0A090880507070600007094
:101B2000888070088870050707060000F8202020CC
:101B3000202020050707060000888888888888708C
:101B40000507070600008888888850502005070789
:101B500006000088888888A8A850050707060000A6
:101B6000888850205088880507070600008888501C
:101B700020202020050707060000F80810204080DC
:101B8000F80309090601FFE080808080808080E002
:101B900005070706000080404020101008030909CF
:101BA0000601FFE020202020202020E0050303067E
:101BB00000052050880501010600FEF80303030616
:101BC000010580402005050506000070087888782A
:101BD0000507070600008080F0888888F005050565
:101BE000060000708080887005070706000008085E
:101BF00078888888780505050600007088F0807070
:101C0000050707060000304840E040404005070750
:101C10000600FE70888888780870050707060000AF
:101C20008080F0888888880307070601004000C08C
:101C3000404040E00409090601FE10003010101079
:101C400010906005070706000080808890E090886B
:101C5000030707060100C04040404040E00505057D
:101C6000060000D0A8A8A8A8050505060000B0C871
:101C70008888880505050600007088888870050733
:101C8000070600FEF0888888F080800507070600B8
:101C9000FE78888888780808050505060000B0C821
:101CA00080808005050506000078807008F0050733
:101CB000070600002020F820202018050505060052
:101CC000008888889868050505060000888888507F
:101CD000200505050600008888A8A850050505060A
:101CE000000088502050880507070600FE88888875
:101CF00050204080050505060000F8102040F8033C
:101D000009090601FF204040408040404020010971
:101D1000090602FF8080808080808080800309091E
:101D20000601FF80404040204040408005030306FC
:101D3000000248A890FF1FFFFFFFFFFFFF600000A9
:101D4000000001FF400000000000FF8000000000D4
:101D5000007F83CF00000C303F87FF80000C301FD6
:101D6000867980000C000F8C30C7838C30E78C3074
:101D7000CFC7CC31F38C30DCECEC33B98C30D86C81
:101D80006C33198C30D06C0C33198C30D86C0C330C
:101D9000198C30DC6C0E3B198C30CF7C079F198C72
:101DA00030C77C038F194000000000000260000073
:101DB000000000061FFFFFFFFFFFF800060900FEFE
:101DC00006018902FE20FFFE07FE06FE0000000657
:101DD0000007010606060200808080800080030361
:101DE00003060103A0A0A00507070600FF5050F856
:101DF00050F850500509090600FE2070A8A0702870
:101E0000A870200608080600FF40A8481020485483
:101E1000080507070600FF6090906098906801032E
:101E2000030602038080800207070602FF408080CD
:101E3000808080400207070602FF8040404040400B
:101E4000800505050600008850F850880505050640
:101E500000002020F820200204040602FEC04040BA
:101E600080050101060002F8020202060200C0C05D
:101E700004060606010010102040808004060606B5
:101E8000010060909090906003060606010040C03B
:101E9000404040E00406060601006090102040F03B
:101EA000040606060100F020601010E00506060694
:101EB000000010305090F810040606060100F08073
:101EC000E01010E00406060601006080E0909060DB
:101ED000040606060100F010102040400406060625
:101EE000010060906090906004060606010060901A
:101EF00090701060020505060200C0C000C0C0025C
:101F000007070602FEC0C000C04040800505050668
:101F100000001860806018050303060001F800F84F
:101F2000050505060000C0300830C004070706019B
:101F300000609010604000400506060600007090AA
:101F4000A8B08070050606060000205088F8888832
:101F5000050606060000F088F08888F004060606EC
:101F60000100609080809060040606060100E09009
:101F7000909090E0040606060100F080E08080F07A
:101F8000040606060100F080E08080800406060654
:101F90000100609080B090600406060601009090F9
:101FA000F0909090030606060100E040404040E0BB
:101FB000050606060000381010109060040606069C
:101FC000010090A0C0A09090040606060100808049
:101FD000808080F005060606000088D8A8A88888BA
:101FE00004060606010090D0B09090900506060603
:101FF0000000708888888870040606060100E0905A
:1020000090E080800407070601FF609090D0B060E8
:1020100010040606060100E09090E0909004060689
:10202000060100609040209060050606060000F85A
:102030002020202020040606060100909090909019
:1020400060040606060100909090F06060050606A8
:102050000600008888A8A8D888050606060000881B
:102060005020205088050606060000888850202051
:1020700020040606060100F010204080F00306064A
:10208000060100E080808080E004060606010080F2
:102090008040201010030606060100E020202020CA
:1020A000E00503030600032050880501010600FE39
:1020B000F8020202060204804004040406010070D3
:1020C0009090700406060601008080E09090E00485
:1020D00004040601007080807004060606010010EA
:1020E000107090907004040406010060B0C0700489
:1020F0000606060100205040E040400406060601A6
:10210000FE6090907010600406060601008080E07A
:102110009090900306060601004000C04040E00396
:1021200008080601FE200060202020A040040606CA
:102130000601008080A0C0A090030606060100C032
:1021400040404040E0050404060000D0A8A88804F0
:102150000404060100E0909090040404060100606D
:102160009090600406060601FEE09090E0808004F6
:1021700006060601FE70909070101004040406011B
:1021800000A0D0808004040406010070C030E00488
:1021900006060601004040E0405020040404060109
:1021A0000090909070040404060100909060600517
:1021B000040406000088A8A8500404040601009046
:1021C0006060900406060601FE9090907090600496
:1021D0000404060100F02040F00307070601002078
:1021E0004040804040200107070602FF8080808039
:1021F0008080800307070601008040402040408027
:1022000004020206010350A0FFFFFFFFFFFFFFFFD4
:10221000FFFFFFFFFFFFFFFFFFFFFFFFFFFFFFFFCE
:10222000FFFFFFFFFFFFFFFFFF00000006000701A9
:1022300006060602008000808080800406060601F3
:10224000FF2070A0A070200507070600FF3048405F
:10225000F04040F8050505060000A8508850A80584
:1022600006060600008850F820F82001070706023D
:10227000FF808080008080800407070601FF708057
:1022800060906010E0030101060105A00607070643
:102290000000788494A49484780305050601016005
:1022A000A06000E00505050600002850A0502804A5
:1022B0000303060100F01010040101060102F006FC
:1022C00007070600007884B4A4A4847804010106FA
:1022D0000105F0040303060102609060050707068C
:1022E00000FF2020F8202000F8030505060101402A
:1022F000A02040E0030505060101C0204020C002E7
:10230000020206020440800405050601FF9090B019
:10231000D08005060606000078E8E8682828010154
:1023200001060202800202020602FE408003050549
:1023300006010140C04040E003050506010140A040
:102340004000E0050505060000A0502850A0050843
:10235000080600FF40C0405070307810050808069D
:1023600000FF40C04050680810380508080600FF0C
:10237000C0204030F030781004070706010020002C
:102380002060809060050707060000402020507004
:1023900088880507070600001020205070888805EF
:1023A00007070600002050205070888805070706A0
:1023B000000028502050708888050707060000504C
:1023C0000020507088880507070600002050205024
:1023D00070888805060606000078A0F0A0A0B80462
:1023E00008080601FE609080809060204004070786
:1023F0000601004020F080E080F00407070601009D
:102400002040F080E080F00407070601002050F033
:1024100080E080F00407070601005000F080E080B3
:10242000F00307070601008040E0404040E003075A
:10243000070601002040E0404040E0030707060196
:102440000040A0E0404040E0030707060100A00074
:10245000E0404040E00506060600007048E84848B5
:102460007004070706010050A090D0B090900407B8
:102470000706010040206090909060040707060165
:1024800000204060909090600407070601002050F3
:10249000609090906004070706010050A060909043
:1024A000906004070706010050006090909060055E
:1024B000050506000088502050880408080601FF22
:1024C0001070B0B0D0D0E0800407070601004020B3
:1024D0009090909060040707060100204090909033
:1024E00090600407070601002050909090906004CF
:1024F00007070601005000909090906005070706BE
:1025000000001020885020202004060606010080CC
:10251000E09090E0800406060601006090A0A09084
:10252000A004070706010040200070909070040787
:102530000706010020400070909070040707060114
:10254000002050007090907004070706010050A012
:102550000070909070040606060100500070909084
:102560007004070706010020502070909070050449
:102570000406000070A8B0780406060601FE70800C
:102580008070204004070706010040200060B0C0B2
:102590007004070706010020400060B0C070040707
:1025A0000706010020500060B0C070040606060156
:1025B00000500060B0C070030707060100804000B3
:1025C000C04040E0030707060100204000C0404033
:1025D000E003070706010040A000C04040E00306FA
:1025E00006060100A000C04040E004070706010005
:1025F0003060107090906004070706010050A00042
:10260000E090909004070706010040200060909041
:1026100060040707060100204000609090600407F6
:102620000706010020500060909060040707060133
:102630000050A00060909060040606060100500063
:10264000609090600505050600002000F800200459
:10265000040406010070B0D0E00407070601004042
:102660002000909090700407070601002040009021
:102670009090700407070601002050009090907021
:1026800004060606010050009090907004090906A7
:1026900001FE2040009090907090600408080601B0
:1026A000FE8080E09090E080800408080601FE50E3
:1026B00000909090709060536E346B3300496E764A
:1026C000616465727300427269636B6F7574004D6B
:1026D00061696E00536D6F6F7468696E6700536D4A
:1026E0006F6F7468696E67005A005A00590059008C
:1026F00058005800436F7272656374696F6E0043CF
:102700006F7272656374696F6E004D61696E004629
:10271000696C616D656E740054656D70657261748D
:10272000757265004261636B6C6173680053746518
:1027300070732F6D6D004A65726B00416363656C49
:1027400065726174696F6E0056656C6F6369747948
:1027500000436F6E66696775726174696F6E0045DC
:1027600073746570732F6D6D004573746570732F8E
:102770006D6D005A73746570732F6D6D005A7374AC
:102780006570732F6D6D005973746570732F6D6D67
:10279000005973746570732F6D6D00587374657094
:1027A000732F6D6D005873746570732F6D6D0041DC
:1027B0006476616E6365642053657474696E6773D3
:1027C0000056652D4A65726B0056652D4A65726B21
:1027D00000567A2D4A65726B00567A2D4A65726BE7
:1027E0000056792D4A65726B0056792D4A65726BD9
:1027F0000056782D4A65726B0056782D4A65726BCB
:1028000000416476616E6365642053657474696E1B
:10281000677300416D6178204500416D6178204506
:1028200000416D6178205A00416D6178205A004165
:102830006D6178205900416D6178205900416D61CA
:1028400078205800416D6178205800412D54726104
:1028500076656C00412D54726176656C00412D5295
:1028600065747261637400412D52657472616374A2
:1028700000416363656C00416363656C004164768D
:10288000616E6365642053657474696E6773005686
:1028900054726176204D696E005654726176204DF7
:1028A000696E00566D696E00566D696E00566D61F9
:1028B00078204500566D6178204500566D6178207E
:1028C0005A00566D6178205A00566D617820590083
:1028D000566D6178205900566D6178205800566D0C
:1028E0006178205800416476616E636564205365A9
:1028F0007474696E67730020082046616374002059
:10290000082046616374002008204D61780020088B
:10291000204D6178002008204D696E002008204D70
:10292000696E004175746F74656D70004F66660066
:102930004F6E004175746F74656D7000416476610F
:102940006E6365642053657474696E6773004C6FC1
:102950006164206D6D004C6F6164206D6D00556E7B
:102960006C6F6164206D6D00556E6C6F6164206DDD
:102970006D00416476616E6365204B004164766151
:102980006E6365204B00416476616E63656420531D
:10299000657474696E67730044697361626C652065
:1029A0005374657070657273004D383400417574EE
:1029B0006F20486F6D6500473238004D6F76652097
:1029C00041786973004D61696E0045787472756471
:1029D000657220004175746F20486F6D6500473245
:1029E00038004D6F7665205A004D6F76652059008E
:1029F0004D6F76652058004D6F74696F6E00457895
:102A000074727564657220004D6F76652025736D54
:102A10006D00004D6F766520302E316D6D004D6F6D
:102A2000766520316D6D004D6F76652031306D6DAE
:102A3000004D6F7665204178697300486F74656E4C
:102A40006420746F6F20636F6C64004578747275D6
:102A500064657220004D6F7665205A004D6F766573
:102A60002059004D6F76652058004D6F7665205ACD
:102A7000004D6F76652059004D6F766520580050E7
:102A800072696E742066726F6D204D6564696100B5
:102A90005072696E742066726F6D204D6564696155
:102AA00000022E2E004D61696E005072696E740036
:102AB00043616E63656C0053746172742050726977
:102AC0006E7420003F005761697420666F72006663
:102AD000696C616D656E7420707572676500005079
:102AE0006C6561736520776169742E00507265733F
:102AF0007320427574746F6E00746F207265737505
:102B00006D65207072696E74005761697420666F1C
:102B1000720066696C616D656E74206C6F61640033
:102B2000496E736572742066696C616D656E7400C0
:102B3000616E6420707265737320627574746F6E59
:102B400000746F20636F6E74696E756500507265F6
:102B5000737320627574746F6E00746F20686561A2
:102B600074206E6F7A7A6C65004E6F7A7A6C65208D
:102B700068656174696E6700506C65617365207784
:102B80006169742E2E2E005761697420666F720081
:102B900066696C616D656E7420756E6C6F61640042
:102BA0005761697420666F720066696C616D656E4D
:102BB00074206368616E676500746F20737461725E
:102BC00074005061726B696E672E2E2E004368612F
:102BD0006E67696E672046696C616D656E7400553D
:102BE0004E4C4F41442046494C414D454E54004CBB
:102BF0004F41442046494C414D454E540020204E03
:102C00006F7A7A6C653A20002000456E6420666910
:102C10006C616D656E74206368616E6765005075E8
:102C2000726765206D6F726500004368616E67654D
:102C30002046696C616D656E7400556E6C6F6164E1
:102C40002046696C616D656E74004C6F616420464E
:102C5000696C616D656E74004D36303020423020F5
:102C6000542564004D373032203B2564004D373009
:102C70003220542564004D373031205425640050F3
:102C800072656865617420437573746F6D0050726E
:102C9000656865617420437573746F6D005072656B
:102CA00068656174204142530050726568656174C3
:102CB00020504C41004261636B004E6F204D6564B3
:102CC0006961005072696E742066726F6D204D6587
:102CD000646961004368616E6765204D6564696180
:102CE000004D32310041626F7574205072696E740C
:102CF0006572004368616E67652046696C616D6549
:102D00006E74004368616E67652046696C616D652D
:102D10006E74004D36303020423000436F6E66696D
:102D20006775726174696F6E0054656D706572616C
:102D300074757265004D6F74696F6E0052657375BE
:102D40006D65205072696E740054756E6500537421
:102D50006F70205072696E740050617573652050F9
:102D600072696E7400496E666F2053637265656E9A
:102D70000053746F70004261636B0053746F702076
:102D80005072696E74003F004261627973746570BD
:102D9000205A004261627973746570205900426163
:102DA000627973746570205800466C6F7700466CCA
:102DB0006F770046616E2053706565642031004670
:102DC000616E205370656564203100426564004285
:102DD0006564004E6F7A7A6C65004E6F7A7A6C6526
:102DE000005370656564005370656564004D6169EA
:102DF0006E004261627973746570205A00426162AC
:102E000079737465702059004261627973746570DA
:102E100020580047616D6573004669726D77617275
:102E2000652056657273696F6E004D61696E00436F
:102E30006F6F6C646F776E0046616E2053706565CE
:102E40006420310046616E20537065656420310056
:102E500042656400426564004E6F7A7A6C65004E8C
:102E60006F7A7A6C65004D61696E006F6F6F00005C
:102E7000001FC07FF0DDD8FFF87FF04440248000C1
:102E8000003180000024804440107CFEFEFE0400DF
:102E90000E000E007FC0FFE0FFE0FFE0FFE0060055
:102EA0000F001F8036C03FC0090016802940060071
:102EB0000F001F8036C03FC0168020401080104099
:102EC00008801FC037607FF05FD050500D801040E9
:102ED00048905FD077707FF01FC0104020200F0017
:102EE0007FE0FFF0E670FFF0198036C0C0300F00C1
:102EF0007FE0FFF0E670FFF0198036C0198047418F
:102F00004D45204F56455200526573746F726520CF
:102F10006661696C73616665004C6F61642053651E
:102F20007474696E67730053746F726520536574AF
:102F300074696E677300416476616E6365642053E3
:102F4000657474696E6773004D61696E004D6F76CC
:102F5000696E672E2E2E004D3234004D32352050D2
:102F60000A4D3234005072696E7420506175736579
:102F700064005061757365205072696E7400507200
:102F8000696E742041626F72746564004C756C7A6E
:102F9000426F742054415A20352072656164792E45
:102FA000005072696E74696E672E2E2E0050726921
:102FB0006E7420506175736564004D6564696120AD
:102FC00052656D6F766564004D6564696120496E78
:102FD000736572746564004D313137004D333100D3
:102FE00043616E6E6F7420656E74657220737562D6
:102FF0006469723A20002E0A006F70656E20666167
:10300000696C65642C2046696C653A2000617574B2
:103010006F25632E67006572726F72207772697414
:10302000696E6720746F2066696C650A004E6F7464
:10303000205344207072696E74696E670A005344AD
:10304000207072696E74696E672062797465200001
:103050002E0A0044656C6574696F6E206661696C48
:1030600065642C2046696C653A200046696C6520D1
:1030700064656C657465643A0057726974696E675B
:1030800020746F2066696C653A20002E0A006F700C
:10309000656E206661696C65642C2046696C653AD2
:1030A00020002E0A006F70656E206661696C656491
:1030B0002C2046696C653A200046696C6520736572
:1030C0006C65637465640A002053697A653A200070
:1030D00046696C65206F70656E65643A20002066F5
:1030E000696C653A2000667265736800646F696E8A
:1030F00067004E6F772000454E4420535542524F93
:103100005554494E450A002220706F7300222070EA
:103110006172656E743A2200535542524F555449BC
:103120004E452043414C4C207461726765743A22CD
:1031300000747279696E6720746F2063616C6C2013
:103140007375622D67636F64652066696C657320B3
:103150007769746820746F6F206D616E79206C657B
:1031600076656C732E204D4158206C6576656C2019
:1031700069733A310A004D3234004D3233202573E1
:103180000053442063617264206F6B0A006F7065A6
:103190006E526F6F74206661696C65640A00766FA9
:1031A0006C756D652E696E6974206661696C656405
:1031B0000A00534420696E6974206661696C0A00D4
:1031C000286E6F2066696C65290043616E6E6F74AE
:1031D000206F70656E2073756264697220007C3C9C
:1031E0003E5E2B3D3F2F5B5D3B2C2A225C000000A6
:1031F00000000000000000000000000000000000CF
:1032000000000000000000000000000000000000BE
:10321000000C000000000000000C00000000000096
:103220000012000000000000002300000000000069
:103230000021000000000000004C800000000000A1
:10324000005E8000000000000092400000000000CE
:1032500000A140000000000001212000000000004B
:10326000027F90000000000002001000000000003B
:1032700007FFF80000000000040008000000000044
:103280000800040000000000080006000000000024
:103290001000020000000000301E010000000000CD
:1032A000207F81000000000041FFE080000000005E
:1032B00043FCF08000000000873B784000000001E4
:1032C0008EDBFC60000000010FEBCC200000000250
:1032D0001FEDB610000000021FDEB6100000000453
:1032E00039CD7F080000000436E0FF080000000828
:1032F0007EC0BB84000000187F005D8600000010C7
:103300007FC0ED82000000203CC07301000000205F
:103310003B337F01000000701BE77E03800000C884
:103320001DEEDE04C00000880FDEDC044000012436
:103330000FDF3C092000012607DBF819200002728C
:1033400003E7F0139000025101FFE022900004898E
:10335000007F802448000904801E004824000BFEE2
:10336000400000DFF40010004000008002001FFF5A
:10337000FFFFFFFFFE000000000000000000000053
:10338000000000000000000000000000000010220B
:10339000103C3C0E1F0010221004221104001022C9
:1033A000100822110400102210083C110400102201
:1033B00010102211040010221020221104001E1CE3
:1033C0001E3C3C0E04000000000000000000000055
:1033D00000000000000000000000000000000000ED
:1033E00000000000000000000000000000000000DD
:1033F00000000000000000000000000000000000CD
:1034000000000000000000000000000000000000BC
:1034100000000000000000000000000000000000AC
:10342000000000000000000000000000000C0D0083
:10343000FE07022603BC017FFE08FE08FE05080801
:1034400006000040F0C88888987810050808060033
:1034500000C0F88888888888F805050506000120DE
:1034600030F830200508080600002070F8202020E1
:1034700020E00509090600FF2070A8A8B888887018
:1034800020050606060001E08CEA8C8A0A05090977
:103490000600FFF8A88888888888A8F8050A0A0620
:1034A00000FE205050505088A8A8887003030306DF
:1034B000000340A040FFFFFFFFFFFFFFFFFFFFFFF4
:1034C000FFFFFFFFFFFFFFFFFFFFFF0000000605FC
:1034D000FF010707060200808080808000800303D0
:1034E00003060105A0A0A005060606000050F8503E
:1034F00050F8500509090600FF2070A8A07028A800
:103500007020050707060000C8C8102040989805DD
:10351000070706000040A0A040A89068010303062A
:1035200002058080800309090601FF204040808059
:10353000804040200309090601FF804040202020F0
:1035400040408005070706000020A8702070A820D2
:103550000505050600012020F820200203030601CE
:10356000FFC04080050101060003F80202020601C7
:1035700000C0C0050707060000081010204040806A
:10358000050707060000708898A8C8887003070719
:1035900006010040C040404040E00507070600002B
:1035A000708808102040F8050707060000F808108A
:1035B0003008887005070706000010305090F8109A
:1035C00010050707060000F880F008088870050756
:1035D00007060000304080F0888870050707060065
:1035E00000F808101020202005070706000070884A
:1035F000887088887005070706000070888878083A
:103600001060020505060100C0C000C0C002060629
:103610000601FFC0C000C04080030505060101206F
:1036200040804020050303060002F800F80305056A
:1036300006010180402040800507070600007088D1
:1036400010202000200507070600007088B8A8B8E1
:103650008070050707060000708888F8888888054C
:103660000707060000F04848704848F005070706BD
:10367000000070888080808870050707060000F0D1
:103680004848484848F0050707060000F88080F0E1
:103690008080F8050707060000F88080F0808080B1
:1036A0000507070600007088808098887005070766
:1036B000060000888888F8888888030707060100C4
:1036C000E04040404040E005070706000038101089
:1036D000101090600507070600008890A0C0A09019
:1036E00088050707060000808080808080F8050735
:1036F0000706000088D8A88888888805070706007C
:10370000008888C8A8988888050707060000708880
:103710008888888870050707060000F08888F08090
:10372000808005070706000070888888A8906805D3
:103730000707060000F08888F0A0908805070706B4
:10374000000070888070088870050707060000F880
:103750002020202020200507070600008888888870
:1037600088887005070706000088888888505020E0
:1037700005070706000088888888A8A8500507075D
:10378000060000888850205088880507070600003A
:1037900088885020202020050707060000F8081020
:1037A000204080F80309090601FFE08080808080C6
:1037B0008080E005070706000080404020101008C8
:1037C0000309090601FFE020202020202020E00539
:1037D00003030600052050880501010600FEF803DA
:1037E000030306010580402005050506000070085A
:1037F0007888780507070600008080F0888888F0C0
:103800000505050600007080808870050707060022
:103810000008087888888878050505060000708803
:10382000F08070050707060000304840E040404047
:103830000507070600FE7088888878087005070766
:103840000600008080F0888888880307070601004A
:103850004000C0404040E00409090601FE1000306D
:1038600010101010906005070706000080808890F7
:10387000E09088030707060100C04040404040E058
:10388000050505060000D0A8A8A8A805050506009E
:1038900000B0C888888805050506000070888888FB
:1038A000700507070600FEF0888888F0808005070D
:1038B000070600FE78888888780808050505060050
:1038C00000B0C8808080050505060000788070087B
:1038D000F00507070600002020F820202018050525
:1038E0000506000088888898680505050600008898
:1038F000888850200505050600008888A8A850057E
:10390000050506000088502050880507070600FEC0
:1039100088888850204080050505060000F81020A2
:1039200040F80309090601FF204040408040404024
:10393000200109090602FF808080808080808080CD
:103940000309090601FF80404040204040408005B7
:10395000030306000248A890FF4F4646004F4E0062
:103960006563686F3A004572726F723A0045727211
:103970006F722077726974696E6720746F20454595
:1039800050524F4D210A0050726573732062757456
:10399000746F6E20286F72204D3130382920746F7B
:1039A0002068656174206E6F7A7A6C650A005072C7
:1039B00065737320627574746F6E20286F72204D6A
:1039C0003130382920746F20726573756D650A0077
:1039D000496E736572742066696C616D656E7420E2
:1039E000616E6420707265737320627574746F6E9B
:1039F00020286F72204D313038290A004D36303082
:103A00003A20546F6F20436F6C6400486F74656E8A
:103A10006420746F6F20636F6C640A00486F746574
:103A20006E6420746F6F20636F6C640A00496E735C
:103A30006572742066696C616D656E7420616E6478
:103A400020707265737320627574746F6E20286FB6
:103A500072204D313038290A0063616E63656C0055
:103A6000726573756D656400726573756D65007060
:103A7000617573656400706F7765726F6666002F9D
:103A80002F616374696F6E3A0020573A0020573AED
:103A900000486F74656E6420436F6F6C696E672EAB
:103AA0002E2E00486F74656E642048656174696EDF
:103AB000672E2E2E00202F002042403A0020403A50
:103AC000004D383420582059205A2045005468654C
:103AD000726D616C2052756E6177617900486F7408
:103AE000656E6420544845524D414C2052554E411C
:103AF0005741590042454420544845524D414C20BD
:103B000052554E4157415900202D20496E76616C27
:103B10006964206578747275646572206E756D6273
:103B2000657220210A0048656174696E67206661CC
:103B3000696C6564004265642048656174696E67FC
:103B4000204661696C656400546865726D616C2023
:103B500052756E6177617900424544205448455260
:103B60004D414C2052554E415741590048656174B2
:103B7000696E67206661696C656400486F74656E84
:103B8000642048656174696E67204661696C65648C
:103B900000546865726D616C2052756E6177617951
:103BA00000486F74656E6420544845524D414C2066
:103BB00052554E41574159004D494E54454D5020A4
:103BC00074726967676572656400486F74656E64D6
:103BD000204572723A204D494E54454D5000457271
:103BE000723A204D494E54454D5020424544004DB7
:103BF000415854454D502074726967676572656419
:103C000000486F74656E64204572723A204D4158C9
:103C100054454D50004572723A204D415854454D1F
:103C2000502042454400626564002C20737973740F
:103C3000656D2073746F70706564212048656174D0
:103C400065725F49443A200023646566696E6520A9
:103C500044454641554C545F004B6420004B69205D
:103C6000004B70200000626564005049442041759B
:103C7000746F74756E652066696E6973686564211A
:103C80002050757420746865206C617374204B70CB
:103C90002C204B6920616E64204B6420636F6E732F
:103CA00074616E74732066726F6D2062656C6F77DD
:103CB00020696E746F20436F6E66696775726174F8
:103CC000696F6E2E680A00504944204175746F7404
:103CD000756E65206661696C6564212074696D6527
:103CE0006F75740A00546865726D616C2052756E50
:103CF0006177617900486F74656E6420544845525D
:103D00004D414C2052554E415741590042454420A7
:103D1000544845524D414C2052554E41574159004F
:103D200048656174696E67206661696C6564004806
:103D30006F74656E642048656174696E67204661C2
:103D4000696C6564004265642048656174696E67EA
:103D5000204661696C656400504944204175746F68
:103D600074756E65206661696C6564212054656DAB
:103D7000706572617475726520746F6F2068696711
:103D8000680A00204B643A2000204B693A2000204A
:103D90004B703A20000A20436C61737369632050B2
:103DA0004944200A00204B643A2000204B693A2005
:103DB00000204B703A20000A204E6F206F7665720B
:103DC00073686F6F740A002054753A2000204B7599
:103DD0003A2000206D61783A2000206D696E3A200B
:103DE0000020643A200020626961733A2000504943
:103DF00044204175746F74756E65207374617274BC
:103E00000A00504944204175746F74756E652066D0
:103E100061696C6564212054656D706572617475AB
:103E2000726520746F6F20686967680A001000ADC2
:103E30000330016A0150022B0170030A019004F55E
:103E400000B005E500D006D800F007CE001009C587
:103E500000300ABE00500BB700700CB100900DABE3
:103E600000B00EA600D00FA200F0109D0010129915
:103E700000301395005014920070158E0090168B30
:103E800000B0178700D0188400F0198100101B7E45
:103E900000301C7B00501D7900701E7600901F734F
:103EA00000B0207000D0216E00F0226B0010246959
:103EB0000030256600502663007027610090285E60
:103EC00000B0295C00D02A5900F02B5600102D5468
:103ED00000302E5100502F4E0070304B0090314872
:103EE00000B0324500D0334200F0343E0010363B83
:103EF00000303737005038330070392E00903A299F
:103F000000B03B2300D03C1B00F03D1100103F01EE
:103F100000F03F00001000C90210012C01400122F6
:103F20000170011801B0010E01F00104015002FA04
:103F300000B002F0003003E600D003DC009004D2B1
:103F4000007005C800A006BE000008B400B009AAB1
:103F500000D00BA000600E960060118C000015824E
:103F60000020197800C01D6E00A0226400B0275AFE
:103F700000902C500000314600E0343C00103832F4
:103F800000903A2800603C1E00A03D1400803E0ACC
:103F900000203F00006F70656E005452494747454E
:103FA000524544003A20007A5F6D6178007A5F6D77
:103FB000696E00795F6D696E00785F6D696E0052A1
:103FC00065706F7274696E6720656E6473746F706C
:103FD000207374617475730A00456E6473746F7036
:103FE0007320256320256320256320256300205A44
:103FF0003A0020593A0020583A00656E6473746F95
:104000007073206869743A2000486F6D696E67208C
:104010004661696C656400496E76616C696420650F
:10402000787472756465720A0045313A2000453033
:104030003A20005A3A2000593A20004D53312C4D75
:1040400053322C4D53332050696E730A583A200076
:104050004D6963726F737465707320756E617661FC
:10406000696C61626C650A00205A3A0020593A0076
:1040700020436F756E7420583A00C23100001C2630
:104080000000F4190000D80F0000EB080000C00485
:104090000000750200004001000024F4D43050C339
:1040A0008E20C2A24017828B7011127A910D816C02
:1040B000D90AA861E108C7586607615143061E4B3B
:1040C0005D05C145A7041A411104093D98037139E2
:1040D00031034036DB0265339102D4305402802E26
:1040E0001D02632CEE01752AC501B028A00110271E
:1040F00081018F2564012B244B01E0223401AC2186
:104100001F018D200D01801FFC00841EED00971DF6
:10411000DF00B81CD200E61BC600201BBC00641ADE
:10412000B200B219A8000A19A0006A189900D117A4
:10413000910040178B00B516840031167E00B31530
:1041400079003A157300C7146F0058146A00EE1313
:1041500066008813630025135E00C7125B006C12B3
:10416000570015125400C111510070114F00211158
:104170004B00D61049008D10470046104400021035
:104180004200C00F4000800F3E00420F3C00060F6F
:104190003B00CB0E3800930E37005C0E3500270E27
:1041A0003400F30D3200C10D3100900D3000600D70
:1041B0002E00320D2D00050D2C00D90C2B00AE0C5D
:1041C0002900850C29005C0C2700350C27000E0CFB
:1041D0002600E80B2400C40B2400A00B23007D0B59
:1041E00023005A0B2100390B2100180B2000F80A7C
:1041F0001F00D90A1E00BB0A1E009D0A1D00800A6E
:104200001D00630A1C00470A1B002C0A1B00110A30
:104210001A00F7091A00DD091900C4091900AB09D1
:104220001900920917007B091800630917004C094F
:10423000160036091600200916000A091500F508AF
:104240001500E0081400CC081400B8081400A408F5
:104250001400900813007D0812006B081300580822
:104260001200460812003408110023081100120839
:10427000110001081100F0071000E0071000D0073E
:104280001000C0071000B0070F00A1071000910731
:104290000E0083070F0074070F0065070E00570715
:1042A0000E0049070E003B070D002E070E002007E9
:1042B0000D0013070D0006070D00F9060C00ED06B2
:1042C0000D00E0060C00D4060C00C8060C00BC066D
:1042D0000C00B0060C00A4060B0099060C008D061D
:1042E0000B0082060B0077060B006C060B006106C4
:1042F0000A0057060B004C060A0042060A00380660
:104300000A002E060A0024060A001A060A001006F1
:10431000090007060A00FD050900F4050900EB0580
:104320000900E2050900D9050900D0050900C70503
:104330000900BE050900B5050800AD050800A50582
:1043400009009C050800940508008C0508008405F8
:1043500008007C050800740508006C050700650569
:1043600008005D050700560508004E0507004705D3
:1043700007004005080038050700310507002A0539
:104380000700230507001C050600160507000F059A
:1043900007000805060002050700FB040600F504F7
:1043A0000700EE040600E8040600E2040700DB0450
:1043B0000600D5040600CF040600C9040600C304A5
:1043C0000600BD040600B7040600B1040500AC04F5
:1043D0000600A6040600A00405009B040600950440
:1043E0000500900406008A04050085040500800489
:1043F00006007A04050075040500700405006B04CE
:10440000050066040500610405005C04050057040E
:104410000500520405004D0405004804050043044E
:1044200005003E0404003A0405003504050030048C
:1044300004002C04050027040400230405001E04C6
:1044400004001A04040016040500110404000D04FD
:104450000400090405000404040000040400FC0333
:104460000400F8030400F4030400F0030400EC0368
:104470000400E8030400E4030400E0030400DC0398
:104480000400D8030400D4030400D0030400CC03C8
:104490000400C8030300C503030024F404D9201B4F
:1044A000C40C5C0E9804C4095F0265077101F40531
:1044B000F900FB04B30048048700C10369005803F6
:1044C000550003034500BE023A0084023100530246
:1044D0002A002902250004022000E4011C00C80172
:1044E0001900AF0117009801140084011300710135
:1044F00010006101100051010E0043010D00360152
:104500000B002B010B0020010B00150109000C0111
:10451000090003010800FB000800F3000800EB009D
:104520000700E4000600DE000600D8000600D20006
:104530000600CC000500C7000500C2000500BD0054
:104540000400B9000400B5000400B1000400AD008F
:104550000400A9000400A5000300A20003009F00BE
:1045600004009B00030098000300950002009300E4
:104570000300900003008D0002008B000300880000
:1045800002008600020084000300810002007F0018
:1045900002007D0002007B0002007900020077002B
:1045A0000100760002007400020072000100710038
:1045B00002006F0002006D0001006C0002006A0042
:1045C000010069000200670001006600010065004B
:1045D000010064000200620001006100010060004F
:1045E00001005F0002005D0001005C0001005B0053
:1045F00001005A0001005900010058000100570055
:104600000100560001005500010054000100530054
:104610000000530001005200010051000100500051
:1046200001004F0001004E0000004E0001004D004F
:1046300001004C0001004B0000004B0001004A004B
:104640000100490001004800000048000100470047
:104650000100460000004600010045000000450042
:10466000010044000100430000004300010042003B
:104670000000420001004100000041000100400034
:1046800001003F0000003F0001003E0000003E002E
:1046900001003D0000003D0001003C0000003C0026
:1046A00000003C0001003B0000003B0001003A001C
:1046B00000003A0001003900000039000100380014
:1046C000000038000000380001003700000037000B
:1046D0000100360000003600000036000100350001
:1046E00000003500000035000100340000003400F7
:1046F00000003400010033000000330000003300EC
:1047000001003200000032000000320001003100E0
:1047100000003100000031000100300000003000D6
:104720000000300001002F0000002F0000002F00CB
:1047300000002F0001002E0000002E0000002E00BF
:1047400001002D0000002D0000002D0000002D00B4
:1047500001002C0000002C0000002C0000002C00A8
:1047600001002B0000002B0000002B0000002B009C
:1047700001002A0000002A0000002A0000002A0090
:104780000100290000002900000029000000290084
:104790000000290001002800000028000000280077
:1047A000000028000000280001002700000027006A
:1047B000000027000000270000002700010026005D
:1047C0000000260000002600000026000000260051
:1047D0000100250000002500000025000000250044
:1047E0000000250000002500010024000000240036
:1047F0000000240000002400000024000100230029
:10480000000023000000230000002300000023001C
:10481000000023000000230001002200000022000D
:104820000000220000002200000022000000220000
:1048300001002100000021000000210000002100F3
:1048400000002100000021000000210001002000E4
:1048500000002000000020000000200000002000D8
:1048600000002000000020000000200001001F00C8
:1048700000001F0000001F0000001F0000001F00BC
:1048800000001F0000001F0001001E0000001E00AD
:1048900000001E0000001E00000020204D363033B6
:1048A000200020286D6D2900205300205A00205937
:1048B0000020580020204D343235204600426163EC
:1048C0006B6C61736820636F6D70656E7361746982
:1048D0006F6E3A0A002055004C0046696C616D65A8
:1048E0006E74206C6F61642F756E6C6F6164206CE8
:1048F000656E677468733A0A0020204D39303020A5
:104900004B004C696E65617220416476616E63652F
:104910003A0A0020440020490020204D3330342042
:10492000500020440020490020204D3330312050D9
:10493000005049442073657474696E67733A0A00C5
:1049400020460020420020480020204D31343520F0
:1049500053004D6174657269616C2068656174759E
:104960007020706172616D65746572733A0A00201F
:104970004500205A002059002058002054002053A0
:104980000020204D32303520420020453C6D6178BA
:104990005F655F6A65726B3E0020583C6D61785FB1
:1049A000785F6A65726B3E20593C6D61785F795F14
:1049B0006A65726B3E205A3C6D61785F7A5F6A650A
:1049C000726B3E00416476616E6365643A20423CDE
:1049D0006D696E5F7365676D656E745F74696D6533
:1049E0005F75733E20533C6D696E5F6665656472EA
:1049F0006174653E20543C6D696E5F7472617665CA
:104A00006C5F66656564726174653E0020540020C9
:104A1000520020204D323034205000416363656CD9
:104A200065726174696F6E2028756E6974732F7377
:104A300032293A20503C7072696E745F616363651D
:104A40006C3E20523C726574726163745F61636393
:104A5000656C3E20543C74726176656C5F61636383
:104A6000656C3E0A00204500205A00205900202095
:104A70004D3230312058004D6178696D756D20419F
:104A80006363656C65726174696F6E2028756E6909
:104A900074732F7332293A0A00204500205A0020EF
:104AA000590020204D3230332058004D6178696D17
:104AB000756D206665656472617465732028756E16
:104AC0006974732F73293A0A0053746570732070E8
:104AD000657220756E69743A0A0020204D313439B0
:104AE0002043203B20556E69747320696E20436516
:104AF0006C736975730A0020204732312020202012
:104B00003B20556E69747320696E206D6D0048619D
:104B10007264636F6465642044656661756C7420BB
:104B200053657474696E6773204C6F616465640AC1
:104B30000028230000282300006400000028230030
:104B4000000000964300009643000040400000C86B
:104B5000410000C9420000C9420000C8440000D220
:104B600043454550524F4D20496E697469616C69E7
:104B70007A65640A00290A002062797465733B2013
:104B800063726320002073746F72656420736574B0
:104B900074696E67732072657472696576656420E6
:104BA0002800202863616C63756C61746564292139
:104BB0000A0020213D2000454550524F4D204352D0
:104BC00043206D69736D61746368202D20287374B0
:104BD0006F7265642920002053697A653A20004984
:104BE0006E6465783A2000204D61726C696E3D56A6
:104BF0003639290A00454550524F4D20766572736B
:104C0000696F6E206D69736D617463682028454516
:104C100050524F4D3D004E6F20454550524F4D2E46
:104C20000A00290A002062797465733B206372636D
:104C3000200053657474696E67732053746F7265D6
:104C4000642028004E6F20454550524F4D2E0A00DB
:104C5000454550524F4D206461746173697A6520F7
:104C60006572726F722E0A005761726E696E673AD2
:104C700020486F6D696E672042756D7020446976BB
:104C800069736F72203C20310A00020204486F6D84
:104C9000652025732573257320466972737400207F
:104CA00046697273740A00486F6D65200020746F46
:104CB0006F206C6F6E6720657874727573696F6EA4
:104CC0002070726576656E7465640A0020636F6C8F
:104CD0006420657874727573696F6E207072657682
:104CE000656E7465640A0020453A00205A3A002037
:104CF000593A00583A00000048420000484200007B
:104D00004040FFFFFF0000A0400000A04000000066
:104D1000400000954300008A4300007A43000000F1
:104D200000000000C0000000000000954300008962
:104D30004300007A4300000000000000C0000000B3
:104D40000020746F6F206C6F6E67206578747275C9
:104D500073696F6E2070726576656E7465640A00A3
:104D600020636F6C6420657874727573696F6E2050
:104D700070726576656E7465640A00627573793A5F
:104D80002070617573656420666F7220696E70753E
:104D9000740A00627573793A2070617573656420D6
:104DA000666F7220757365720A00627573793A20B6
:104DB00070726F63657373696E670A0020496E765F
:104DC000616C696420657874727564657220004D49
:104DD00031343520533C696E6465783E206F7574BC
:104DE000206F662072616E67652028302D31290A98
:104DF00000436C69636B20746F20526573756D6539
:104E00002E2E2E00220A00556E6B6E6F776E206379
:104E10006F6D6D616E643A202200454550524F4DD2
:104E2000204F4B0A004E6F204D6F76652E00454394
:104E3000484F00494E464F004552524F525300448E
:104E4000525952554E00434F4D4D554E49434154D2
:104E5000494F4E006F6666002E4E334E384E3F4E21
:104E6000464E44454255473A004C756C7A426F7441
:104E70002054415A2035204F46462E00205A00200B
:104E80005900580020204D61783A2000205A002017
:104E90005900580020204D696E3A2000536F667407
:104EA00020656E6473746F70733A20002569730017
:104EB00025696D20256973002569682025696D20A5
:104EC00025697300256964202569682025696D209E
:104ED0002569730025697920256964202569682082
:104EE00025696D20256973005072696E742074699C
:104EF0006D653A20004D3131332053002F2F2000B3
:104F00004361703A004348414D4245525F54454D1C
:104F10005045524154555245004D4F54494F4E5FF4
:104F20004D4F44455300544845524D414C5F5052FB
:104F30004F54454354494F4E004155544F524550EC
:104F40004F52545F53445F53544154555300505291
:104F50004F4D50545F535550504F525400454D459E
:104F60005247454E43595F504152534552004341C9
:104F700053455F4C494748545F4252494748544E55
:104F800045535300544F47474C455F4C494748549D
:104F90005300534F4654574152455F504F57455267
:104FA000004255494C445F50455243454E54004CD5
:104FB0004556454C494E475F44415441005A5F5065
:104FC000524F4245004155544F4C4556454C0050B8
:104FD00052494E545F4A4F420050524F4752455338
:104FE00053004155544F5245504F52545F54454D14
:104FF0005000564F4C554D4554524943004545507D
:10500000524F4D0042494E4152595F46494C455F0F
:105010005452414E534645520053455249414C5F0C
:10502000584F4E5F584F4646004649524D574152E1
:10503000455F4E414D453A4D61726C696E20322E8E
:10504000302E302E31373020284769746875622938
:1050500020534F555243455F434F44455F55524C93
:105060003A68747470733A2F2F636F64652E616CA5
:105070006570686F626A656374732E636F6D2F6409
:105080006966667573696F6E2F4D41524C494E20AB
:1050900050524F544F434F4C5F56455253494F4E19
:1050A0003A312E30204D414348494E455F545950C6
:1050B000453A4C756C7A426F742054415A20352021
:1050C00045585452554445525F434F554E543A311A
:1050D00020555549443A63333235356339362D34DA
:1050E0003039372D343838342D386564302D6465C7
:1050F000643266663962616536310A0020284E6F77
:105100007420796574206D6561737572656429001A
:10511000202041766572616765206D6561737572E7
:105120006564206261636B6C61736820286D6D2912
:105130003A002020536D6F6F7468696E6720286D88
:105140006D293A20202020202020202020202020EF
:1051500020202020530020204261636B6C61736823
:105160002044697374616E636520286D6D293A204F
:105170002020202020202000202846312E30203DD5
:105180002066756C6C2C2046302E30203D206E6FD2
:105190006E65290A002020436F7272656374696F1F
:1051A0006E20416D6F756E742F466164652D6F754D
:1051B000743A202020202046006163746976653AA5
:1051C0000A00696E004261636B6C61736820436F13
:1051D0007272656374696F6E2000486F6D65205848
:1051E000592046697273740A00486F6D65205859DA
:1051F0002046697273740043757272656E7420661E
:10520000696C653A2000456E642066696C65206CA7
:105210006973740A00426567696E2066696C65206F
:105220006C6973740A00416476616E6365204B3D5E
:10523000003F4B2076616C7565206F7574206F663A
:105240002072616E67652028302D3130292E0A00CA
:105250004732380020466C6F773A200020643A00CD
:1052600020693A0020703A00204500205A00205959
:1052700000204D393220580043290A0061626C65D4
:105280006420286D696E2074656D702000646973F8
:1052900000656E00436F6C64206578747275646598
:1052A0007320617265200020540020520041636326
:1052B000656C65726174696F6E3A205000496E7654
:1052C000616C69642065787472756465720A002087
:1052D000643A0020693A0020703A00536C656570AA
:1052E0002E2E2E0047322F473320626164207061DA
:1052F00072616D65746572730A00446F6E65207328
:105300006176696E672066696C652E0A00534420D9
:1053100072656164206572726F720A00446F6E6517
:10532000207072696E74696E672066696C650A0028
:105330004D32390053544F505045442E2000507286
:10534000696E7465722073746F7070656420647523
:105350006520746F206572726F72732E20466978B3
:1053600020746865206572726F7220616E642075AA
:105370007365204D39393920746F207265737461FB
:1053800072742E202854656D706572617475726533
:105390002069732072657365742E205365742069CB
:1053A00074206166746572207265737461727469C9
:1053B0006E67290A004E6F20436865636B73756DD5
:1053C0002077697468206C696E65206E756D626502
:1053D000722C204C617374204C696E653A20004E2B
:1053E0006F20436865636B73756D207769746820FF
:1053F0006C696E65206E756D6265722C204C6173F0
:1054000074204C696E653A2000636865636B737540
:105410006D206D69736D617463682C204C617374C9
:10542000204C696E653A20004C696E65204E756DA2
:10543000626572206973206E6F74204C61737420F2
:105440004C696E65204E756D6265722B312C204C57
:10545000617374204C696E653A20004D3131300023
:10546000526573656E643A20002042002050006F40
:105470006B00220A00656E7175657565696E67203F
:105480002200504944204175746F74756E65206622
:1054900061696C656421204261642065787472756D
:1054A000646572206E756D6265720A0042656420E3
:1054B000436F6F6C696E672E2E2E00426564204824
:1054C000656174696E672E2E2E006F6B004732384F
:1054D0005859002020506C616E6E65724275666688
:1054E000657242797465733A2000204672656520C2
:1054F0004D656D6F72793A2000436F6D70696C6510
:10550000643A204F637420203720323031390A004A
:10551000207C20417574686F723A2028416C657058
:1055200068204F626A6563747320496E632E2C2075
:105530004C756C7A426F7420476974205265706FA5
:105540007369746F7279290A004F637420203720C1
:105550003230313931373A33313A323900204C6107
:10556000737420557064617465643A2000322E3083
:105570002E302E3137300A004D61726C696E00207A
:10558000536F6674776172652052657365740A00A3
:10559000205761746368646F672052657365740A8D
:1055A000002042726F776E206F75742052657365AC
:1055B000740A002045787465726E616C20526573C0
:1055C00065740A00506F77657255700A00737461D4
:1055D00072740A004B494C4C45442E2000507269AD
:1055E0006E7465722068616C7465642E206B696CE2
:1055F0006C28292063616C6C6564210A004B494C5E
:105600004C2063617573656420627920746F6F202C
:105610006D75636820696E6163746976652074696D
:105620006D65202D2063757272656E7420636F6DD9
:105630006D616E643A200050726F746563746564C6
:105640002050696E0A0025301D0C282924311C0BBE
:105650004527232F1B0A1E4443222B1A414203389D
:1056600009FF3603080602020001FA425E82938CAB
:1056700074A28EBDE6F7E000E400E200B38C1124D2
:105680001FBECFEFD1E2DEBFCDBF00E00CBF13E005
:10569000A0E0B2E0ECE9F3E702E00BBF02C0079044
:1056A0000D92A83BB107D9F726E1A8EBB3E001C002
:1056B0001D92A435B207E1F71BE2CEE3DBE200E086
:1056C00006C021970109802FFE010F94042FC533D6
:1056D000D10780E00807A9F70E94E9370D94BC398B
:1056E0000C9400001F920F920FB60F9211242F936B
:1056F0003F938F939F93AF93BF938091B903909102
:10570000BA03A091BB03B091BC033091B80323E06E
:10571000230F2D3720F40196A11DB11D05C026E8E9
:10572000230F0296A11DB11D2093B8038093B903E6
:105730009093BA03A093BB03B093BC038091BD03C5
:105740009091BE03A091BF03B091C0030196A11D2B
:10575000B11D8093BD039093BE03A093BF03B0938C
:10576000C003BF91AF919F918F913F912F910F9067
:105770000FBE0F901F9018952FB7F8946091B90342
:105780007091BA038091BB039091BC032FBF089521
:105790003FB7F8948091BD039091BE03A091BF03E1
:1057A000B091C00326B5A89B05C02F3F19F0019604
:1057B000A11DB11D3FBFBA2FA92F982F8827820F97
:1057C000911DA11DB11DBC01CD0142E0660F771FE7
:1057D000881F991F4A95D1F708958F929F92AF9293
:1057E000BF92CF92DF92EF92FF926B017C01D0DFEC
:1057F0004B015C01C114D104E104F104F1F09CD32C
:10580000C7DFDC01CB0188199909AA09BB09883EC9
:105810009340A105B10570F321E0C21AD108E10857
:10582000F10888EE880E83E0981EA11CB11CC114FB
:10583000D104E104F10421F7DDCFFF90EF90DF9078
:10584000CF90BF90AF909F908F9008958230910538
:1058500038F0880F991F880F991F05970197F1F766
:105860000895789484B5826084BD84B5816084BDD8
:1058700085B5826085BD85B5816085BDEEE6F0E0C9
:10588000808181608083E1E8F0E010828081826025
:105890008083808181608083E0E8F0E080818160A6
:1058A0008083E1EBF0E0808184608083E0EBF0E0D6
:1058B000808181608083E1E9F0E080818260808383
:1058C000808181608083E0E9F0E080818160808375
:1058D000E1EAF0E080818260808380818160808362
:1058E000E0EAF0E0808181608083E1E2F1E08081A4
:1058F00082608083808181608083E0E2F1E080814A
:1059000081608083EAE7F0E0808184608083808129
:1059100082608083808181608083808180688083D1
:105920001092C10008951F93CF93DF93182FEB01BE
:1059300061E016D1209711F460E004C0CF3FD1059B
:1059400031F461E0812FDF91CF911F9145C1E12FAB
:10595000F0E0EF5FFC4FE4914E2F50E0FA013197F9
:10596000E231F10508F09DC08827EE58FF4F8F4FB8
:105970000D94042F84B5806884BDC7BD97C084B5DD
:10598000806284BDC8BD92C0809180008068809391
:105990008000D0938900C093880088C080918000E7
:1059A000806280938000D0938B00C0938A007EC079
:1059B00080918000886080938000D0938D00C09398
:1059C0008C0074C08091B00080688093B000C09358
:1059D000B3006CC08091B00080628093B000C0932F
:1059E000B40064C080919000806880939000D09350
:1059F0009900C09398005AC0809190008062809373
:105A00009000D0939B00C0939A0050C0809190006A
:105A1000886080939000D0939D00C0939C0046C006
:105A20008091A00080688093A0008091A0008F7B6F
:105A30008093A000D093A900C093A80037C08091A4
:105A4000A00080628093A000D093AB00C093AA0016
:105A50002DC08091A00088608093A000D093AD00FD
:105A6000C093AC0023C08091200180688093200106
:105A7000D0932901C093280119C080912001806230
:105A800080932001D0932B01C0932A010FC08091F5
:105A90002001886080932001D0932D01C0932C01B8
:105AA00005C0C038D1050CF04CCF46CFDF91CF9167
:105AB0001F91089590E0FC013197E231F10508F063
:105AC0004EC08827EC57FF4F8F4F0D94042F8091C5
:105AD00080008F7703C0809180008F7D809380004D
:105AE000089580918000877FF9CF84B58F7702C0B9
:105AF00084B58F7D84BD08958091B0008F7703C0F9
:105B00008091B0008F7D8093B000089580919000C7
:105B10008F7707C0809190008F7D03C080919000A7
:105B2000877F8093900008958091A0008F7707C0B1
:105B30008091A0008F7D03C08091A000877F80931B
:105B4000A0000895809120018F7707C080912001E7
:105B50008F7D03C080912001877F8093200108956D
:105B6000CF93DF9390E0FC01E95BFC4F2491FC01B3
:105B7000E357FC4F8491882361F190E0880F991FCF
:105B8000FC01E95FFB4FC591D491FC01E351FC4F4F
:105B9000A591B491611109C09FB7F89488812095AF
:105BA00082238883EC912E230BC0623061F49FB76F
:105BB000F8943881822F809583238883EC912E2B53
:105BC0002C939FBF06C08FB7F894E8812E2B2883B3
:105BD0008FBFDF91CF9108951F93CF93DF93282F2D
:105BE00030E0F901EF5FFC4F8491F901E95BFC4F74
:105BF000D491F901E357FC4FC491CC23C1F0162F87
:105C0000811158DFEC2FF0E0EE0FFF1FE351FC4F46
:105C1000A591B4918FB7F894111105C09C91ED2F07
:105C2000E095E92302C0EC91ED2BEC938FBFDF915F
:105C3000CF911F910895CF93DF93282F30E0F90182
:105C4000EF5FFC4F8491F901E95BFC4FD491F901BE
:105C5000E357FC4FC491CC2389F081112BDFEC2F4B
:105C6000F0E0EE0FFF1FED52FC4FA591B491EC91C7
:105C7000ED2381E090E021F480E002C080E090E03C
:105C8000DF91CF91089508951F920F920FB60F9252
:105C900011240BB60F922F933F934F935F936F9303
:105CA0007F938F939F93AF93BF93EF93FF93E09175
:105CB0000802F09109021995FF91EF91BF91AF9100
:105CC0009F918F917F916F915F914F913F912F9114
:105CD0000F900BBE0F900FBE0F901F9018951F9244
:105CE0000F920FB60F9211240BB60F922F933F9382
:105CF0004F935F936F937F938F939F93AF93BF93D4
:105D0000EF93FF93E0910A02F0910B021995FF9136
:105D1000EF91BF91AF919F918F917F916F915F9123
:105D20004F913F912F910F900BBE0F900FBE0F9090
:105D30001F9018951F920F920FB60F9211240BB659
:105D40000F922F933F934F935F936F937F938F9314
:105D50009F93AF93BF93EF93FF93E0910C02F09169
:105D60000D021995FF91EF91BF91AF919F918F9186
:105D70007F916F915F914F913F912F910F900BBE4B
:105D80000F900FBE0F901F9018951F920F920FB695
:105D90000F9211240BB60F922F933F934F935F9363
:105DA0006F937F938F939F93AF93BF93EF93FF93E3
:105DB000E0910E02F0910F021995FF91EF91BF91C2
:105DC000AF919F918F917F916F915F914F913F9193
:105DD0002F910F900BBE0F900FBE0F901F90189534
:105DE0001F920F920FB60F9211240BB60F922F93A2
:105DF0003F934F935F936F937F938F939F93AF9353
:105E0000BF93EF93FF93E0910402F091050219957F
:105E1000FF91EF91BF91AF919F918F917F916F9182
:105E20005F914F913F912F910F900BBE0F900FBE3E
:105E30000F901F9018951F920F920FB60F9211247A
:105E40000BB60F922F933F934F935F936F937F9374
:105E50008F939F93AF93BF93EF93FF93E0910602CD
:105E6000F09107021995FF91EF91BF91AF919F912A
:105E70008F917F916F915F914F913F912F910F90F3
:105E80000BBE0F900FBE0F901F9018951F920F9290
:105E90000FB60F9211240BB60F922F933F934F938F
:105EA0005F936F937F938F939F93AF93BF93EF9382
:105EB000FF93E0911002F09111021995FF91EF917B
:105EC000BF91AF919F918F917F916F915F914F9112
:105ED0003F912F910F900BBE0F900FBE0F901F9010
:105EE00018951F920F920FB60F9211240BB60F92B6
:105EF0002F933F934F935F936F937F938F939F93D2
:105F0000AF93BF93EF93FF93E0911202F0911302CE
:105F10001995FF91EF91BF91AF919F918F917F91D3
:105F20006F915F914F913F912F910F900BBE0F900A
:105F30000FBE0F901F90189508951F93CF93DF9376
:105F4000EC011D821C821F821E82198681E08887D7
:105F500082E28A871F861E86FE01B396CE01C19615
:105F60002FEF2193E817F907E1F711E018A3CE010D
:105F700022D61F8B188E198E80E48A8F1B8E8CEA96
:105F800093E39AAB89ABDF91CF911F910895DB0129
:105F9000ED91FC911994EF92FF921F93CF93DF93B1
:105FA0001F921F92CDB7DEB77C01DC01D196ED9137
:105FB000FC91D29782E069837A83199520E030E0E2
:105FC0004AE069817A81C701E2DF182FD701D196B3
:105FD000ED91FC91D29783E01995D701D196ED917F
:105FE000FC91D29780E01995812F0F900F90DF914F
:105FF000CF911F91FF90EF9008950F931F93CF9330
:10600000DF93EC018B01E9A9FAA982E01995E9A9CE
:10601000FAA981E0199520E030E044E1B801CE0111
:10602000B6DF9E012D5C3F4F47E1B801CE01AFDFE7
:10603000E9A9FAA980E0DF91CF911F910F911994FE
:10604000EF92FF921F93CF93DF93EC017B01E9A9BD
:10605000FAA982E01995E9A9FAA981E0199520E049
:1060600030E045E1B701CE0192DF182F882339F0E7
:106070009E012D5C3F4F47E1B701CE0188DFE9A9C2
:10608000FAA980E01995812FDF91CF911F91FF90A0
:10609000EF900895FC01448F258F9C01245E3F4FB3
:1060A00042E375CFCF93DF931F92CDB7DEB79E014A
:1060B0002F5F3F4F46E46BDF89810F90DF91CF91D7
:1060C0000895CF93DF931F92CDB7DEB79E012F5F68
:1060D0003F4F47E45CDF89810F90DF91CF910895B6
:1060E00020E030E048E453CFCF93DF93EC016A81A6
:1060F0007B81D8DF88836A817B81CE01E2DF89835F
:106100006A817B81CE01ECDF8B879E012D5C3F4F46
:106110006A817B8147E1CE01DF91CF9138CFCF9368
:10612000DF93EC016A817B8136DF882319F0CE0191
:10613000DBDF81E0DF91CF9108958F929F92AF9244
:10614000BF92CF92EF920F93CF93DF931F921F9244
:10615000CDB7DEB74C015B012A834983EEDEF40143
:10616000B382A282498147A32A8120A705A3E4A282
:10617000C3A2C4010F900F90DF91CF910F91EF90C8
:10618000CF90BF90AF909F908F90C9CFFC0162815C
:10619000738133CFCF93DF93EC01EE85FF8530978A
:1061A00009F019956A817B81CE01DF91CF9148CFAB
:1061B000362F242FFC0162817381432F6BCF0F9305
:1061C000FC0182819381648F458F278F068F9F0109
:1061D000245E3F4F4BE3BC01CF010F91D8CEFC01B1
:1061E00060A30895BF92CF92DF92EF92FF920F9338
:1061F0001F93CF93DF936C01D62FB42EC22F78015B
:10620000CC2369F0F701049120E04B2D6D2FC601DE
:10621000D6DFFFEFEF1AFF0AC150D85FF1CFDF9151
:10622000CF911F910F91FF90EF90DF90CF90BF9093
:1062300008958F929F92AF92BF92CF92DF92EF928A
:10624000FF920F931F93CF93DF935C01C62EC42F51
:10625000D22ED02F220F220F220F1ED0882379F0AA
:10626000DC0F8D2C912CCD1751F087012D2D4C2F4B
:106270006C2DC501B7DFE80CF91CCF5FF4CFDF91BF
:10628000CF911F910F91FF90EF90DF90CF90BF9033
:10629000AF909F908F9008950F93FC010150040FD1
:1062A00084A996A9941718F0081728F402C00817B3
:1062B00050F0041740F42150260F83A995A9961792
:1062C00020F4281720F480E007C0281720F481E08C
:1062D000261710F0F8CF81E00F91089581E008951E
:1062E0002EE93FE0009729F0F9013197F1F7019786
:1062F000F9CF0895FC01128280818150838314823A
:106300000895FC0180819281980F928321819217D8
:1063100060F494819F5F94839381890F821710F0BA
:106320008FEF820F838381E0089580E00895FC0160
:1063300091E08381861708F490E031E0461708F079
:1063400030E0832F892B21E05281451708F420E0AB
:106350002823832F8923822B0895DC01FB011082DF
:1063600012968C911297818315968C911597815076
:10637000828313968C9183830895FB01418123814D
:10638000213029F0233031F468EF640F04C0642F0A
:10639000485F01C0642FCBCFDC0115962C91159777
:1063A0001696ED91FC911797CF01820F911D820FE8
:1063B000911D1192E817F907E1F70895FC01A681F4
:1063C000B7818281481B8581483018F0A80FB11D24
:1063D0004770382F369536953695562F577080E88A
:1063E00090E002C0959587955A95E2F7439F402D1E
:1063F0001124669566956695E62FF0E0E40FF11D91
:10640000EA0FFB1F3081222311F0832B02C08095FD
:10641000832380830895FB014181DC0112962C9136
:106420001297421760F013962C911397241738F0A7
:10643000608115962C91621710F42481BFCF0895C6
:10644000CF92DF92FF920F931F93CF93DF936C0154
:10645000EB01FA809B81913051F030F0923049F09D
:10646000933051F41FEF09C010E001E007C011E0C4
:1064700004C010E00FEF02C010E000E0F7FE03C020
:10648000BE01C601C8DF9881900F98839981910F52
:106490009983FF0C99F7DF91CF911F910F91FF9096
:1064A000DF90CF9008950F931F93CF93DF938901CF
:1064B000FB01C281D3814233D9F058F44531E1F078
:1064C000473109F1443141F5CE0166DFCE0112DFDB
:1064D00023C04634E1F04734E1F04B33E9F4B9012D
:1064E000CE014BDF8823C1F0B801CE01A9DF14C073
:1064F000B901CE0190DF10C0CE0103DF882369F01F
:10650000CE014ADF09C0B901CE0127DF05C08D8168
:1065100001C08981F801808381E0DF91CF911F91D3
:106520000F910895CF92DF92EF92FF920F931F93F6
:10653000CF93DF937C01D62FD42EC22F122FC62EDD
:10654000C20E6C2D611B183038F00FEF20E04D2D7E
:10655000C70135DE1850F5CF6C2F687F6D0F2C2FDB
:10656000277071F097E029272F5F27700FEF10E059
:1065700001C0000F2A95EAF720E04D2DC7011FDE6C
:10658000DF91CF911F910F91FF90EF90DF90CF900F
:106590000895CF92DF92EF92FF920F931F93CF93C4
:1065A000DF937C01D62ED42FC22F122FC42EC20E01
:1065B0004C2D411B183038F00FEF21E06D2DC70135
:1065C000FEDD1850F5CF4C2F487F4D0F2C2F277034
:1065D00071F097E029272F5F27700FEF10E001C0BF
:1065E000000F2A95EAF721E06D2DC701E8DDDF9164
:1065F000CF911F910F91FF90EF90DF90CF90089572
:10660000EF92FF920F931F93CF93DF93EC01162F1E
:10661000F42EE22E01E040DE882359F02E2D4F2D7E
:10662000612FCE01DF91CF911F910F91FF90EF90DD
:1066300079CFDF91CF911F910F91FF90EF90089547
:10664000EF92FF920F931F93CF93DF93EC01162FDE
:10665000F42EE22E022F21E01FDE882359F02E2D8A
:106660004F2D612FCE01DF91CF911F910F91FF90A0
:10667000EF908FCFDF91CF911F910F91FF90EF900F
:106680000895DF92EF92FF920F931F93CF93DF93C2
:106690007C01162FC42FD22ED02FFEDD8823F9F0D7
:1066A0002D2D4C2F612FC7013DDF2D2F4C2F612F3A
:1066B000C7016FDF6FEF6D0D610F2D2F4C2FC701DD
:1066C00068DF4FEF4D0F4C0F2D2D612FC701DF916C
:1066D000CF911F910F91FF90EF90DF9023CFDF912B
:1066E000CF911F910F91FF90EF90DF900895EF925F
:1066F000FF920F931F93CF93DF937C01D62F122F1E
:10670000C42F040F212F4C2F6D2FC7010BDFCF5F3C
:106710000C13F8CFDF91CF911F910F91FF90EF9065
:106720000895DF92EF92FF920F931F93CF93DF9321
:10673000EC01162FF42EE22EAFDD882329F02E2D4A
:106740004F2D612FCE01D3DFDF91CF911F910F919C
:10675000FF90EF90DF9008950895FC01E60FF11D82
:10676000849190E0982F88273196E4918E0F911DA7
:106770000895FC0184910895FCDF882321F0823084
:1067800011F083E0089586E0089580E00895FC010B
:106790008081089566E0E1CF68E0DFCF0A96FC01D2
:1067A000849108950B96FC0184910895DC01149660
:1067B000ED91FC911597319684910895BF92CF92F7
:1067C000DF92EF92FF920F931F93CF93DF938C0191
:1067D000E62EDC011496CD91DC911597CE01C9DF30
:1067E000F82EF80184819581C7DFC82EF1E0FF12F1
:1067F00003C02FE0B22E02C0BB24BA94D801149675
:106800008D919C911597CADFF82EF80184819581AE
:10681000C9DFD82ED80114968D919C911597BCDFB5
:10682000B0E6BE1538F4009729F0C80FD91F91E6DD
:10683000F92E0FC0F80184819581ACDFF0E4FE15DC
:1068400038F4009729F0C80FD91F81E4F82E01C051
:106850006196DE1490F4D80150961C92509753968E
:106860001C92539754961C92549751961C92519790
:1068700052961C9280E090E066C0DF1460F38C2D8D
:1068800090E0FE0124912F3F11F4219657C0FE1095
:106890004CC0D80114968D919C9115976ADF9E018A
:1068A0002F5F3F4FFE01882311F08230E1F4849185
:1068B000D80153968C935397F901249154962C93B5
:1068C0005497FE013396E4915096EC935097FE0155
:1068D0003496E4915196EC935197FE013596E491EC
:1068E0005296EC9320C08491982F9F709250D801BB
:1068F00052969C93529782958F7051968C93519794
:10690000F9012491822F8F7054968C93549722957D
:106910002F7053962C935397FE013296E491E29593
:10692000EF705096EC93CE010EC0FE013296E491CA
:10693000EB219C012E0F311DC20FD31FFD1409F452
:106940008ACFF3949ECFDF91CF911F910F91FF904B
:10695000EF90DF90CF90BF9008954F925F926F922B
:106960007F929F92AF92BF92CF92DF92EF92FF926F
:106970000F931F93CF93DF931F92CDB7DEB72C01F8
:10698000C62E942E622F1ADF7C01892B09F43AC09F
:10699000F20184819581F0DEB82EF2011389048919
:1069A0008189C80E8289981AD92CD01A212F4D2D91
:1069B0006C2DC20171DC882311F1EB0CF11C195F05
:1069C000169516951695612E712CD914C1F03C2D93
:1069D00057018A2D8E19811770F4F501049120E07A
:1069E0004D2D632FC2013983EADBFFEFAF1ABF0AD7
:1069F0003981385FEECFE60CF71CD394E6CFF20175
:106A0000808901C080E00F90DF91CF911F910F919D
:106A1000FF90EF90DF90CF90BF90AF909F907F90CE
:106A20006F905F904F9008950F931F93CF93DF93D4
:106A300000D0CDB7DEB78C01DC015596ED91FC910D
:106A400056972B834A83698319954A81480F2B8176
:106A50006981C8010F900F900F90DF91CF911F9126
:106A60000F917BCFAF92BF92DF92EF92FF920F9385
:106A70001F93CF93DF931F921F92CDB7DEB77C0198
:106A8000D62E042FDC015596ED91FC915697298363
:106A90003A831995080F2981A22E3A81B32E10E06E
:106AA000F50121915F01222339F0402F6D2DC7019F
:106AB00054DFD80E180FF4CF812F0F900F90DF9175
:106AC000CF911F910F91FF90EF90DF90BF90AF900B
:106AD0000895DF92EF92FF920F931F93CF93DF936E
:106AE0007C01D62FD42E8901DC015596ED91FC91C5
:106AF00056971995D80EC0E0F8012491222349F049
:106B00004D2D6D2FC70129DFD80FC80F0F5F1F4F05
:106B1000F3CF8C2FDF91CF911F910F91FF90EF90CA
:106B2000DF900895DC0114962D913C911597211565
:106B3000310509F43FC057968C915797F90181119F
:106B400008C03596E4915896EC935897F9013C9615
:106B500011C0813041F43F96E4915896EC935897D8
:106B6000F901709607C03D96E4915896EC935897BA
:106B7000F9013E96E4915996EC93599758968C9169
:106B80005897082E000C990B59962C915997821BF7
:106B9000910927FD93955A962C915A97203441F0EC
:106BA000829FC001112426E0969587952A95E1F7EA
:106BB0005B968C93089525EC33E3FC01368B258B93
:106BC0000895CF92DF92EF92FF920F931F93CF938E
:106BD000DF938C017B016A01CB01FA011995D82F53
:106BE000882311F1682FC801E9DDF801C189C19539
:106BF000FFEFEF1AFF0AC701F6011995F801882384
:106C000051F08089C80FC701F6011995D82F682F58
:106C1000C801D4DDEDCFD03221F091898389890F6D
:106C200001C080898C0F01C080E0DF91CF911F915E
:106C30000F91FF90EF90DF90CF90089547EC53E3D2
:106C4000C0CFCF93DF93FC0124813581261737070E
:106C500041F0EC017583648365DF85EC93E39E8BE3
:106C60008D8BDF91CF910895CF93DF9300D01F924A
:106C7000CDB7DEB7611571058105910579F09B01EE
:106C8000AC0169833A834B835C830F94932F2981F2
:106C90003A814B815C810F94E82E03C060E070E084
:106CA000CB010F900F900F900F90DF91CF9108952F
:106CB000CF92DF92EF92FF920F931F9362177307A9
:106CC000840795077CF489019A016B017C01C90155
:106CD000B8016C197D098E099F09C6DF6C0D7D1DF9
:106CE0008E1D9F1D1F910F91FF90EF90DF90CF9011
:106CF00008954F925F926F927F92AF92BF92CF9220
:106D0000DF92EF92FF920F931F93CF93DF93CDB754
:106D1000DEB729013A019B01AC0124193509460966
:106D200057098A899B89AC89BD89BC01CD016A1943
:106D30007B098C099D090F94842EA80197012419C1
:106D40003509460957090F94E82ECA01B9016A0DA1
:106D50007B1D8C1D9D1DDF91CF911F910F91FF9089
:106D6000EF90DF90CF90BF90AF907F906F905F904B
:106D70004F90089580E090E008950895CF92DF92BB
:106D8000EF92FF920F931F93CF93DF936C017A01E1
:106D90008B01C0E0D0E0CE15DF0589F0D8016D9100
:106DA0008D01D601ED91FC910190F081E02DC6019D
:106DB0001995892B11F47E0102C02196ECCFC701F1
:106DC000DF91CF911F910F91FF90EF90DF90CF90C7
:106DD00008956115710579F0FB0101900020E9F734
:106DE0003197AF01461B570BDC01ED91FC910280FE
:106DF000F381E02D199480E090E00895EACFDC0162
:106E0000ED91FC910190F081E02D19944F925F92E9
:106E10006F927F92EF92FF920F931F93CF93DF9326
:106E2000CDB7DEB7A1970FB6F894DEBF0FBECDBFCA
:106E30007C01FA01CB0119A2223008F42AE08E016C
:106E40000F5D1F4F422E512C612C712CBF01A301ED
:106E500092010F94C62EF901CA01015011096A303E
:106E600014F4605D01C0695CD8016C93232B242B62
:106E7000252B61F7B801C701ACDFA1960FB6F894D6
:106E8000DEBF0FBECDBFDF91CF911F910F91FF905D
:106E9000EF907F906F905F904F900895CF92DF9228
:106EA000EF92FF920F931F93CF93DF93EC016A0150
:106EB0007B012115310579F4E881F9810190F08198
:106EC000E02D642FDF91CF911F910F91FF90EF90F4
:106ED000DF90CF9019942A303105D9F477FF18C08C
:106EE0006DE28DDF8C0144275527BA014C195D09ED
:106EF0006E097F092AE0CE0189DF800F911FDF91A3
:106F0000CF911F910F91FF90EF90DF90CF90089558
:106F10002AE0B701A601CE01DF91CF911F910F9119
:106F2000FF90EF90DF90CF9071CF9A01AB01770F78
:106F3000660B770BB3CFCF93CFB7F8948091C10393
:106F4000811127C0E2ECF3E08491ECE7F3E0949147
:106F5000E82FF0E0EE0FFF1FE95FFB4FA591B49122
:106F6000EC91E92321F461E085E30E94EC2D61E0DE
:106F700085E30E94B02D8CB580618CBD8CB580649A
:106F80008CBD61E084E30E94B02D61E083E30E9448
:106F9000B02D8091C1038F5F8093C103CFBFCF918C
:106FA0000895CF92EF920F93FC0113AE14AE15AE7D
:106FB0000496C3D80F91EF90CF9008958EBD000036
:106FC0000DB407FEFDCF8EB5089580E090E00895E2
:106FD00008950E94312CFCDF0F94F329C0E0D0E02B
:106FE0000F947D2A2097E1F30E940000F9CFEEED87
:106FF000F3E083AF64AF08954AE050E0BC018EED4A
:1070000093E093CFEF92FF920F931F93CF93DF9371
:107010007A016F3F71058105910509F040F48EED0D
:1070200093E0EDDE82EE93E0C1DB90E014C0C0910E
:107030001904D0911A044D2F50E0EC2FF0E08B0191
:107040009C01BF0182EE93E03ED6C80FC0931904A5
:10705000D0931A049927DF91CF911F910F91FF9040
:10706000EF900895EF92FF920F931F93CF93DF93CA
:107070008B01CEEDD3E0FBACECAC4E2D50E06F2D90
:1070800070E09C0182EE93E076D6F80EFBAEECAE9B
:107090009927DF91CF911F910F91FF90EF90089565
:1070A000EF92FF920F931F93CF93DF938B01CEED5F
:1070B000D3E0FBACECAC4E2D50E06F2D70E09C01AA
:1070C00082EE93E0A4D6F80EFBAEECAE9927DF91EA
:1070D000CF911F910F91FF90EF9008956FEF7FEF89
:1070E000C1CFCF93DF93EA0182DFCE01DF91CF9151
:1070F000F5CF4FEF5FEF86CFCF93DF9300D01F9296
:10710000CDB7DEB729833A834B835C8370DF298157
:107110003A814B815C81CA01B9010F900F900F90A9
:107120000F90DF91CF91E5CF0F931F93CF93DF9314
:107130001F92CDB7DEB7082F8CE196E00E94D07A7F
:10714000182F863168F48CE196E0C8DF153109F418
:107150003DC060E270E080E090E0CBDF1F5FF6CFE3
:10716000CE0101960E94727E60E870E07BDF89812B
:10717000853120F56EE270E080E090E0BADF1981A1
:107180001431E1F06EE270E080E090E0B2DF1331A4
:10719000A9F089812EEF3FEF281B310986E0829FFD
:1071A000B001839F700D112460587F4F8CE196E0F1
:1071B00059DF60E270E080E090E09BDF8091C203E5
:1071C000801721F00093C2030E94547E0F90DF913C
:1071D000CF911F910F9108954F925F926F927F927E
:1071E0008F929F92AF92BF92CF92DF92EF92FF92D7
:1071F0000F931F93CF93DF93CDB7DEB72D970FB6C5
:10720000F894DEBF0FBECDBF80911206882309F42B
:107210008AC06091890C70918A0C072E000C880B33
:10722000990B0F94222C11E02091850C3091860C43
:107230004091870C5091880C0F94832D18160CF0F8
:1072400010E06091630C7091640C072E000C880BA9
:10725000990B0F94222C20915F0C3091600C40917F
:10726000610C5091620C0F94832D18160CF4106869
:107270001093D5038090650290906602A0906702FB
:10728000B090680220E030E0A901C501B4010F947C
:10729000802B87FD05C020E030E040E05FE304C0C4
:1072A00020E030E040E05FEBC501B4010F94A72A75
:1072B0000F94EF2BCB010F947D21BC0180ED93E067
:1072C0000F940E348090690290906A02A0906B0235
:1072D000B0906C0220E030E0A901C501B4010F9428
:1072E000802B87FD05C020E030E040E05FE304C074
:1072F00020E030E040E05FEBC501B4010F94A72A25
:107300000F94EF2BCB010F947D21BC018BEC93E00C
:107310000F940E348DE692E00F947D26BC0183EC31
:1073200093E00F940E340E940F7D182F81E037D622
:107330002091D50327FD03C042E102E002C048E0EE
:107340000CE08091160490E044977CF4809118043E
:10735000841758F027FD36C189E397E17C0123E0CB
:1073600060E582EE93E00E94193180911604843129
:10737000B8F480911804823098F0112309F425C1E3
:1073800080917F0C882309F420C189EA96E17C0171
:1073900002E123E042E068E682EE93E00E941931C8
:1073A000809116048C31D0F59091D5038090850C96
:1073B0009090860CA090870CB090880CC090890C9F
:1073C000D0908A0C843128F480911804883008F019
:1073D00017C280911604883008F4F2C18091160417
:1073E0008C3108F4F4C180905F0C9090600CA090F8
:1073F000610CB090620C6091630C7091640C809190
:107400001604883008F4E9C1809116048C3108F420
:10741000EBC1809116048C3108F4ECC18091F60820
:1074200083FF27C080912607882319F180911604D5
:107430008433F8F4809118048A32D8F007E028E009
:107440004AE26AE282EE93E06CD905E022E04CE287
:1074500062E382EE93E065D904E02AE041E36AE268
:1074600082EE93E00ED94BE262E382EE93E00E945B
:10747000D83080911604853328F480911804813324
:1074800008F0A6C00E942C82823048F09091160429
:10749000943328F490911804923308F0A1C080919D
:1074A00016048F3208F05DC080911804883208F409
:1074B00058C00F942B282B013C018CE3882E912C73
:1074C000A12CB12CC301B201A50194010F94C62EC9
:1074D000CA01B901A50194010F94C62ECA01D62E86
:1074E000C72E4901AE014F5F5F4F5A0150E8451664
:1074F00051E5550651E06506710408F48BC0B901E9
:1075000028E130E040E050E00F94C62E29013A0116
:10751000CF92DF92C40168E170E00F949F2E9F9399
:107520008F935F924F928BE996E19F938F93BF92D7
:10753000AF920F943D340FB6F894DEBF0FBECDBFAF
:107540005AE0451651046104710408F08DC098E0BA
:10755000892F880F980F892F8195A5016FE2855A91
:10756000C0DD809116048632A0F4809118048E311B
:1075700080F008E020E84EE160E082EE93E0D1D8B0
:1075800080911604863228F4809118048F3108F017
:107590006DC080911604823328F4809118048B32D8
:1075A00008F0F3C080911604813408F012C2809173
:1075B0001804873308F40DC26EE380E018DD812FD4
:1075C000B3DD07C285E197E1C9CE8FED96E1DFCE4D
:1075D00004E02AE441E366E382EE93E052D852CF1E
:1075E000F8E48F9FB0011124072E000C880B990B33
:1075F0000F94222C2AE037ED43E25CE30F94BE2D7A
:107600000F94F42B262F02E042E367E382EE93E02F
:1076100088D845CF84E68816910498F4CF92DF92FB
:107620003F932F9381E996E19F938F93BF92AF92FF
:107630000F943D340FB6F894DEBF0FBECDBF95E07A
:1076400087CFCF92DF923F932F9389E896E19F9364
:107650008F93BF92AF920F943D340FB6F894DEBF74
:107660000FBECDBF96E074CF99E072CF60E082EE9E
:1076700093E00E94EF3028E530E040E050E065E222
:1076800083E03ADD65E28BE0B2DC112321F080ED8E
:1076900093E024DD1BC08091380D80FDF8CF30EDE4
:1076A000C32E33E0D32EF60161916F01662371F092
:1076B0006F3234F4062E000C770B880B990B04C044
:1076C0006FE370E080E090E014DDEDCF29E530E07D
:1076D00040E050E065E288E20FDD65E280E387DCB0
:1076E000112321F08BEC93E0F9DC1CC08091380D64
:1076F000869580FDF7CF2BECC22E23E0D22EF6012B
:1077000061916F01662371F06F3234F4062E000C24
:10771000770B880B990B04C06FE370E080E090E07A
:10772000E8DCEDCF2AE530E040E050E065E28DE4B2
:10773000E3DC65E285E55BDC112321F083EC93E07B
:10774000CDDC1DC08091380D8695869580FDF6CFE5
:1077500093ECC92E93E0D92EF60161916F01662357
:1077600071F06F3234F4062E000C770B880B990BF6
:1077700004C06FE370E080E090E0BBDCEDCF61E03F
:1077800082EE93E00E94EF3004CF83E008D426E03D
:1077900030E040E050E062E383E0AEDC81E0FFD324
:1077A00080915F02909160020F944721AC0162E3E7
:1077B0008CE097DC65E270E080E090E09ADCF2CE4D
:1077C0008091760C11112DC0811108CE2AC08091B4
:1077D0001804853108F056C006CE8091520C111164
:1077E0007EC0811111CE7BC080911804853108F0D4
:1077F000A7C00FCE80911804853108F0CEC00ECE00
:1078000090FD03C08FE397E102C087E597E17C011B
:107810000CE022E048E068E082EE93E00E9419313B
:10782000D8CDB601DD0C880B990B0F94222C20E0EB
:1078300030E040E05FE30F94A72A0F94EF2BCB01D9
:107840000F944721FC0180818032D1F48181803204
:1078500011F491E001C092E043E050E0491B51096E
:107860004E0F5F1F892F880F980F892F819567E032
:10787000815F37DC69E070E080E090E03ADCAECD1B
:1078800093E0EACF20E030E040E05FE3C501B401DF
:107890000F94A72A0F94EF2BCB010F944721FC01E3
:1078A00080818032D1F48181803211F491E001C075
:1078B00092E043E050E0491B51094E0F5F1F892FB2
:1078C000880F980F892F81956CE1815F0ADC69E050
:1078D00070E080E090E00DDC86CD93E0EACF072EEB
:1078E000000C880B990B0F94222C20E030E040E034
:1078F0005FE30F94A72A0F94EF2BCB010F9447213E
:10790000FC0180818032D1F48181803211F491E0D8
:1079100001C092E043E050E0491B51094E0F5F1F48
:10792000892F880F980F892F819567E0865AD9DBB8
:1079300069E070E080E090E0DCDB66CD93E0EACFC8
:1079400020E030E040E05FE3C501B4010F94A72AD6
:107950000F94EF2BCB010F944721FC0180818032E3
:10796000D1F48181803211F491E001C092E043E0D2
:1079700050E0491B51094E0F5F1F892F880F980F48
:10798000892F81956CE1865AACDB69E070E080E07C
:1079900090E0AFDB3ECD93E0EACF80917F0C88236F
:1079A00009F43CCD24E6829FC001112481589F4FE9
:1079B0006FEF70E00F94B32ECB010F944721AC0111
:1079C0006CE187E68EDB65E270E080E090E091DBC1
:1079D00025CD2D960FB6F894DEBF0FBECDBFDF913B
:1079E000CF911F910F91FF90EF90DF90CF90BF90BC
:1079F000AF909F908F907F906F905F904F90089581
:107A00000F931F93CF93DF93CDB7DEB728970FB6B1
:107A1000F894DEBF0FBECDBF8A0123E0660F771F4B
:107A20002A95E1F7680F791F48E050E0CE010196F2
:107A30000F94713329813A81F8018081918128174F
:107A4000390790F08217930760F09C818281981724
:107A500058F081E090E03B812381231738F080E0EB
:107A600005C081E090E002C08FEF9FEF28960FB62F
:107A7000F894DEBF0FBECDBFDF91CF911F910F9164
:107A80000895EF92FF920F931F93CF93DF93EC0132
:107A90008B017A018A859B858617970729F0888153
:107AA0009981CFD81B870A8788859985019681F0AF
:107AB0000E811F81B70188819981C0D8080F111DDF
:107AC000888599858017910718F481E090E011C0AE
:107AD0006E818A81680F97014C81888199810E940B
:107AE00032352E813F81280F311D3F832E8380E068
:107AF00090E0DF91CF911F910F91FF90EF9008954B
:107B00004F925F926F927F928F929F92AF92BF92AD
:107B1000CF92DF92EF92FF920F931F93CF93DF9359
:107B2000CDB7DEB72D970FB6F894DEBF0FBECDBF31
:107B30006C012A013B01490158011B861C86CE01BC
:107B400001967C0188E0F70111928A95E9F7DB0143
:107B5000CA0127E0B695A795979587952A95D1F7FD
:107B60009A838983F42FFF77FD878F2F80588B832B
:107B70008C831A8619864F3F51056105710509F0FE
:107B800018F460E070E026C06091D8037091D903CA
:107B90008E01075F1F4F970140E05DE38091D603A0
:107BA0009091D7030E94217997FDEBCF69857A8563
:107BB00083E0660F771F8A95E1F78091D603909155
:107BC000D703680F791F48E050E0C7010F94713365
:107BD0006F8178856115710519F44B86B60106C071
:107BE000C616D70619F08D8580688B87AE01455F74
:107BF0005F4FC401F50119952D960FB6F894DEBFBD
:107C00000FBECDBFDF91CF911F910F91FF90EF90ED
:107C1000DF90CF90BF90AF909F908F907F906F90AC
:107C20005F904F9008956F927F928F929F92AF9244
:107C3000BF92CF92DF92EF92FF920F931F93CF9359
:107C4000DF9300D01F92CDB7DEB76C017B013A0104
:107C50005901480119821A821B821C82AE014F5FB2
:107C60005F4FB301C7010E9481797C0149815A812C
:107C70006B817C81411551056105710529F08401F5
:107C80009501C6013DDFE6CF0F900F900F900F904A
:107C9000DF91CF911F910F91FF90EF90DF90CF90E8
:107CA000BF90AF909F908F907F906F90089521E04C
:107CB0002093DA03E6EDF3E091838083738362839C
:107CC00080E090E008957F92AF92BF92CF92DF92D2
:107CD000EF92FF920F931F93CF93DF93CDB7DEB751
:107CE0002C970FB6F894DEBF0FBECDBF6C01762E79
:107CF000F72F842FE52FB901A801D6011496AD9076
:107D0000BC9015979091DA0391110AC02FEA37E1E0
:107D1000482F672DC6010E94693580E090E019C0A8
:107D2000DA82C9827B82FC838D83EE8318861F8270
:107D3000FA86E9861C861B8601E41DE39E012F5FFF
:107D40003F4FC501DDDEB501C6010E9421368F819E
:107D500098852C960FB6F894DEBF0FBECDBFDF918D
:107D6000CF911F910F91FF90EF90DF90CF90BF9038
:107D7000AF907F900895CF92DF92EF92FF920F9392
:107D80001F93CF93DF93CDB7DEB72C970FB6F89440
:107D9000DEBF0FBECDBF7C01C901F701C480D58015
:107DA0002091DA03211108C02FE837E1C7010E94B2
:107DB000693580E090E01CC0FA82E9826B837C83A5
:107DC0004D835E8318861F821A8709871C861B864F
:107DD00001E41DE39E012F5F3F4F4BE159E7BC01DA
:107DE000C60121DFB601C7010E9421368F81988527
:107DF0002C960FB6F894DEBF0FBECDBFDF91CF91AA
:107E00001F910F91FF90EF90DF90CF900895CF9248
:107E1000DF92EF92FF920F931F93CF93DF93CDB733
:107E2000DEB72C970FB6F894DEBF0FBECDBF7C0136
:107E3000C901F701C480D5802091DA03211108C05F
:107E40002FE637E1C7010E94693580E090E01CC051
:107E5000FA82E9826B837C834D835E8318861F825E
:107E60001A8709871C861B8601E41DE39E012F5F8C
:107E70003F4F4EE159E7BC01C601D5DEB601C7014F
:107E80000E9421368F8198852C960FB6F894DEBF1C
:107E90000FBECDBFDF91CF911F910F91FF90EF905B
:107EA000DF90CF900895CF93DF93EC01262F4CAD58
:107EB0006BAD04960E9414352BAD082E000C990B67
:107EC000820F911D8BAF81E090E0DF91CF910895FB
:107ED0000F939CE0899F802D112421E0280F20938F
:107EE000DD03845F8093DC0390E0029640911604EA
:107EF00050E08417950714F480E033C0822F90E09F
:107F00002091180430E082179307B4F76623A9F094
:107F100061E082EE93E00E94EF304091DD034E5F1E
:107F20000BE020E860E082EE93E00E94913360E095
:107F300082EE93E00E94EF3005C061E082EE93E0B4
:107F40000E94EF306091DC03809116046817A0F264
:107F50009091DD0380911804891770F280E047D872
:107F600081E00F910895CF93DF93FC0185ADEF0180
:107F70002496811105C081E085AFCE010E948F302B
:107F8000CE01DF91CF910C94C630CF93DF93EA01FD
:107F90002ED86FEF7FEFCE01DF91CF9181C8482FB0
:107FA00050E02091DB03022E000C330B42175307E5
:107FB00081F08093DB03813031F46BEB7DE182EE65
:107FC00093E00C94213669E078E182EE93E00C9422
:107FD0002136089581E008958EED93E0C4DF80E0BE
:107FE0000E94559A82EE93E00E94CA308111F7CF29
:107FF00064EC79E080E090E00C94AD9AEF92FF920F
:108000000F9380911B04811107C081E080931B04B2
:1080100082EE93E00E948F3082EE93E00E94C630A1
:1080200086E3E82E8DE1F82E03E127E047E064E2E5
:1080300082EE93E00E94193183E0B1DF4FEF57E108
:108040006BE285E2A2DF4BEE57E167E387E09DDF5D
:1080500082EE93E00E94CA308111E2CF0F91FF902F
:10806000EF90089581E0CADF64EC79E080E090E071
:108070000C94AD9AB1DFF6CF60E070E08BEB9DE140
:1080800016CE1F93CF93DF93C091E303C695C69599
:108090008EED93E068DFDC2FDD0F1D2F1C0F83E0DA
:1080A0007EDF6C2F80E00E94F7378CE196E016D8D7
:1080B0004CED57E16D2F80E068DF4FEC57E1612F09
:1080C00080E063DF82EE93E00E94CA308111E7CF47
:1080D000DF91CF911F9108950895CF93E62F6CE023
:1080E000869F602D112481E0860F8093DD03645FFD
:1080F0006093DC03462F50E04E5F5F4F20911604E3
:1081000030E0421753070CF44CC090E02091180463
:1081100030E0821793070CF044C0CE2F8EE30E940C
:10812000F73765E470E080E090E00E94793861E321
:108130006C0F062E000C770B880B990B0E94793878
:1081400060E270E080E090E00E9479386091850CF8
:108150007091860C8091870C9091880C0F94EF2B76
:10816000CB010F9447210E946E386FE270E080E0EF
:1081700090E00E9479380E940F7D811109C085E04E
:10818000C89FF0011124EE58F34F8481811109C07A
:108190008091890C90918A0C0F944721CF910C9477
:1081A0006E38CF910895CF92DF92EF92FF920F93A6
:1081B0001F93CF93DF931F921F92CDB7DEB77B0142
:1081C000622F498385DE4981882309F444C0442312
:1081D00011F101151105F9F4C7010E94F17A25E1A9
:1081E00030E0281B310937FF02C02F5F3F4F359524
:1081F000279530E82158822F830F87FD0DC060E25C
:1082000070E080E090E02A8339830E9479383981D8
:1082100031502A81F0CF30E8C32ED12CB601C701EE
:108220000E9450387601E81AF90A0115110511F477
:108230001E2D07C0FF24B701C8010E9432381E2D31
:10824000181B173040F060E270E080E090E00E9480
:108250007938181BF6CF0F900F90DF91CF911F91B7
:108260000F91FF90EF90DF90CF9008950F93CF93F1
:10827000DF93982F862FEA01692F2ADE882331F1B8
:1082800062E770E0CE010E945038C2E7C81BC730D9
:1082900040F060E270E080E090E00E947938C81B16
:1082A000F6CF6091DC038AE70E94F737602F000F5A
:1082B000770B880B990B0E94793860E270E080E0C0
:1082C00090E0DF91CF910F910C947938DF91CF91AD
:1082D0000F910895CF92DF92EF92FF920F931F9329
:1082E000CF93DF93982F862F6A017901692FF0DDF4
:1082F000882309F44BC0C701002321F00E94F17AC2
:10830000182F03C00E94D07A182FC3E1D0E0C11B00
:10831000D1098C2F880FC80FCC0FD0E0BE01C60149
:108320000E945038C81B6AE370E080E090E00E9431
:108330007938C73040F060E270E080E090E00E9461
:108340007938C81BF6CF8AEF189F802D11246091D1
:10835000DC0380580E94F737002369F06FEF7FEF4E
:10836000C701DF91CF911F910F91FF90EF90DF90A8
:10837000CF900C945038C701DF91CF911F910F918E
:10838000FF90EF90DF90CF900C946E38DF91CF91FB
:108390001F910F91FF90EF90DF90CF900895BF92C3
:1083A000CF92DF92EF92FF920F931F93CF93DF93C1
:1083B0006C017B010E94F17AC82FC7010E94D07A1C
:1083C00003E110E0081B11098C2F90E0BB24B3944B
:1083D000081719071CF0B12CC5E201C0CFE12C2F02
:1083E00030E0A9014E5F5F4F8091160490E048177E
:1083F000590744F0295031096091180470E0621760
:108400007307BCF5D0E0E114F104C9F16AE370E050
:1084100080E090E00E947938BB2081F0C45F8091B9
:108420001604C81760F12C2F30E0295031098091D3
:10843000180490E0821793071CF421C0DD23F9F0A3
:10844000802F880F800F6C2F880F0E94F73760E213
:1084500070E080E090E00E947938C701DF91CF9111
:108460001F910F91FF90EF90DF90CF90BF900C94F1
:108470006E38A6016C2F80E088DDD1E0C4CFDF919B
:10848000CF911F910F91FF90EF90DF90CF90BF9011
:108490000895CF92DF92EF92FF920F931F93CF93A5
:1084A000DF931F92CDB7DEB7182F7A01D22ECA0103
:1084B00069830E94F17A082F812F880F810FC82EBF
:1084C000CC0C1CE06981169F100D1124DD20C1F039
:1084D00061E082EE93E00E94EF30202F220F200F08
:1084E000220F2E5F0BE047EF410F6FEF6C0D82EE16
:1084F00093E00E94913360E082EE93E00E94EF30BF
:10850000A701612F8C2D41DDDD2071F061E082EE4D
:1085100093E00F90DF91CF911F910F91FF90EF901B
:10852000DF90CF900C94EF300F90DF91CF911F919F
:108530000F91FF90EF90DF90CF900895AF92BF9290
:10854000DF92EF92FF920F931F93CF93DF93EC0193
:108550005B01D42EC901B801A7010E94A07C91E063
:108560002D2D2927A50164E081E093DFCE010E9433
:10857000F17A2D2DAE0164E094E1981B892FDF91F3
:10858000CF911F910F91FF90EF90DF90BF90AF9030
:1085900080CFEF92FF920F93CF93DF93D82FC62F08
:1085A0007901682F8C2F94DC8823F1F0002331F0BF
:1085B00062E070E080E090E00E9479382D2F4C2F2F
:1085C00064E1C7010E947C7B68E770E00E9432385A
:1085D000C8E7C81BC73040F060E270E080E090E080
:1085E0000E947938C81BF6CFDF91CF910F91FF9091
:1085F000EF900895CF92EF920F93CF93DF93CEED4C
:10860000D3E01B821A828BE293E099838883CC2487
:10861000CA94EE24EA9406E427E448E464E172E0B4
:10862000CE010E94D13787E393E099838883DF915D
:10863000CF910F91EF90CF90089590910501947094
:108640009093030187FD76C0A398909105019095C2
:10865000947090930301909105019470909303019D
:10866000982F990F86FD72C0A3988091050180957F
:1086700084708093030180910501847080930301CD
:10868000292F220F96FD60C0A39880910501809547
:1086900084708093030180910501847080930301AD
:1086A000922F990F26FD4EC0A398809105018095C9
:1086B000847080930301809105018470809303018D
:1086C000292F220F96FD3CC0A3988091050180952B
:1086D000847080930301809105018470809303016D
:1086E000922F990F26FD2AC0A398809105018095AD
:1086F000847080930301809105018470809303014D
:10870000292F220F96FD18C0A3988091050180950E
:10871000847080930301809105018470809303012C
:1087200026FD16C0A39880910501809584708093E2
:1087300003010895A39A89CFA39AE7CFA39AD5CF2F
:10874000A39AC3CFA39AB1CFA39A9FCFA39A8DCF59
:10875000A39A809105018095847080930301089508
:108760002F923F925F927F929F92AF92BF92CF9251
:10877000DF92EF92FF920F931F93CF93DF937C01D1
:108780001B01942E69018AE0481709F47BC0A5E11A
:108790004A134EC0DB011296ED91FC9113971281A2
:1087A000C681D781A49A88E28A950000E9F700EE95
:1087B000010F80E1582E510E98E2792E88EF3DDFAF
:1087C000872D8A950000E9F7103208F046C0812F06
:1087D0008077806832DF812F8295807F2EDF872D22
:1087E0008A950000E9F780E828DF80E026DF872D02
:1087F0008A950000E9F78AEF20DF872D8A9500002F
:10880000E9F75E01B0E1AB0EB11C8881807F15DF16
:1088100089918295807F11DFCA15DB05B1F7872D1D
:108820008A950000E9F71F5F0F5F1511C7CFA49865
:108830009601492DB101C701DF91CF911F910F9191
:10884000FF90EF90DF90CF90BF90AF909F907F9080
:108850005F903F902F900C945332802F80778068E8
:10886000ECDE802F8295807FE8DE872D8A950000E0
:10887000E9F780E8E2DE80E8E0DE872D8A950000F7
:10888000E9F7B9CF9C9AA4989B9AA3988091040188
:1088900084608093040180910501809584708093A9
:1088A0000301A49AC8E28C2F8A950000E9F788E7B3
:1088B00090E00E94703188EFC0DE8C2F8A95000016
:1088C000E9F780E2BADE80E0B8DE8C2F8A950000FE
:1088D000E9F780E0B2DE80E8B0DE8C2F8A950000F8
:1088E000E9F780E0AADE80E1A8DE8C2F8A950000FF
:1088F000E9F78FE090E00E94703180E29EDE80E434
:108900009CDE8C2F8A950000E9F780E296DE80E6F7
:1089100094DECA950000E9F710E0D8E208E2812F62
:10892000807780688ADE812F8295807F86DE8D2F1A
:108930008A950000E9F780E880DE80E07EDE8D2FFA
:108940008A950000E9F78AEF78DE8D2F8A9500007E
:10895000E9F7C0E280E071DE80E06FDE9D2F9A953E
:108960000000E9F7C150B1F788EF67DE802F8A95E4
:108970000000E9F71F5F103209F0D1CF80E05DDE23
:1089800080EC5BDE88E28A950000E9F7A49850CF7E
:10899000CF93DF931F921F92CDB7DEB789839A835F
:1089A0000E946C7620E040E060E070E089819A816E
:1089B0000F900F90DF91CF910C941F770F93CF936F
:1089C000DF9361E081E00E943878D091EA05C0E051
:1089D000D11117C08091E905811104C00E94C67BA6
:1089E000811165C080912202882309F457C081E07B
:1089F0009091E905911180E004E024E04FEC56E20B
:108A00004BC0D130C1F48091E905813021F40E943E
:108A1000C67B811155C080912202882309F43EC093
:108A200081E09091E905913009F080E003E02EE3C8
:108A300046EC56E231C0D230B9F48091E90582307B
:108A400021F40E94C67B811144C0809122028823B8
:108A500029F181E09091E905923009F080E003E08E
:108A60002EE34DEB56E218C0D330C1F48091E905F6
:108A7000833021F40E94C67B811134C08091220290
:108A8000882361F081E09091E905933009F080E05E
:108A900003E02EE347EB56E26C2FE8DBCF5FDF5FAE
:108AA000C53009F095CF84E08093E80522C081E0CD
:108AB0000E9452778091B605882309F493CF19C09C
:108AC0008EE59CE665DF8091B605882309F4A3CF87
:108AD00010C080E891E75CDF8091B605882309F437
:108AE000B4CF07C088E995E753DF8091B6058823A6
:108AF00029F2DF91CF910F910895CF93DF93EC018D
:108B0000CB01BA010F94222C23E333E343E250E478
:108B10000F94BE2D0F94F42B6883DF91CF910895AD
:108B2000CF93DF93EC01CB01BA010F94222C2FE6F7
:108B300032E143E85AE30F94BE2D688379838A8338
:108B40009B83DF91CF9108956DE775E480EB95E409
:108B50000C94767760E975E483ED95E40C94767770
:108B60000F94222C23E333E343E250E40F94BE2D11
:108B70000F94F42B862F0D949C20CF93DF9300D07D
:108B80001F92CDB7DEB769837A838B839C8360E2C3
:108B9000CE0101960F94BE230F900F900F900F906F
:108BA000DF91CF9108950F94222C2FE632E143E814
:108BB0005AE30F94BE2DE1CF2F923F924F925F92D6
:108BC0006F927F928F929F92AF92BF92CF92DF92DD
:108BD000EF92FF920F931F93CF93DF93CDB7DEB742
:108BE00029970FB6F894DEBF0FBECDBF1C01798761
:108BF0006887CA01B901E982FA820B831C83DE828D
:108C0000CD82AF8220E030E04AE754E40F94BE2DDD
:108C10006B017C0120E030E040E057EC0F94832DA5
:108C200018162CF0C12CD12CE12C27ECF22EC70108
:108C3000B6010F94EF2B2B013C0120E030E04AE716
:108C400054E469817A818B819C810F94BE2D4B0104
:108C50005C0120E03EEF4FEF56E40F94802B87FD40
:108C600007C0812C9EEF992EAA24AA9496E4B92ECF
:108C700020E030E04AE754E4E885F98560817181BD
:108C8000828193810F94BE2D6B017C01C301B201DF
:108C90000F94222C9B01AC01C701B6010F94A62AA8
:108CA0000F94F42B69837A838B839C83C501B40171
:108CB0000F94EF2B7B018C01E418F50806091709C6
:108CC000FF81FF938D809E808AEAA82E85E4B82ECE
:108CD000C980DA80A301920168857985C1010E946B
:108CE00093760F9029960FB6F894DEBF0FBECDBFD6
:108CF000DF91CF911F910F91FF90EF90DF90CF9078
:108D0000BF90AF909F908F907F906F905F904F90AB
:108D10003F902F9008958F929F92AF92BF92CF92E3
:108D2000DF92EF92FF920F931F93CF93DF9361E057
:108D300081E00E943878D091EA05C0E0D11119C0D5
:108D40008091E905811104C00E94C67B8111C4C0D5
:108D500080912202882309F4B6C081E09091E90550
:108D6000911180E004E024E04AE057E26C2F7EDAC3
:108D7000AAC0D130E1F48091E905813021F40E944C
:108D8000C67B8111B2C080912202882309F49BC066
:108D900011E08091E905813009F010E08091FA0B33
:108DA0000F949C2000E09C0144EF56E289C0D23031
:108DB00009F58091E905823021F40E94C67B81117A
:108DC000C3C080912202882309F47DC011E0809104
:108DD000E905823009F010E06091FB0B7091FC0B0B
:108DE0008091FD0B9091FE0BC8DE00E09C0140EFEE
:108DF00056E266C0D33009F58091E905833021F44D
:108E00000E94C67B8111B9C080912202882309F497
:108E10005AC011E08091E905833009F010E06091BB
:108E2000FF0B7091000C8091010C9091020CA5DE5B
:108E300000E09C014CEE56E243C0D43001F5809135
:108E4000E905843021F40E94C67B8111AFC0809176
:108E500022028823C1F111E08091E905843009F0F4
:108E600010E06091030C7091040C8091050C9091BE
:108E7000060C83DE00E09C0148EE56E221C0D530AE
:108E800011F58091E905853021F40E94C67B81119E
:108E9000A6C0809122028823B1F011E08091E905FB
:108EA000853009F010E060912602709127028091D0
:108EB00028029091290261DE00E09C0144ED56E217
:108EC0006C2F812F07DACF5FDF5FC53009F036CF17
:108ED00086E08093E8059BC081E00E9452778091F4
:108EE000B605882309F434CF92C081E00E94BB7B91
:108EF0006091FA0B70E080E090E00F94202C29EC58
:108F000038EC48EC5EE30F94BE2D0F94F42B1F92C7
:108F1000812C912C44EAA42E45E4B42E6B0114E676
:108F2000E12EF12C00E010E020E030E0A9016AEF32
:108F30007BE08FEF96E20E9493760F908091B605CA
:108F4000882309F420CF63C081E00E94BB7BA12C61
:108F5000C12CD12C16E6E12EFE2C0EE111E420E00E
:108F600030E0A9016BEF7BE082EF96E225DE809195
:108F7000B605882309F425CF4AC081E00E94BB7B57
:108F8000A12CC12CD12C16E6E12EFE2C0EE111E411
:108F900020E030E0A9016FEF7BE08EEE96E20CDE80
:108FA0008091B605882309F42FCF31C081E00E945B
:108FB000BB7BA12CC12CD12C16E6E12EFE2C0EE1A0
:108FC00011E420E030E0A90163E07CE08AEE96E263
:108FD000F3DD8091B605882309F439CF18C081E00C
:108FE0000E94BB7BA12CC12CD12C16E6E12EFE2CBD
:108FF0000EE111E420E030E0A90166E272E08EEDBE
:1090000096E2DADD8091B605882309F442CFDF913C
:10901000CF911F910F91FF90EF90DF90CF90BF9075
:10902000AF909F908F900895CF93DF93EC01CB0189
:10903000BA010F94222C2AE037ED43E25CE30F944F
:10904000BE2D688379838A839B83DF91CF910895B6
:10905000CF93DF93EC01CB01BA010F94222C6883EC
:1090600079838A839B83DF91CF910895CF93DF9398
:10907000EC01CB01BA010F94222C20E030E048EC47
:1090800051E40F94BE2D688379838A839B83DF919B
:10909000CF910895CF93DF93EC01CB01BA010F94E8
:1090A000222C688379838A839B83DF91CF910895F3
:1090B000CF93DF93EC01CB01BA010F94222C20E077
:1090C00030E048EC51E40F94BE2D0F94F42B6883EC
:1090D00079838A839B83DF91CF910895CF93DF9328
:1090E000EC01CB01BA010F94222C20E030E048ECD7
:1090F00052E40F94BE2D0F94F42B688379838A83F6
:109100009B83DF91CF910895CF93DF93EC01CB0147
:10911000BA010F94222C2AE037ED43E25CE30F946E
:10912000BE2D688379838A839B83DF91CF910895D5
:10913000CF93DF93EC01CB01BA010F94222C2DECDD
:109140003CEC4CEC5DE30F94BE2D688379838A83FD
:109150009B83DF91CF91089564E178E481E399E402
:109160000C94767768E278E48FEA99E40C94767749
:109170006AE478E480EE98E40C94767766E378E429
:109180008EE499E40C94767768E578E48BEC99E4C6
:109190000C9476776EE678E48BE699E40C94767717
:1091A00064E878E487EF98E40C94767768E978E4EB
:1091B00084E199E40C9476770C9445F70C948CF741
:1091C000CF93DF9300D01F92CDB7DEB70F94222C40
:1091D00069837A838B839C83CE0101960F94FF244D
:1091E0000F900F900F900F90DF91CF910895CF9334
:1091F000DF9300D01F92CDB7DEB70F94222C2AE068
:1092000037ED43E25CE30F94BE2D69837A838B8351
:109210009C83CE0101960F9431250F900F900F90F3
:109220000F90DF91CF910895CF93DF9300D01F92DD
:10923000CDB7DEB70F94222C2DEC3CEC4CEC5DE36B
:109240000F94BE2D69837A838B839C83CE01019614
:109250000F94CE250F900F900F900F90DF91CF912C
:109260000895CF93DF9300D01F92CDB7DEB70F9450
:10927000222C2AE037ED43E25CE30F94BE2D698394
:109280007A838B839C83CE0101960F9482220F9068
:109290000F900F900F90DF91CF910895CF93DF93B0
:1092A00000D01F92CDB7DEB70F94222C20E030E023
:1092B00048EC51E40F94BE2D69837A838B839C83A1
:1092C000CE0101960F94FF240F900F900F900F90F6
:1092D000DF91CF910895CF93DF9300D01F92CDB748
:1092E000DEB70F94222C20E030E048EC52E40F94DB
:1092F000BE2D0F94F42B0F94202C69837A838B83DB
:109300009C83CE0101960F94FF240F900F900F9035
:109310000F90DF91CF910895CF92DF92EF92FF925D
:109320006B017C0120E030E0A9010F94802B87FDC8
:1093300005C020E030E040E05FE304C020E030E022
:1093400040E05FEBC701B6010F94A72A0F94EF2B03
:10935000CB01FF90EF90DF90CF900D9447210F94B9
:10936000222CDACFCF93DF9300D01F92CDB7DEB798
:109370000F94F42B0F94202C69837A838B839C8326
:10938000CE0101960F94FF240F900F900F900F9035
:10939000DF91CF9108950F94222C20E030E048EC2B
:1093A00051E40F94BE2DDECF81E00C9452776F9282
:1093B0007F928F929F92AF92BF92CF92DF92EF9265
:1093C000FF920F931F93CF93DF9300D01F92CDB7DF
:1093D000DEB761E081E00E9438786090EA05712C88
:1093E00061101AC08091E905811104C00E94C67BFA
:1093F000811159C180912202882309F44BC181E077
:109400009091E905911180E004E024E04DE758E2F5
:10941000672D0E9436413EC181E068122CC08091C8
:10942000E905813021F40E94C67B811143C18091FE
:109430002202882309F42EC111E08091E9058130D0
:1094400009F010E08091FB0D9091FC0DA091FD0DB5
:10945000B091FE0D89839A83AB83BC83CE010196C4
:109460000F94FF2400E09C0141E758E2672D812F13
:109470000E946A410FC182E068122CC08091E90508
:10948000823021F40E94C67B81114CC1809122025E
:10949000882309F4FFC011E08091E905823009F0CA
:1094A00010E08091FF0D9091000EA091010EB091FF
:1094B000020E89839A83AB83BC83CE0101960F94FD
:1094C000FF2400E09C014DE558E2672D812F0E94AA
:1094D0006A41E0C083E068122CC08091E9058330C6
:1094E00021F40E94C67B81114FC180912202882302
:1094F00009F4D0C011E08091E905833009F010E053
:109500008091030E9091040EA091050EB091060E6D
:1095100089839A83AB83BC83CE0101960F94FF2489
:1095200000E09C014BE458E2672D812F0E946A41C4
:10953000B1C084E0681227C08091E905843021F42D
:109540000E94C67B811158C180912202882309F4B0
:10955000A1C011E08091E905843009F010E060912C
:10956000C70D7091C80D8091C90D9091CA0D0F94CF
:10957000202CF8DE00E09C014DE358E2672D812F9E
:109580000E946A4187C085E0681227C08091E90582
:10959000853021F40E94C67B81116AC1809122022C
:1095A000882309F477C011E08091E905853009F03E
:1095B00010E06091CB0D7091CC0D8091CD0D90910C
:1095C000CE0D0F94202CCEDE00E09C014FE258E23D
:1095D000672D812F0E946A415DC086E0681227C016
:1095E0008091E905863021F40E94C67B81117CC1FF
:1095F00080912202882309F44DC011E08091E90591
:10960000863009F010E06091CF0D7091D00D8091FF
:10961000D10D9091D20D0F94202CA4DE00E09C017E
:1096200041E258E2672D812F0E946A4133C087E0F2
:10963000681230C08091E905873021F40E94C67B12
:10964000811187C180912202882321F111E080914C
:10965000E905873009F010E06091D30D7091D40DC9
:109660008091D50D9091D60D0F94202C0F94F42B52
:109670000F94202C69837A838B839C83CE0101967F
:109680000F94FF2400E09C0143E158E2672D812FF5
:109690000E946A417394639485E07812A1CE88E0B9
:1096A0008093E80591C180DE8091B605882309F496
:1096B000A1CE8AC181E00E94BB7B2AE037ED43E264
:1096C0005DE36091FB0D7091FC0D8091FD0D90911B
:1096D000FE0D0F94BE2D20E030E040E85FE30F94D4
:1096E000A62A0F94F42B1F92812C912C5EEBA52EB1
:1096F00058E4B52E6B0117E7E12E1FE0F12E00E0D4
:1097000010E021E030E040E050E06BEF7DE087E7E3
:1097100098E20E9493760F908091B605882309F411
:1097200086CE52C181E00E94BB7B20E030E048EC55
:1097300052E46091FF0D7091000E8091010E9091A6
:10974000020E0F94A62A0F94F42B1F92812C912CB9
:1097500038EBA32E38E4B32E6B011BE9E12E1FE793
:10976000F12E00E010E024E630E040E050E06FEF42
:109770007DE087E698E20E9493760F908091B6058F
:10978000882309F483CE20C181E00E94BB7B2AE0BC
:1097900037ED43E25DE36091030E7091040E80911A
:1097A000050E9091060E0F94BE2D20E030E040E8AB
:1097B0005FE30F94A62A0F94F42B1F92812C912C17
:1097C0009EEBA92E98E4B92E6B0117E7E12E1FE05E
:1097D000F12E00E010E021E030E040E050E063E0F6
:1097E0007EE084E598E20E9493760F908091B60522
:1097F000882309F47ACEE8C081E00E94BB7B6091A7
:10980000C70D7091C80D8091C90D9091CA0D0F942C
:10981000202C2AE037ED43E25DE30F94BE2D20E0DB
:1098200030E040E850E40F94A62A0F94F42B1F92E6
:10983000BCED8B2EB8E49B2E14ECA12E18E4B12EB7
:109840006B0114E7E12E1FE0F12E00E010E024E0B0
:1098500030E040E050E067EC7DE084E498E20E9474
:1098600093760F908091B605882309F46DCEACC035
:1098700081E00E94BB7B6091CB0D7091CC0D8091FB
:10988000CD0D9091CE0D0F94202C2AE037ED43E2C0
:109890005DE30F94BE2D20E030E040E850E40F94EB
:1098A000A62A0F94F42B1F92ECED8E2EE8E49E2E48
:1098B000F4ECAF2EF8E4BF2E6B0114E7E12E1FE0AD
:1098C000F12E00E010E024E030E040E050E06BECEE
:1098D0007DE086E398E20E9493760F908091B60532
:1098E000882309F45BCE70C081E00E94BB7B60914D
:1098F000CF0D7091D00D8091D10D9091D20D0F941C
:10990000202C2AE037ED43E25DE30F94BE2D0F9447
:10991000F42B1F923CED832E38E4932E44ECA42EBE
:1099200048E4B42E6B0118E7E12E1FE0F12E00E0B1
:1099300010E020E030E0A9016FEC7DE088E298E2E1
:109940000E9493760F908091B605882309F450CE3B
:109950003BC081E00E94BB7B6091D30D7091D40D20
:109960008091D50D9091D60D0F94202C2AE037EDE3
:1099700043E25CE30F94BE2D20E030E040E85FE37B
:109980000F94A62A0F94F42B1F928CED882E88E456
:10999000982E9AECA92E98E4B92E6B011DEDE12EBC
:1099A00013E0F12E00E010E021E030E040E050E074
:1099B00063ED7DE08AE198E20E9493760F908091BA
:1099C000B605882309F43ECE0F900F900F900F90AC
:1099D000DF91CF911F910F91FF90EF90DF90CF908B
:1099E000BF90AF909F908F907F906F9008950F934E
:1099F0001F93CF93DF9361E081E00E943878C0919C
:109A0000EA05D0E0C1111AC08091E905811104C0B6
:109A10000E94C67B8111E8C080912202882309F44C
:109A200061C081E09091E905911180E004E024E0BB
:109A300041E557E26D2F0E94364154C0C130D9F440
:109A40008091E905813021F40E94C67B8111D3C049
:109A500080912202882309F445C081E09091E905B4
:109A6000913009F080E003E02EE348E457E26D2FE7
:109A70000E94364137C0C230D1F48091E90582306E
:109A800021F40E94C67B8111C0C0809122028823EC
:109A900049F181E09091E905923009F080E003E01E
:109AA0002EE34BE357E26D2F0E9436411BC0C330BB
:109AB000C9F48091E905833021F40E94C67B8111AD
:109AC000AEC080912202882369F081E09091E9057F
:109AD000933009F080E003E02EE346E357E26D2F78
:109AE0000E9436410E94087781111DC0C430E9F4FC
:109AF0008091E905843021F40E94C67B811199C0D0
:109B000080912202882309F49EC081E09091E905AA
:109B1000943009F080E003E02EE34DE257E26D2F30
:109B20000E94364190C014E001C015E0C1131BC073
:109B30008091E9058C1304C00E94C67B811185C009
:109B400080912202882371F081E09091E9059C13B5
:109B500080E003E02EE344E257E26D2F0E9436419D
:109B60001C2F01C01C2F81E0810FC81318C08091E9
:109B7000E9058C1304C00E94C67B811170C08091DE
:109B80002202882361F081E09091E9059C1380E036
:109B900003E02EE348E157E26D2F0E94364182E058
:109BA000810FC81318C08091E9058C1304C00E946E
:109BB000C67B81115EC080912202882361F081E022
:109BC0009091E9059C1380E003E02EE34FE057E21B
:109BD0006D2F0E943641DF5FCF5FD53009F012CF85
:109BE0001D5F1093E8054EC0DFDB8091B60588232A
:109BF00009F412CF47C083E691E50E94C8448091E2
:109C0000B605882309F424CF3DC087ED99E40E946E
:109C1000C8448091B605882309F437CF33C081E367
:109C200093E50E94C8448091B605882309F449CF82
:109C300029C085E695E50E94C8448091B605882331
:109C400009F45ECF1FC015E08ECF8BE896E40E942A
:109C5000C8448091B605882309F472CF13C084E00C
:109C600090E50E94C8448091B605882309F487CF07
:109C700009C082ED9EE40E94C8448091B605882305
:109C800009F499CFDF91CF911F910F9108952F92F1
:109C90003F924F925F926F927F928F929F92AF927C
:109CA000BF92CF92DF92EF92FF920F931F93CF93C9
:109CB000DF9300D000D0CDB7DEB71C017E836D836B
:109CC00029013A01460120E030E040E057ECB201C2
:109CD000C3010F94832D18162CF0412C512C612CAC
:109CE00027EC01C0272DB201862D922F0F94EF2B68
:109CF0002B013C0120E03EEF4FEF56E4B701C801D5
:109D00000F94802B87FD06C0B12C9EEFF92E0FEF2C
:109D100016E401C0BE2CC301B2010F94222C9B019A
:109D2000AC01ED81FE8160817181828193810F940C
:109D3000A62A0F94F42B69837A838B839C836B2DE3
:109D40007F2DC8010F94EF2B7B018C01E418F508DF
:109D500006091709AF9282EBA82E88E4B82EC980B5
:109D6000DA80A30192016D817E81C1010E94937608
:109D70000F9026960FB6F894DEBF0FBECDBFDF91D1
:109D8000CF911F910F91FF90EF90DF90CF90BF90F8
:109D9000AF909F908F907F906F905F904F903F908B
:109DA0002F9008956F927F928F929F92AF92BF9261
:109DB000CF92DF92EF92FF920F931F93CF93DF9397
:109DC00000D01F92CDB7DEB761E081E00E94387805
:109DD0006090EA05712C61101AC08091E90581112B
:109DE00004C00E94C67B811198C080912202882302
:109DF00009F48AC081E09091E905911180E004E0C6
:109E000024E046E859E2672D0E9436417DC081E09A
:109E100068122CC08091E905813021F40E94C67B34
:109E2000811182C080912202882309F46DC011E063
:109E30008091E905813009F010E080915D0D9091ED
:109E40005E0DA0915F0DB091600D89839A83AB8305
:109E5000BC83CE0101960F94822200E09C0142E770
:109E600059E2672D812F0E946A414EC082E068123C
:109E700025C08091E905823021F40E94C67B8111C2
:109E800081C080912202882309F43EC011E08091B4
:109E9000E905823009F010E06091C40B7091C50BA8
:109EA0008091C60B9091C70B37DA00E09C014EE51C
:109EB00059E2672D812F0E946A4126C083E0681213
:109EC00023C08091E905833021F40E94C67B811173
:109ED00071C0809122028823B9F011E08091E905D8
:109EE000833009F010E06091C80B7091C90B80912C
:109EF000CA0B9091CB0B10DA00E09C014EE459E2C2
:109F0000672D812F0E946A417394639485E07812D3
:109F100062CF84E08093E80564C046DA8091B6059C
:109F2000882309F462CF5DC020E030E048EC52E4C1
:109F300060915D0D70915E0D80915F0D9091600D4F
:109F40000F94BE2D0F94F42B1F92812C912C2CEA90
:109F5000A22E28E4B22E6B01EE24EA941FE7F12E24
:109F600000E010E020E030E0A9016DE57DE08CE745
:109F700099E20E9493760F908091B605882309F4A8
:109F800051CF2FC081E00E94BB7BA12CC12CD12CD2
:109F9000E12CF12C08E413E420E030E0A90164ECAA
:109FA0007BE088E699E273DE8091B605882309F4A8
:109FB00068CF17C081E00E94BB7BA12CC12CD12CA3
:109FC000E12CF12C08E413E420E030E0A90168EC76
:109FD0007BE086E599E25BDE8091B605882309F493
:109FE00078CF0F900F900F900F90DF91CF911F912E
:109FF0000F91FF90EF90DF90CF90BF90AF909F9028
:10A000008F907F906F9008956F927F928F929F9222
:10A01000AF92BF92CF92DF92EF92FF920F931F9376
:10A02000CF93DF9300D01F92CDB7DEB761E081E020
:10A030000E9438786090EA05712C61101AC08091F6
:10A04000E905811104C00E94C67B8111BDC08091C9
:10A050002202882309F4B0C081E09091E9059111B2
:10A0600080E004E024E04CE359E2672D0E94364191
:10A07000A3C081E0681223C08091E905813021F4FA
:10A080000E94C67B8111A7C080912202882309F417
:10A0900093C080918A0D811103C02CE239E202C085
:10A0A00020E339E281E09091E905913009F080E008
:10A0B00001E043E259E2672D0E946A417DC082E0DF
:10A0C000681225C08091E905823021F40E94C67B88
:10A0D00081118FC080912202882309F46DC011E0A4
:10A0E0008091E905823009F010E060917902709169
:10A0F0007A0280917B0290917C020ED900E09C0153
:10A1000045E159E2672D812F0E946A4155C083E0E5
:10A11000681225C08091E905833021F40E94C67B36
:10A1200081117CC080912202882309F445C011E08E
:10A130008091E905833009F010E060917D02709113
:10A140007E0280917F0290918002E6D800E09C011F
:10A1500047E059E2672D812F0E946A412DC084E0BB
:10A1600068122AC08091E905843021F40E94C67BE0
:10A17000811169C0809122028823F1F011E0809161
:10A18000E905843009F010E0809175029091760223
:10A19000A0917702B091780289839A83AB83BC83C4
:10A1A000CE0101960F94822200E09C0147EF58E215
:10A1B000672D812F0E946A417394639485E0781221
:10A1C0003CCF7092E8056CC0EFD88091B60588232B
:10A1D00009F43DCF65C040E050E06AE87DE083E3EC
:10A1E00099E20E94FA768091B605882309F44CCF53
:10A1F00057C0A12CC12CD12CE12CF12C01E913E486
:10A2000020E030E0A90169E772E08CE199E23FDDEE
:10A210008091B605882309F45DCF42C0A12CC12CE2
:10A22000D12CE12CF12C01E913E420E030E0A9016C
:10A230006DE772E08EE099E22ADD8091B605882311
:10A2400009F470CF2DC020E030E048EC52E460917A
:10A2500075027091760280917702909178020F9446
:10A26000BE2D0F94F42B1F92812C912C8CEAA82EDA
:10A2700088E4B82E6B0118EEE12E13E0F12E00E019
:10A2800010E020E030E0A90165E772E08FEF98E28E
:10A290000E9493760F908091B605882309F46ACFC7
:10A2A0000F900F900F900F90DF91CF911F910F9112
:10A2B000FF90EF90DF90CF90BF90AF909F908F90E6
:10A2C0007F906F900895AF92CF92DF92EF92FF92BE
:10A2D0000F931F93CF93DF9361E081E00E94387862
:10A2E000D091EA05C0E0D1111AC08091E905811131
:10A2F00004C00E94C67B811109C18091220288237B
:10A3000009F4FBC081E09091E905911180E004E03F
:10A3100024E045EE58E26C2F0E943641EEC0D13069
:10A3200031F58091E905813021F40E94C67B8111CD
:10A33000F5C080912202882309F4DFC011E08091EA
:10A34000E905813009F010E06091EB0D7091EC0DA2
:10A350008091ED0D9091EE0D0E948C4900E09C01E2
:10A3600047ED58E26C2F812F0E946A41C6C0D2305F
:10A3700031F58091E905823021F40E94C67B81117C
:10A38000E7C080912202882309F4B7C011E08091D0
:10A39000E905823009F010E06091EF0D7091F00D49
:10A3A0008091F10D9091F20D0E948C4900E09C018A
:10A3B00049EC58E26C2F812F0E946A419EC0D33035
:10A3C00031F58091E905833021F40E94C67B81112B
:10A3D000D9C080912202882309F48FC011E08091B6
:10A3E000E905833009F010E06091F30D7091F40DF0
:10A3F0008091F50D9091F60D0E948C4900E09C0132
:10A400004BEB58E26C2F812F0E946A4176C0D4300A
:10A4100031F58091E905843021F40E94C67B8111D9
:10A42000CBC080912202882309F467C011E080919B
:10A43000E905843009F010E06091F70D7091F80D96
:10A440008091F90D9091FA0D0E948C4900E09C01D9
:10A450004DEA58E26C2F812F0E946A414EC0D530E0
:10A4600031F58091E905853021F40E94C67B811188
:10A47000BDC080912202882309F43FC011E0809181
:10A48000E905853009F010E06091070E7091080E23
:10A490008091090E90910A0E0E948C4900E09C0167
:10A4A00043EA58E26C2F812F0E946A4126C0D630C1
:10A4B00021F58091E905863021F40E94C67B811147
:10A4C000AEC0809122028823C1F011E08091E9059D
:10A4D000863009F010E060910B0E70910C0E8091A7
:10A4E0000D0E90910E0E0E948C4900E09C014FE8E9
:10A4F00058E26C2F812F0E946A41CF5FDF5FC53029
:10A5000009F0F1CE87E08093E805A1C00E94D4490C
:10A510008091B605882309F4F0CE99C081E00E94AD
:10A52000BB7BA12CC12CD12CE12C10ECF12E09E726
:10A5300014E420E030E040E85FE36BEE7DE08EED78
:10A5400098E2A5DB8091B605882309F4F2CE7FC09E
:10A5500081E00E94BB7BA12CC12CD12CE12C10EC02
:10A56000F12E09E714E420E030E040E85FE36FEE0D
:10A570007DE080ED98E28BDB8091B605882309F4BD
:10A5800000CF65C081E00E94BB7BA12CC12CD12CE7
:10A59000E12C10ECF12E09E714E420E030E040E873
:10A5A0005FE363EF7DE082EC98E271DB8091B605BA
:10A5B000882309F40ECF4BC081E00E94BB7BA12C05
:10A5C000C12CD12CE12C10ECF12E09E714E420E091
:10A5D00030E040E85FE367EF7DE084EB98E257DB33
:10A5E0008091B605882309F41CCF31C081E00E9418
:10A5F000BB7BA12CC12CD12CE12C10ECF12E09E756
:10A6000014E420E030E0A90167E07EE088EA98E207
:10A610003EDB8091B605882309F42BCF18C081E07A
:10A620000E94BB7BA12CC12CD12CE12C10ECF12E73
:10A6300009E714E420E030E0A9016BE07EE089E95D
:10A6400098E225DB8091B605882309F43ACFDF91A3
:10A65000CF911F910F91FF90EF90DF90CF90AF902F
:10A6600008956F927F928F929F92AF92BF92CF92F6
:10A67000DF92EF92FF920F931F93CF93DF9300D05F
:10A680001F92CDB7DEB761E081E00E94387860901C
:10A69000EA05712C61101AC08091E905811104C08E
:10A6A0000E94C67B8111C2C080912202882309F4D6
:10A6B000B5C081E09091E905911180E004E024E0CB
:10A6C00041E058E2672D0E943641A8C081E068123F
:10A6D00026C08091E905813021F40E94C67B81115A
:10A6E000ADC080912202882309F498C011E08091C6
:10A6F000E905813009F010E06091970D7091980D97
:10A700008091990D90919A0D0E948C4900E09C01D6
:10A7100041EF57E2672D812F0E946A417FC082E09E
:10A72000681226C08091E905823021F40E94C67B20
:10A7300081119EC080912202882309F46FC011E02C
:10A740008091E905823009F010E060919B0D7091D5
:10A750009C0D80919D0D90919E0D0E948C4900E072
:10A760009C0141EE57E2672D812F0E946A4156C03D
:10A7700083E068122CC08091E905833021F40E94A7
:10A78000C67B81118FC080912202882309F446C0C4
:10A7900011E08091E905833009F010E080919F0D70
:10A7A0009091A00DA091A10DB091A20D89839A83E3
:10A7B000AB83BC83CE0101960F94312500E09C0150
:10A7C00041ED57E2672D812F0E946A4127C084E046
:10A7D000681224C08091E905843021F40E94C67B70
:10A7E000811198C0809122028823C1F011E08091EC
:10A7F000E905843009F010E06091A30D7091A40D7B
:10A800008091A50D9091A60D0E948C4900E09C01BD
:10A8100041EC57E2672D812F0E946A417394639443
:10A8200085E0781237CF7092E8058DC00E94D44938
:10A830008091B605882309F437CF85C081E00E9456
:10A84000BB7BA12CC12CD12CE12C10E8F12E07E709
:10A8500014E420E030E040E85FE367E97DE089EF61
:10A8600097E215DA8091B605882309F43ACF6BC0D8
:10A8700081E00E94BB7BA12CC12CD12CE12C10E8E3
:10A88000F12E07E714E420E030E040E85FE36BE9F5
:10A890007DE089EE97E2FBD98091B605882309F423
:10A8A00049CF51C081E00E94BB7B20E030E048EC02
:10A8B00052E460919F0D7091A00D8091A10D909137
:10A8C000A20D0F94BE2D20E030E040E251E40F9441
:10A8D000A62A0F94F42B1F92812C912C90EDA92E77
:10A8E00098E4B92E6B0115EFE12E1FE7F12E00E081
:10A8F00010E02AE030E040E050E06FE97DE089EDD3
:10A9000097E20E9493760F908091B605882309F410
:10A910003ACF19C081E00E94BB7BA12CC12CD12C65
:10A92000E12C10E8F12E07E714E420E030E040E8E5
:10A930005FE363EA7DE089EC97E2A9D98091B605EF
:10A94000882309F44FCF0F900F900F900F90DF9155
:10A95000CF911F910F91FF90EF90DF90CF90BF901C
:10A96000AF909F908F907F906F9008952F923F921D
:10A970004F925F926F927F928F929F92AF92BF920F
:10A98000CF92DF92EF92FF920F931F93CF93DF93BB
:10A99000CDB7DEB729970FB6F894DEBF0FBECDBF97
:10A9A0001C0179876887CA01B901E982FA820B83A1
:10A9B0001C83DE82CD82AF8220E030E040E251E4B1
:10A9C0000F94BE2D6B017C0120E030E040E057EC9D
:10A9D0000F94832D18162CF0C12CD12CE12C27ECD0
:10A9E000F22EC701B6010F94EF2B2B013C0120E0A2
:10A9F00030E040E251E469817A818B819C810F943F
:10AA0000BE2D4B015C0120E03EEF4FEF56E40F946A
:10AA1000802B87FD07C0812C9EEF992EAA24AA9433
:10AA200096E4B92E20E030E040E251E4E885F98573
:10AA300060817181828193810F94BE2D6B017C01B5
:10AA4000C301B2010F94222C9B01AC01C701B601D6
:10AA50000F94A62A0F94F42B69837A838B839C83AB
:10AA6000C501B4010F94EF2B7B018C01E418F508AC
:10AA700006091709FF81FF938D809E8086EDA82E21
:10AA800088E4B82EC980DA80A301920168857985AF
:10AA9000C1010E9493760F9029960FB6F894DEBFFD
:10AAA0000FBECDBFDF91CF911F910F91FF90EF901F
:10AAB000DF90CF90BF90AF909F908F907F906F90DE
:10AAC0005F904F903F902F9008959F92AF92BF92CA
:10AAD000CF92DF92EF92FF920F931F93CF93DF936A
:10AAE00000D01F92CDB7DEB761E081E00E943878D8
:10AAF0009090EA05B12C91101AC08091E90581115E
:10AB000004C00E94C67B8111D4C080912202882398
:10AB100009F4C7C081E09091E905911180E004E05B
:10AB200024E04FEA57E26B2D0E943641BAC081E023
:10AB300098122CC08091E905813021F40E94C67BD7
:10AB40008111BFC080912202882309F4AAC011E0BC
:10AB50008091E905813009F010E08091DB0D909142
:10AB6000DC0DA091DD0DB091DE0D89839A83AB835E
:10AB7000BC83CE0101960F94CE2500E09C014BE9E9
:10AB800057E26B2D812F0E946A418BC082E09812A0
:10AB90002CC08091E905823021F40E94C67B81118E
:10ABA000ACC080912202882309F47BC011E080911F
:10ABB000E905823009F010E08091DF0D9091E00D01
:10ABC000A091E10DB091E20D89839A83AB83BC83A0
:10ABD000CE0101960F94CE2500E09C0147E857E294
:10ABE0006B2D812F0E946A415CC083E098122CC0BB
:10ABF0008091E905833021F40E94C67B811199C0C0
:10AC000080912202882309F44CC011E08091E9056B
:10AC1000833009F010E08091E30D9091E40DA09154
:10AC2000E50DB091E60D89839A83AB83BC83CE0199
:10AC300001960F94CE2500E09C0143E757E26B2D6F
:10AC4000812F0E946A412DC084E098122AC0809111
:10AC5000E905843021F40E94C67B811186C0809171
:10AC600022028823F1F011E08091E905843009F097
:10AC700010E08091E70D9091E80DA091E90DB09161
:10AC8000EA0D89839A83AB83BC83CE0101960F942E
:10AC9000CE2500E09C014FE557E26B2D812F0E94ED
:10ACA0006A41B394939485E0B81225CFB092E80539
:10ACB00077C00E94D4498091B605882309F425CF36
:10ACC0006FC081E00E94BB7BA12C6EEDC62E68E4B4
:10ACD000D62EE12C1CE3F12E0CE116E420E030E04E
:10ACE00040EA50E46BED7DE085EA97E23FDE80913B
:10ACF000B605882309F426CF53C081E00E94BB7BB0
:10AD0000A12C4EEDC42E48E4D42EE12C1CE3F12EF0
:10AD10000CE116E420E030E040EA50E46FED7DE025
:10AD200081E997E223DE8091B605882309F439CFC3
:10AD300037C081E00E94BB7BA12C2EEDC22E28E4FF
:10AD4000D22EE12C1CE3F12E0CE116E420E030E0E1
:10AD500040EA50E463EE7DE08DE797E207DE809104
:10AD6000B605882309F44CCF1BC081E00E94BB7B51
:10AD7000A12C8EEDC82E88E4D82EE12C1CE3F12EF8
:10AD80000CE116E420E030E040EA50E467EE7DE0BC
:10AD900089E697E2EBDD8091B605882309F45FCF61
:10ADA0000F900F900F900F90DF91CF911F910F9107
:10ADB000FF90EF90DF90CF90BF90AF909F9008955D
:10ADC0000F93CF93DF9361E081E00E943878C091C8
:10ADD000EA05D0E0C11118C08091E905811104C0D5
:10ADE0000E94C67B8111B5C080912202882361F048
:10ADF00081E09091E905911180E004E024E047EFC3
:10AE000059E26D2F0E9436418091380D877087304E
:10AE100009F058C0C130D9F48091E905813021F49E
:10AE20000E94C67B81119EC080912202882309F472
:10AE3000C1C081E09091E905913009F080E003E024
:10AE40002EE340EF59E26D2F0E943641B3C0C2306D
:10AE5000D9F48091E905823021F40E94C67B8111EA
:10AE60008BC080912202882309F4A4C081E09091D4
:10AE7000E905923009F080E003E02EE349EE59E263
:10AE80006D2F0E94364196C0C330D1F58091E905FF
:10AE9000833021F40E94C67B811178C08091220208
:10AEA000882309F487C081E09091E905933009F087
:10AEB00080E003E02EE342EE59E26D2F0E9436411E
:10AEC00084E03EC0C130F1F48091E905813021F485
:10AED0000E94C67B811164C080912202882309F4FC
:10AEE0006BC081E09091E905913009F080E000E2CB
:10AEF0002EE344ED59E26D2F0E94364182E020C0DE
:10AF000084E001C082E0C8131BC08091E9058C1366
:10AF100004C00E94C67B811151C080912202882307
:10AF200071F081E09091E9059C1380E003E02EE34D
:10AF30004AEC59E26D2F0E9436418C2F01C08C2FB4
:10AF4000DF5FCF5FD53009F045CF8F5F8093E80595
:10AF50003EC081E00E9452778091B605882309F4B3
:10AF600043CF35C08DE09CE50E94C8448091B60572
:10AF7000882309F459CF2BC082E19CE50E94C84484
:10AF80008091B605882309F46CCF21C087E19CE548
:10AF90000E94C8448091B605882309F47FCF17C06A
:10AFA0008EED99E20E9491768091B605882309F48E
:10AFB00093CF0DC084E0C4CF82E0C2CF8CE19CE58A
:10AFC0000E94C8448091B605882309F4A6CFDF917A
:10AFD000CF910F910895CF92DF92EF92FF92CF938E
:10AFE000C82F0E94BC2B6B017C0124EA30E74DE79F
:10AFF0005FE36091010670910206809103069091D3
:10B0000004060F94802B87FD05C04AEF50E060E0F6
:10B0100070E003C040E050E0BA01C40ED51EE61E49
:10B02000F71EC092FD05D092FE05E092FF05F0925A
:10B030000006C0932302CF91FF90EF90DF90CF9056
:10B0400008952F923F924F925F926F927F928F92CC
:10B050009F92AF92BF92CF92DF92EF92FF921F9397
:10B06000CF93DF93CDB7DEB728970FB6F894DEBF46
:10B070000FBECDBF1C01162F0E94C67B882331F066
:10B080001092180680E00E945277DDC020911006D1
:10B09000309111063E832D83232B09F4A0C0E4E0F8
:10B0A0001E9FC001112498878F83FC01EB59FD4F2F
:10B0B00080809180A280B38020E030E04AE754E4B1
:10B0C000C501B4010F94A62A2B013C0120E030E019
:10B0D0004AE754E4C501B4010F94A72A6B017C012F
:10B0E00080915E028823B9F1113029F198F0123075
:10B0F00091F540905602509057026090580270901F
:10B100005902C0905A02D0905B02E0905C02F0902D
:10B110005D0221C040904602509047026090480274
:10B1200070904902C0904A02D0904B02E0904C02CD
:10B13000F0904D0210C040904E0250904F0260902F
:10B14000500270905102C0905202D0905302E09091
:10B150005402F09055022D813E81B901330F880BC6
:10B16000990B0F94222C20910106309102064091F8
:10B170000306509104060F94BE2D9B01AC01C5013E
:10B18000B4010F94A72A9B01AC018F8198858B593C
:10B190009D4F5C01FC0120833183428353838D8169
:10B1A0009E8197FF0CC0C301B2010F94832D181626
:10B1B0008CF4F50140825182628273820BC0C70118
:10B1C000B6010F94802B87FF05C0F501C082D182A4
:10B1D000E282F382812FFFDE81E0809322021092CF
:10B1E00011061092100680912202882361F124E05A
:10B1F000129FF0011124EB59FD4F80819181A281B2
:10B20000B38189839A83AB83BC832DEC3CEC4CECFB
:10B210005DE36091010670910206809103069091B2
:10B2200004060F94832D87FD05C0CE0101960F946F
:10B23000472305C060E2CE0101960F94BE23BC01F6
:10B24000C1010E94CF4128960FB6F894DEBF0FBE11
:10B25000CDBFDF91CF911F91FF90EF90DF90CF9006
:10B26000BF90AF909F908F907F906F905F904F9026
:10B270003F902F90089560E088E79AE2E2CE61E087
:10B2800081E79AE2DECE62E08AE69AE2DACECF93F6
:10B29000DF9300D01F92CDB7DEB70E94C67B882314
:10B2A00031F01092180680E00E94527757C06091EA
:10B2B0001006709111066115710569F1072E000CD9
:10B2C000880B990B0F94222C2091010630910206D5
:10B2D00040910306509104060F94BE2D9B01AC01D2
:10B2E0006091710270917202809173029091740268
:10B2F0000F94A72A60937102709372028093730275
:10B300009093740283E067DE81E0809322021092C2
:10B31000110610921006809122028823F9F02091E4
:10B320001E0530911F054091200550912105609127
:10B3300071027091720280917302909174020F9465
:10B34000A62A69837A838B839C83CE0101960F940E
:10B350004723BC018EEF99E20E94CF410F900F90DE
:10B360000F900F90DF91CF91089521E02093180660
:10B37000609301067093020680930306909304067F
:10B3800020E040E060E070E080911C0590911D0598
:10B390000C941F7760E070E080E291E4E6CF60E01B
:10B3A00070E080E89FE3E1CF6DEC7CEC8CEC9DE3FA
:10B3B000DCCF6DEC7CEC8CEC9CE3D7CF8F929F9232
:10B3C000AF92BF92CF92DF92EF92FF920F931F93B3
:10B3D000CF93DF93CDB7DEB76E970FB6F894DEBF8D
:10B3E0000FBECDBFD82E70931D0560931C0561E084
:10B3F00081E00E943878F090EA058CE0C82EE12CBC
:10B4000091E028E0A22E2AE2B22E9E012F5F3F4F4C
:10B41000490131E0D31659F1D31628F082E0D8164D
:10B4200009F449C06CC0F110D2C0992389F0809111
:10B43000E90518166CF020911006309111062F5F67
:10B440003F4F30931106209310068F5F8093E905DC
:10B4500080912202882309F432C100E010E021E04B
:10B4600041E063E67AE28E2D0E94D34028C1F110BC
:10B47000AEC0992389F08091E90518166CF02091EF
:10B480001006309111062F5F3F4F30931106209325
:10B4900010068F5F8093E90580912202882309F4CA
:10B4A00011C100E010E021E041E06CE57AE28E2D70
:10B4B0000E94D34007C1F1108AC0992389F080917E
:10B4C000E90518166CF020911006309111062F5FD7
:10B4D0003F4F30931106209310068F5F8093E9054C
:10B4E00080912202882309F40BC100E010E021E0E2
:10B4F00041E065E57AE28E2D0E94D34001C1409182
:10B5000071025091720260917302709174024093C3
:10B510001E0550931F056093200570932105F110BF
:10B5200020C0992389F08091E90518166CF02091CC
:10B530001006309111062F5F3F4F30931106209374
:10B5400010068F5F8093E90580912202882349F0DD
:10B5500000E010E021E041E06BE47AE28E2D0E94F1
:10B56000D34093E0D91233C06091850C7091860C62
:10B570008091870C9091880C20914D0C211127C04F
:10B580000F94EF2B20913602309137026217730728
:10B59000F4F421E0F21219C08091E905813021F420
:10B5A0000E94C67B8111C0C080912202882369F06D
:10B5B00081E09091E905913009F080E004E024E019
:10B5C0004BE35AE26E2D0E94364182E0A2C031E088
:10B5D000F3121BC08091E905813021F40E94C67BE3
:10B5E0008111ABC080912202882309F468C081E0F8
:10B5F0009091E905913009F080E004E024E041E316
:10B600005AE26E2D0E9436415AC082E0F8121BC0E9
:10B610008091E905823021F40E94C67B811196C099
:10B6200080912202882309F49BC081E09091E90572
:10B63000923009F080E003E02EE347E25AE26E2DFB
:10B640000E9436418DC093E0F9121BC08091E9053C
:10B65000833021F40E94C67B811186C08091220232
:10B66000882309F4C3C081E09091E905933009F083
:10B6700080E003E02EE34EE15AE26E2D0E94364157
:10B68000B5C024E0F2121BC08091E905843021F49A
:10B690000E94C67B811172C080912202882309F426
:10B6A000A5C081E09091E905943009F080E003E0C5
:10B6B0002EE343E15AE26E2D0E94364197C032E0FC
:10B6C000D31611F085E025C085E0F81219C08091ED
:10B6D000E905853021F40E94C67B811159C0809113
:10B6E0002202882369F081E09091E905953009F004
:10B6F00080E003E02EE342E15AE26E2D0E943641E3
:10B7000080912202882321F095E0F91609F44AC0BD
:10B7100086E0E394F3942CE0C20E90E035E0E3126F
:10B7200078CE8093E80566C081E00E9452778091D0
:10B73000B605882309F438CF5DC081E00E945277B6
:10B740008091B605882309F44DCF54C08AEC99E561
:10B750000E94C8448091B605882309F461CF4AC08D
:10B7600082E0D812AFCFCCCF8FEC99E50E94C844CD
:10B770008091B605882309F471CF3CC084ED99E52A
:10B780000E94C8448091B605882309F485CF32C051
:10B7900089ED99E50E94C8448091B605882309F493
:10B7A0009ECF28C06C2D86E00E94F7378E010B5E7D
:10B7B0001F4F23E041E06DEC7CEC8CEC9CE30F949C
:10B7C0002B2F9F938F93BF92AF929F928F920F9444
:10B7D0003D34B4018EED93E00E94FE360F900F9041
:10B7E0000F900F900F900F9086E093CF92E0D912B8
:10B7F00069CF86CF6E960FB6F894DEBF0FBECDBF71
:10B80000DF91CF911F910F91FF90EF90DF90CF903C
:10B81000BF90AF909F908F9008954FEF6BE379E5C5
:10B8200080E0CCCD4FEF6FE379E581E0C7CD4FEFFE
:10B8300063E479E582E0C2CD4FEF67E479E583E028
:10B84000BDCD0F93CF93DF9361E081E00E94387804
:10B85000D091EA05C0E0D1111AC08091E9058111AB
:10B8600004C00E94C67B81116FC080912202882390
:10B8700009F461C081E09091E905911180E004E054
:10B8800024E045EC59E26C2F0E94364154C0D1307F
:10B89000D9F48091E905813021F40E94C67B8111A1
:10B8A0005CC080912202882309F445C081E0909118
:10B8B000E905913009F080E003E02EE34BEB59E21B
:10B8C0006C2F0E94364137C0D230D1F48091E90507
:10B8D000823021F40E94C67B811149C080912202EE
:10B8E000882349F181E09091E905923009F080E0E8
:10B8F00000E22EE34DEA59E26C2F0E9436411BC054
:10B90000D330C9F48091E905833021F40E94C67BCD
:10B91000811137C080912202882369F081E09091E3
:10B92000E905933009F080E000E22EE348E959E2AE
:10B930006C2F0E943641CF5FDF5FC53009F08BCF9F
:10B9400084E08093E80525C081E00E9452778091D1
:10B95000B605882309F489CF1CC080EE96E50E94C5
:10B96000C8448091B605882309F49BCF12C087EBA9
:10B9700099E20E9491768091B605882309F4AECFB2
:10B9800008C089EA99E20E9491768091B6058823E1
:10B9900009F2DF91CF910F910895CF92DF92EF924C
:10B9A000FF920F931F938091A708811103C089EE26
:10B9B00098E002C087EA98E024ECC22E2AE2D22E58
:10B9C0007C0107EB1AE224EF3CE547EF5CE560EB16
:10B9D0007AE28AEA9AE20E94C1781F910F91FF9061
:10B9E000EF90DF90CF90089580E00C94527789EE2D
:10B9F00098E00E949A860E944B770C94D2810E9414
:10BA00003C8B21E030E0811102C020E030E0309337
:10BA10001106209310061092EA0581E08093B60586
:10BA200083E0809322020895EF92FF920F931F9379
:10BA3000CF93DF9380911206882331F00E944C8CC3
:10BA4000909323058093220561E081E00E9438787D
:10BA5000C091EA05D0E0C11118C08091E9058111BB
:10BA600004C00E94C67B811197C080912202882366
:10BA700061F081E09091E905911180E004E024E01B
:10BA800045EA5AE26D2F0E9436418091F60885FD05
:10BA90001FC083FF1DC0C130C9F48091E90581300A
:10BAA00021F40E94C67B811180C0809122028823EC
:10BAB00069F081E09091E905913009F080E000E2C1
:10BAC0002EE341EA5AE26D2F0E94364192E001C016
:10BAD00091E080912202882309F456C0E12CF12CD8
:10BAE00011E01C0F2091220530912305E216F30688
:10BAF00008F04AC0C91343C0C901019760E070E073
:10BB00008E199F090E940F889091F6088091E9058F
:10BB100094FF1CC08C1350C00E94C67B882309F47C
:10BB20004BC089EE98E00E94E18A1092EA0582E01B
:10BB300090E0909311068093100681E08093B60503
:10BB40001092130683E08093220254C08C1304C029
:10BB50000E94C67B81113FC080912202882369F038
:10BB600081E09091E9059C1380E000E02DE436E14E
:10BB70004FE75AE26D2F0E94C942912F01C09F5F8B
:10BB80008FEFE81AF80AAECFDF5FCF5FD53009F04C
:10BB900062CF9093E8052EC081E00E945277809199
:10BBA000B605882309F461CF25C029DF8091B60549
:10BBB000882309F47ACF1EC0809122028823E9F2FB
:10BBC00081E09091E9059C1380E001E02DE436E1ED
:10BBD00040E95AE2CFCF0E946C7620E040E060E07E
:10BBE00070E08DEC9CE50E941F778091B60588235C
:10BBF00009F4B2CFDF91CF911F910F91FF90EF9099
:10BC00000895CF93DF93EC01CB01BA010F94222C5E
:10BC10000F94EF2B79836883DF91CF91089561E0D2
:10BC20007EE588E99EE50C9476770F931F93CF937A
:10BC3000DF9361E081E00E943878C091EA05D0E0AE
:10BC400081E0C11122C0882389F08091E90518168E
:10BC50006CF020911006309111062F5F3F4F30930A
:10BC60001106209310068F5F8093E90580912202D0
:10BC7000882309F441C000E010E020E041E069E2DF
:10BC80007CE28D2F0E94D34037C0C130D1F4809127
:10BC9000E905813021F40E94C67B811137C0809173
:10BCA0002202882349F181E09091E905913009F061
:10BCB00080E000E22EE34EE15CE26D2F0E9436410F
:10BCC0001BC0C230C9F48091E905823021F40E9482
:10BCD000C67B811122C080912202882369F081E015
:10BCE0009091E905923009F080E000E22EE34AE00D
:10BCF0005CE26D2F0E943641DF5FCF5F80E0D53080
:10BD000009F09FCF83E08093E8050DC0C093CC0B72
:10BD10008091B605882319F206C0C093CC0B8091A0
:10BD2000B6058823C1F2DF91CF911F910F9108953D
:10BD30000F94222C0F94EF2BCB010D944721EF92FF
:10BD4000FF920F931F93CF93DF93CDB7DEB72B975F
:10BD50000FB6F894DEBF0FBECDBF7C014091250524
:10BD6000842F042E000C990B20912605223051F0CF
:10BD7000233019F028E53CE20AC047FF06C024E65C
:10BD80003CE205C026E73CE202C02DE63CE29F9380
:10BD90004F933F932F938E010F5F1F4F1F930F936E
:10BDA0000F943D3440913402509135024F50510967
:10BDB00097010F900F900F900F900F900F904E15CE
:10BDC0005F050CF49A0130938A0C2093890C80E073
:10BDD0000E94BCAEC8010E949E782B960FB6F894C4
:10BDE000DEBF0FBECDBFDF91CF911F910F91FF90AE
:10BDF000EF900895E091250587E1E802F001112414
:10BE0000EF57F34F808591859ACF7F928F929F92C3
:10BE1000AF92BF92CF92DF92EF92FF920F931F9358
:10BE2000CF93DF93782E809326056093250561E0FC
:10BE300081E00E943878D091EA05C0E081E0D1111C
:10BE40002EC0882389F08091E90518166CF02091A6
:10BE50001006309111062F5F3F4F3093110620934B
:10BE600010068F5F8093E90580912202882309F4F0
:10BE700094C022E0721649F033E0731203C06AE303
:10BE80007CE205C06AE27CE202C06AE47CE200E097
:10BE900010E021E041E08C2F0E94D3407EC0D130E1
:10BEA000D9F48091E905813021F40E94C67B81118B
:10BEB0007DC080912202882309F46FC081E09091B7
:10BEC000E905913009F080E004E024E045EB5CE214
:10BED0006C2F0E94364161C0D230D9F48091E905BF
:10BEE000823021F40E94C67B811169C080912202B8
:10BEF000882309F452C081E09091E905923009F05D
:10BF000080E000E22EE349EA5CE26C2F0E943641B9
:10BF100044C0D330D1F48091E905833021F40E94EC
:10BF2000C67B811157C0809122028823B1F181E044
:10BF30009091E905933009F080E000E22EE34DE9AD
:10BF40005CE26C2F0E94364128C0D43031F58091DC
:10BF5000E905843021F40E94C67B811146C080919E
:10BF600022028823D1F011E08091E905843009F0A4
:10BF700010E02091250537E12303F0011124EF574C
:10BF8000F34F808591850F94472100E09C014FE796
:10BF90005CE26C2F812F0E946A41CF5FDF5F80E0FF
:10BFA000C53009F04CCFC093E8055CC081E00E9429
:10BFB00052778091B605882309F47BCF53C08091D6
:10BFC0002D0590912E05BBDE8091B605882309F4DE
:10BFD0008DCF48C080912F0590913005B0DE8091C3
:10BFE000B605882309F49FCF3DC081E00E94BB7B4A
:10BFF0000091250527E1020380011124F801EF5784
:10C00000F34F60857185072E000C880B990B0F94F8
:10C01000222C20E030E040EF52E40F94A62A0F9447
:10C02000F42BF801E757F34F1F928AEF882E8EE525
:10C03000982E9FE0A92E9EE5B92E6B011AEAE12EFB
:10C04000F12C00E010E028E730E040E050E0BF01D4
:10C050008EE89CE20E9493760F908091B60588232B
:10C0600009F47DCFDF91CF911F910F91FF90EF9059
:10C07000DF90CF90BF90AF909F908F907F9008956A
:10C0800060E081E0C2CE8F929F92AF92BF92CF923A
:10C09000DF92EF92FF920F931F93CF93DF934C01A8
:10C0A0005B016A0160E085E00E943878D091EA0582
:10C0B000F12C82E0E82ED1111AC08091220288234F
:10C0C00021F180912502823041F0833019F46FED27
:10C0D0007BE205C06DEC7BE202C06FEE7BE200E02C
:10C0E00010E021E041E08F2D0E94D3400EC0D130FE
:10C0F00061F480912202882341F000E010E020E00A
:10C1000041E0B4018F2D0E94D340A114B10481F00D
:10C11000D23081F480912202882309F46EC000E0BD
:10C1200010E020E041E0B5018F2D0E94D34065C0B2
:10C13000C2E001C0C3E0C114D10491F0DC130FC010
:10C1400080912202882351F000E010E020E041E0DD
:10C15000B6018F2D0E94D340CD2F01C0CD2FCF5FD0
:10C1600021E030E0A114B10411F420E030E081E0DE
:10C1700090E0C114D10411F480E090E0820F931F8D
:10C18000029781F0DC130DC080912202882349F0D0
:10C1900000E010E020E041E068E07CE28F2D0E94AA
:10C1A000D340CF5FDC1314C080912202882371F04A
:10C1B00000E010E021E040E06DEF7BE28F2D0E9477
:10C1C000D340609124058F2D0E946D40E0922202A1
:10C1D000F394DF5F85E0F8126ECFCF5FC093E80580
:10C1E000DF91CF911F910F91FF90EF90DF90CF9053
:10C1F000BF90AF909F908F900895C3E0C114D10479
:10C2000009F0ADCFADCF40E050E060E070E082ECEF
:10C210009BE239CF49EB5BE269EA7BE280EA9BE291
:10C2200032CF40E050E060E97BE287E89BE22BCF31
:10C2300040E050E068E77BE289E69BE224CF40E003
:10C2400050E06AE57BE28DE49BE21DCF41E45BE2D6
:10C2500060E37BE280E29BE216CF40E050E062E1E7
:10C260007BE289E09BE20FCF40E050E069EF7AE2A9
:10C270008CEE9AE208CF40E050E06FED7AE28EED6E
:10C280009AE201CF40E050E06FEC7AE286EC9AE26D
:10C29000FACE61116093250240932405082E000C0C
:10C2A000990BAA0BBB0B8C309105A0F5FC018827DC
:10C2B000EA56FF4F8F4F0D94042F8AE091E61FC07E
:10C2C00081E191E61CC084E391E619C086E291E623
:10C2D00016C08DE291E613C082E491E610C08BE3B4
:10C2E00091E60DC08FE191E60AC088E191E607C0B2
:10C2F0001092CC0B85E19EE502C083E091E60097A9
:10C3000049F021E02093180620E040E060E070E072
:10C310000C941F770C944B77CF92DF92EF92FF92A1
:10C320000F931F9386E8C82E8DE2D82EE12CF12CB6
:10C330000BE71DE224EF3CE542EF51E866E77DE2C2
:10C3400081E79DE20E94C1781F910F91FF90EF90CD
:10C35000DF90CF9008959091F60893FB882780F99D
:10C3600093FF06C081E090912607911101C080E003
:10C370000895EF92FF920F931F93CF93DF9361E0A5
:10C3800081E00E943878C091EA0510E0C11118C020
:10C390008091E905811104C00E94C67B8111C8C14A
:10C3A00080912202882361F081E09091E90591114A
:10C3B00080E004E024E045E65DE2612F0E94364122
:10C3C0008091F60882FB002700F982FD07C0D1E0CA
:10C3D00090914116913019F0D0E001C0D02F83FB2D
:10C3E000EE24E0F883FF03C0B6DFF82E01C0F12C85
:10C3F000DD2309F458C0C130D9F48091E9058130BA
:10C4000021F40E94C67B81119CC180912202882365
:10C4100009F4A9C181E09091E905913009F080E02B
:10C4200000E22EE349E55DE2612F0E9436419BC1A7
:10C43000C230D9F48091E905823021F40E94C67B94
:10C44000811187C180912202882309F48CC181E087
:10C450009091E905923009F080E003E02EE34EE48C
:10C460005DE2612F0E9436417EC1C33009F063C096
:10C470008091E905833021F40E94C67B811175C14A
:10C4800080912202882309F46EC181E09091E90530
:10C49000933009F080E003E02EE349E45DE2612F90
:10C4A0000E94364160C180914116823029F053DFED
:10C4B0008823F9F001111DC0C130E9F48091E9052C
:10C4C000813021F40E94C67B811159C180912202E2
:10C4D000882309F45CC181E09091E905913009F06D
:10C4E00080E000E22EE34CE35DE2612F0E943641E2
:10C4F0004EC1D1E001C0D2E0CD131BC08091E9054F
:10C500008C1304C00E94C67B811143C1809122021A
:10C51000882371F081E09091E9059C1380E003E0AD
:10C520002EE345E35DE2612F0E943641DC2F01C01E
:10C53000DC2FDF5F01C0D4E0CD131BC08091E90583
:10C540008C1304C00E94C67B81112DC180912202F0
:10C55000882371F081E09091E9059C1380E003E06D
:10C560002EE349E25DE2612F0E943641DC2F01C0DB
:10C57000DC2F81E08D0FC81318C08091E9058C1362
:10C5800004C00E94C67B811118C1809122028823B9
:10C5900061F081E09091E9059C1380E003E02EE3D7
:10C5A0004BE15DE2612F0E94364182E08D0F4091A8
:10C5B000890C50918A0C90914D0C911107C02091DB
:10C5C00036023091370242175307DCF0C81333C0EC
:10C5D0008091E9058C1304C00E94C67B8111F7C0CD
:10C5E00080912202882339F181E09091E9059C1322
:10C5F00080E000E22EE343E05DE2612F0E943641DD
:10C600001AC0C81318C08091E9058C1304C00E9499
:10C61000C67B8111E6C080912202882361F081E00F
:10C620009091E9059C1380E003E02EE343EF5CE288
:10C63000612F0E943641DD5FCD1318C08091E9055E
:10C640008C1304C00E94C67B8111D5C08091220248
:10C65000882361F081E09091E9059C1380E003E07C
:10C660002EE345EE5CE2612F0E94364191E09D0F82
:10C67000EE2009F43BC0F11053C0C91318C08091DB
:10C68000E9058C1304C00E94C67B8111BEC0809155
:10C690002202882361F081E09091E9059C1380E0FB
:10C6A00000E22EE344ED5CE2612F0E94364182E01D
:10C6B0008D0FC81318C08091E9058C1304C00E9427
:10C6C000C67B8111ACC080912202882361F081E099
:10C6D0009091E9059C1380E003E02EE343EC5CE2DB
:10C6E000612F0E94364193E09D0F1AC0C91316C0F6
:10C6F0008091E9058C1302C00E94C67B80912202C2
:10C70000882361F081E09091E9059C1380E000E2CC
:10C710002EE34AEB5CE2612F0E94364192E09D0FCE
:10C720001F5FCF5F153009F031CE9093E80580C0D0
:10C7300081E00E9452778091B605882309F430CEBB
:10C7400077C00E9405828091B605882309F45DCEEA
:10C750006FC08CE891E60E94C8448091B60588239A
:10C7600009F470CE65C0D4E004CF8EE795E60E9450
:10C77000C8448091B605882309F482CE59C00E942E
:10C7800016828091B605882309F4A0CE51C0D2E06C
:10C79000D0CE81E29CE50E94C8448091B6058823F2
:10C7A00009F4B4CE45C088E098E60E94C844809160
:10C7B000B605882309F4CACE3BC08EE995E70E94EE
:10C7C000C8448091B605882309F4DFCE31C083E1E7
:10C7D0009DE20E9491768091B605882309F400CFEE
:10C7E00027C080E490E60E94C8448091B605882363
:10C7F00009F411CF1DC08BE797E60E94C8448091D1
:10C80000B605882309F422CF13C081EE9CE20E9472
:10C8100091768091B605882309F439CF09C084E167
:10C820009DE50E94C8448091B605882309F44BCF4A
:10C83000DF91CF911F910F91FF90EF90089560913C
:10C840007D0C70E080E00C948FA96091850270915E
:10C850008602072E000C880B990B0F94222C2AE0DD
:10C8600037ED43E25CE30F94BE2D60938102709339
:10C87000820280938302909384020895CF93DF9382
:10C88000EC01CB01BA010F94222C0F94F42B688396
:10C89000DF91CF91089580E00C94BCAE6EE374E616
:10C8A00084E594E60C9476770F94222C0F94F42B65
:10C8B000862F0D94CB20EF92FF920F931F93CF936F
:10C8C000DF9300D01F92CDB7DEB7082F7B010E9407
:10C8D000C67B882331F01092180680E00E945277C0
:10C8E0003BC060911006709111066115710551F001
:10C8F000109211061092100681E080932202802F80
:10C900000E94A4A280912202882331F184E0089F32
:10C91000800111240955124F6091B60B7091B70B2D
:10C92000072E000C880B990B0F94222C9B01AC0155
:10C93000F80160817181828193810F94BE2D69839A
:10C940007A838B839C8360E2CE0101960F945224FC
:10C95000BC01C7010E94CF410F900F900F900F9024
:10C96000DF91CF911F910F91FF90EF90089568E0B4
:10C970007EE280E0A0CF6DEF7DE281E09CCF62EFB0
:10C980007DE282E098CF20E040E060E070E00E942D
:10C990001F7781E0809318061092B70B1092B60BA8
:10C9A000089587EB94E6EFCF8BEB94E6ECCF8FEB1B
:10C9B00094E6E9CF2F923F924F925F926F927F92CF
:10C9C0008F929F92AF92BF92CF92DF92EF92FF929F
:10C9D0000F931F93CF93DF93CDB7DEB729970FB691
:10C9E000F894DEBF0FBECDBF1C017987688769014F
:10C9F0001A830983EB82BA01550F880B990B0F94A8
:10CA0000222C4B015C0120E030E040E057EC0F9419
:10CA1000832D18162CF0812C912CA12C27ECB22EF2
:10CA2000C501B4010F94EF2B2B013C01B601DD0CC5
:10CA3000880B990B0F94222C4B015C0120E03EEFF8
:10CA40004FEF56E40F94802B87FD07C0812C9EEF9B
:10CA5000992EAA24AA9496E4B92EE885F9856081D6
:10CA60007181072E000C880B990B0F94222C6B01FF
:10CA70007C01C301B2010F94222C9B01AC01C701C0
:10CA8000B6010F94A62A0F94F42B6C837D838E83BA
:10CA90009F83C501B4010F94EF2B7B018C01E41837
:10CAA000F50806091709FB81FF9389809A808FE0BA
:10CAB000A82E8EE5B82ECC80DD80A301920168857A
:10CAC0007985C1010E9493760F9029960FB6F8944C
:10CAD000DEBF0FBECDBFDF91CF911F910F91FF90B1
:10CAE000EF90DF90CF90BF90AF909F908F907F900E
:10CAF0006F905F904F903F902F9008958F929F92EC
:10CB0000AF92BF92CF92DF92EF92FF920F931F935B
:10CB1000CF93DF9361E081E00E943878D091EA05FD
:10CB2000C0E0D1111AC08091E905811104C00E94B2
:10CB3000C67B811121C180912202882309F413C18F
:10CB400081E09091E905911180E004E024E04DEE50
:10CB50005DE26C2F0E94364106C1D13011F5809103
:10CB6000E905813021F40E94C67B81110EC18091BC
:10CB70002202882309F4F7C011E08091E905813091
:10CB800009F010E080915F02909160020F944721BC
:10CB900000E09C0141EE5DE26C2F812F0E946A4112
:10CBA000E2C0D23011F58091E905823021F40E9473
:10CBB000C67B8111FCC080912202882309F4D3C076
:10CBC00011E08091E905823009F010E08091890C34
:10CBD00090918A0C0F94472100E09C0143ED5DE2A7
:10CBE0006C2F812F0E946A41BEC0D33011F5809115
:10CBF000E905833021F40E94C67B8111EDC080914C
:10CC00002202882309F4AFC011E08091E905833046
:10CC100009F010E08091630C9091640C0F9447210F
:10CC200000E09C014BEC5DE26C2F812F0E946A4179
:10CC30009AC0D43001F58091E905843021F40E9436
:10CC4000C67B8111DEC080912202882309F48BC04B
:10CC500011E08091E905843009F010E080917D0CAD
:10CC60000F94CB2000E09C0143EB5DE26C2F812F01
:10CC70000E946A4178C0D53011F58091E905853070
:10CC800021F40E94C67B8111DFC08091220288239B
:10CC900009F469C011E08091E905853009F010E0E0
:10CCA00080918502909186020F94472100E09C01BB
:10CCB00049EA5DE26C2F812F0E946A4154C0D63050
:10CCC000D9F48091E905863021F40E94C67B811158
:10CCD000CDC080912202882309F445C081E0909163
:10CCE000E905963009F080E003E02EE34EE95DE2CD
:10CCF0006C2F0E94364137C0D730D1F48091E905BE
:10CD0000873021F40E94C67B8111BAC08091220233
:10CD1000882349F181E09091E905973009F080E09E
:10CD200003E02EE343E95DE26C2F0E9436411BC015
:10CD3000D830C9F48091E905883021F40E94C67B7F
:10CD40008111A8C080912202882369F081E090912E
:10CD5000E905983009F080E003E02EE348E85DE261
:10CD60006C2F0E943641CF5FDF5FC53009F0D9CE0E
:10CD700089E08093E80597C081E00E945277809116
:10CD8000B605882309F4D7CE8EC0E12C00E010E070
:10CD900027EE33E04AE050E06FE572E087EE9DE277
:10CDA00009DE8091B605882309F4E1CE7CC081E0DC
:10CDB0000E94BB7BE12C0BE414E622E231E040E070
:10CDC00050E069E87CE08AED9DE2F4DD8091B605F3
:10CDD000882309F4F0CE67C081E00E94BB7BE12C80
:10CDE00009E01FEA2CE830E040E050E063E67CE038
:10CDF0008FEC9DE2DFDD8091B605882309F4FFCE3C
:10CE000052C081E00E94BB7BC0907D0CD12C1F9250
:10CE10008FE1882E84E6982E9EE4A92E94E6B92E02
:10CE2000E12CF12C8701EA9420E030E0A9016DE7C4
:10CE30007CE08FEB9DE20E9493760F908091B60587
:10CE4000882309F400CF2FC0E12C05E214E627EE79
:10CE500033E04AE050E065E872E08EEA9DE2AADD48
:10CE60008091B605882309F410CF1DC081ED94E6AA
:10CE70000E94C8448091B605882309F42ACF13C0C4
:10CE800084ED94E60E94C8448091B605882309F495
:10CE90003DCF09C087ED94E60E94C8448091B60555
:10CEA000882309F44FCFDF91CF911F910F91FF900D
:10CEB000EF90DF90CF90BF90AF909F908F900895AC
:10CEC0000E94C67B882329F01092180680E00E94F9
:10CED000527780E00C94FE3F0E94C67B882341F08D
:10CEE00020E040E060E070E080E697E60E941F7777
:10CEF00080E00C94559A0F93CF93DF9361E081E02B
:10CF00000E943878D091EA05C0E0D11117C0809115
:10CF1000E905811104C00E94C67B81114CC080913B
:10CF20002202882309F43EC081E09091E905911125
:10CF300080E004E024E04AE25EE231C0D130B9F49E
:10CF40008091E905813021F40E94C67B81113CC0AB
:10CF500080912202882331F181E09091E90591309E
:10CF600009F080E003E02EE349E15EE218C0D5302D
:10CF7000C9F48091E905853021F40E94C67B8111B6
:10CF80002DC080912202882369F081E09091E9050B
:10CF9000953009F080E003E02EE343E15EE26C2F80
:10CFA0000E943641CF5FDF5FC53009F0AECF86E02B
:10CFB0008093E8051BC081E00E9452778091B605FE
:10CFC000882309F4ACCF12C08CE697E60E94C844CF
:10CFD0008091B605882309F4BBCF08C08EED94E498
:10CFE0000E94C8448091B605882359F2DF91CF9101
:10CFF0000F91089560E070E080E00E948FA960E0EA
:10D0000070E081E00E948FA90E9456AF0C944B778C
:10D010008F929F92AF92BF92CF92DF92EF92FF9248
:10D020000F931F93CF93DF9361E081E00E943878E4
:10D03000D091EA05C0E0D1111AC08091E9058111B3
:10D0400004C00E94C67B8111ABC08091220288235C
:10D0500009F474C081E09091E905911180E004E049
:10D0600024E046E65EE26C2F0E94364167C0D13074
:10D0700011F58091E905813021F40E94C67B811170
:10D0800098C080912202882309F458C011E0809151
:10D09000E905813009F010E08091890C90918A0CAB
:10D0A0000F94472100E09C0148E55EE26C2F812F40
:10D0B0000E946A4143C0D23009F58091E90582306F
:10D0C00021F40E94C67B81119AC08091220288239C
:10D0D000A9F111E08091E905823009F010E080911A
:10D0E000630C9091640C0F94472100E09C0140E593
:10D0F0005EE26C2F812F0E946A4120C0D330F1F490
:10D100008091E905833021F40E94C67B81119CC087
:10D1100080912202882391F011E08091E90583300B
:10D1200009F010E080917D0C0F949C2000E09C01A0
:10D1300048E35EE26C2F812F0E946A418091890C46
:10D1400090918A0C2091630C3091640C232B11F484
:10D15000892BE9F0D430C9F48091E905843021F4B9
:10D160000E94C67B8111A1C080912202882369F0B0
:10D1700081E09091E905943009F080E000E22EE32F
:10D180004FE25EE26C2F0E94364185E001C084E0F0
:10D19000CF5FDF5FC53009F04ECF8093E8058BC0CD
:10D1A00081E00E9452778091B605882309F44DCF23
:10D1B00082C081E00E94BB7BC090890CD0908A0C19
:10D1C0001F926BE4862E64E6962E7FE0A72E7EE506
:10D1D000B72E12E2E12EFF24F39400E010E020E0ED
:10D1E00030E0A90169E87CE08FE59EE20E94937639
:10D1F0000F908091B605882309F443CF5CC081E08D
:10D200000E94BB7BC090630CD090640C1F9239E0ED
:10D21000832E3FEA932E4FE0A42E4EE5B42E1CE859
:10D22000E12EF12C00E010E020E030E0A90163E6FF
:10D230007CE084E59EE20E9493760F908091B60593
:10D24000882309F442CF37C081E00E94BB7B609104
:10D250007D0C70E080E090E00F94202C29EC38ECFD
:10D2600048EC5EE30F94BE2D0F94F42B1F928FE1D8
:10D27000882E84E6982E94EAA92E95E4B92E6B01A7
:10D2800014E6E12EF12C00E010E020E030E0A901EE
:10D290006DE77CE084E49EE20E9493760F9080919B
:10D2A000B605882309F434CF06C0A4DE8091B60504
:10D2B000882309F459CFDF91CF911F910F91FF90EF
:10D2C000EF90DF90CF90BF90AF909F908F90089598
:10D2D00080E095E290934105809340058CE491E0D5
:10D2E000909345058093440580EC9EEF9093430511
:10D2F0008093420590913C0580E2890F863740F08B
:10D3000080EF890F20E431E03093430520934205FC
:10D3100010923E0580933F058FEF80933D05089561
:10D320008F929F92BF92CF92DF92EF92FF920F93D4
:10D330001F93CF93DF931F92CDB7DEB7F7D7882324
:10D3400009F4D6C180911006863214F085E202C03D
:10D3500087FD80E0282F082E000C330B3093110638
:10D3600020931006982F990F890F80933C05809188
:10D37000A005882309F4BCC12091420530914305E2
:10D3800000913E0510913F05020F131FE0904005EC
:10D39000F09041058091440590914505E80EF91EF5
:10D3A00001304FE7140768F031952195310930932A
:10D3B0004305209342056CED70E085E090E00F940A
:10D3C000A727F7FE15C080914405909145059195DA
:10D3D00081959109909345058093440568E171E03A
:10D3E00085E090E00F94A72781E080933D0517C06A
:10D3F00081E0E81680E4F80694F06BE470E084EFD6
:10D4000091E00F94A72780913205815080933205D7
:10D41000882311F05DDF6CC11092A00569C12091D5
:10D42000440530914505C7019A508130934108F079
:10D4300098C08F2D992787FD9A950A9765E070E02F
:10D440000F94B32E812F17FF02C087E0810F482F62
:10D4500045954595459581E090E0A0E0B0E004C099
:10D46000880F991FAA1FBB1F4A95D2F7FB01EE0F29
:10D47000FF1FEC5CFA4F408151818A010823192378
:10D48000012B09F419C180959095842395239183EC
:10D49000808384E090E0861B970B4091A10550911A
:10D4A000A205840F951F9093A2058093A1058091FA
:10D4B0003305815080933305811103C082E080934E
:10D4C000A005932F9095991F9927991F80913D054D
:10D4D000881F8827881F9817F1F031952195310909
:10D4E000309345052093440520E130E040E050E0D2
:10D4F00060EF7FEF8FEF9FEF0E945836209142053B
:10D5000030914305620F731F70934305609342058A
:10D5100060E773E021C080914205909143059195A9
:10D5200081959109909343058093420520E130E075
:10D5300040E050E060EF7FEF8FEF9FEF0E945836A2
:10D540002091440530914505620F731F7093450586
:10D550006093440560E872E085E090E00F94A727AF
:10D56000ABC0121613060CF0A7C0FDE3FF1A41E092
:10D57000E41642E0F40608F09FC080913C05181BB9
:10D58000103108F099C03195219531093093450546
:10D590002093440560E773E083E090E00F94A727B1
:10D5A0008FEF80933D0521E012300CF020E08EEFEC
:10D5B000810F8C30A0F0809142059091430541E0AD
:10D5C00050E01816190614F040E050E030E0421721
:10D5D000530709F055C091958195910927C01430E2
:10D5E00050F520E030E0A90160EC7FEF8FEF9FEF76
:10D5F0000E9458362091420530914305620F731FF7
:10D60000709343056093420561157E4F34F480E0CA
:10D610009EEF90934305809342058091420590913F
:10D6200043058130924064F180E092E0909343059D
:10D630008093420525C01C301CF120E430E040E01E
:10D6400050E060E070E0CB010E9458362091420526
:10D6500030914305620F731F709343056093420539
:10D6600061157E4F34F480E09EEF909343058093E4
:10D670004205809142059091430581309240A4F685
:10D680008091A0058230C1F480E4809333058FEF50
:10D690009FEF9093350580933405909337058093E1
:10D6A0003605909339058093380590933B05809318
:10D6B0003A0581E08093A00520913E0530913F0519
:10D6C0008091420590914305820F931F90933F05EF
:10D6D00080933E052091400530914105809144059D
:10D6E00090914505820F931F9093410580934005CB
:10D6F00061E082EE93E00E94EF30809116048E315B
:10D7000030F0809116048E3308F456C05AC08091D0
:10D7100018048A30B0F382E3E82E85E0F82E9AE010
:10D72000892E912CB82C8091160490E094012C5FE6
:10D730003F4F281739075CF442E0E40EF11C85E006
:10D74000880E911CEEE18E16910461F7DACF80917C
:10D750001804881588F330E0C12CD12CF7018281A0
:10D760009381A0E0B0E00C2C04C0B695A7959795E6
:10D7700087950A94D2F780FD07C0FFEFCF1ADF0A22
:10D78000385F303859F7D8CF00E010E0A801480DD5
:10D79000591D8091160490E0481759073CF080917C
:10D7A000180490E0841795070CF056C00F5F1F4FC8
:10D7B0000430110559F7E1CF809118048C3308F03B
:10D7C00056C08091A0058823B1F080914105482F73
:10D7D000582F550F550B9A0133272F5F3F4F8091DC
:10D7E000160490E0281739073CF08091180484173C
:10D7F00008F04EC001C0B3D5809116048B30D8F428
:10D800000091A1051091A20569E080E00E94F73720
:10D81000C8010E94FC3769E08EE60E94F73720912C
:10D82000320583E090E0821B91096FEF7FEF85590D
:10D83000914D0E9450380E94C67B882391F10F9031
:10D84000DF91CF911F910F91FF90EF90DF90CF90DC
:10D85000BF909F908F90C0C527E04B2D400F632F46
:10D8600082EE93E039830E94003339819FCF20E11B
:10D870004DE360913C0582EE93E00E94003320E18D
:10D880004CE360913C0582EE93E00E94003399CF17
:10D8900060913F0502E022E082EE93E00E94413376
:10D8A000ABCF0F90DF91CF911F910F91FF90EF9031
:10D8B000DF90CF90BF909F908F90089560E979E6B8
:10D8C00082E079D5E2E3F5E088E3828783E0808334
:10D8D00080E4818313821282158214821782168259
:10D8E00011861086F5DC82E190E09093110680931A
:10D8F000100608958F929F92AF92BF92CF92DF92BF
:10D90000EF92FF9260915D0520E030E090E080E0D2
:10D91000F901EE5CFA4FC7A4CC2011F061E0620F70
:10D920008C29722F7295707F40E050E0D12CE12C51
:10D93000F12C46015701042E04C0B694A794979485
:10D9400087940A94D2F780FE08C0E92FF0E0EE5CDD
:10D95000FA4FA72FA42BA2AB9F5F4F5F5F4F4530BD
:10D96000510539F72F5F3F4F2330310589F660931A
:10D970005D0540E050E020E090E0A0E0B0E06C0108
:10D980007D01042E04C0F694E794D794C7940A94BA
:10D99000D2F7C0FE05C020935B052AE335E007C03F
:10D9A0002E504F5F5F4F4530510549F7F4CF422F5E
:10D9B0003150A0F0225F6C017D01032E04C0F6946B
:10D9C000E794D794C7940A94D2F7C0FEF0CF40935F
:10D9D0005C0580915E05823069F403C020935C058C
:10D9E000F8CF80915A05181614F08CEF01C084E02E
:10D9F00080935A05FF90EF90DF90CF90BF90AF904B
:10DA00009F908F90089580E090E0FC01EE5CFA4FCB
:10DA1000168203968E319105C1F70895E2E3F5E091
:10DA200010828AE0818383E080A78FE084A78FE162
:10DA300087A780AB81AB5EDFE6CF1F93CF93DF93E9
:10DA4000EC01162FE0DF809135058093570587E3C1
:10DA50008093580586E0809359056AE070E088EE6F
:10DA600093E00F94A727909134059150909334053B
:10DA7000992351F010925605188310923505109293
:10DA800011061092100601C01882DF91CF911F91EC
:10DA900008952F923F925F926F927F928F929F9202
:10DAA000AF92BF92CF92DF92EF92FF920F931F93AC
:10DAB000CF93DF931F92CDB7DEB784E0809322022D
:10DAC00080911206882309F470C28091100690910B
:10DAD00011068E31910514F08DE190E097FF02C0A0
:10DAE00080E090E09093110680931006880F991FB4
:10DAF000880F991F20913505422F022E000C550BDF
:10DB00004817590774F42D5FAC01421B510927FDDA
:10DB10005395423051051CF02093350502C0809387
:10DB2000350520913505422F022E000C550B841728
:10DB300095077CF42350422F022E000C550B481BF6
:10DB4000590B423051051CF02093350502C08093DB
:10DB500035058091A005882309F427C2209174051A
:10DB6000222349F090917305920F90937305933F90
:10DB700014F410927405823070F081508093A005E7
:10DB8000823011F44BDF11C2843609F00EC281E0FD
:10DB90008093A0050AC2809160058F5F8093600525
:10DBA00040915E0590E0242F30E0359527952817A9
:10DBB00039070CF0B3C09091750581E089278093F7
:10DBC000750510926005442309F4A8C090915A0588
:10DBD00080913205890F20915B05821724F02091F6
:10DBE0005C052817D4F4919590935A05209133053C
:10DBF0002B5F209333058093320580915D053AE0D9
:10DC00008302C0011124820F911D27FD9A95C997A7
:10DC100024F064E180EA95E010DF90915A0580914C
:10DC20003205890F8093320580915E05882309F4BF
:10DC300075C024E130E040E050E060E070E0CB01EE
:10DC40000E945836672B682B692B09F067C0E8E300
:10DC5000F5E080E090E0208121115AC09C01220F64
:10DC6000331F8901080F191FC8018A5C9A4F892B3D
:10DC700009F454C020915E0530E02F5F3F4F032E22
:10DC8000000C440B550B60E070E0CB010E9458364D
:10DC9000FB01EE5CFA4F42A9242F30E0B4E0359549
:10DCA0002795BA95E1F7F901EB5BFC4F808190E095
:10DCB0000E5C1A4F4F70509132056EE0469F500D2A
:10DCC0001124452FFC01EE5BFC4F5081450FFC01F8
:10DCD000E15CFC4F90819695842F890FF801848335
:10DCE0008091330582502F5F3F4FFAE02F9F800DC8
:10DCF0001124F801858322E030E040E050E060E04C
:10DD000070E0CB010E9458366E5FF801668306C052
:10DD1000019633968A30910509F09DCF9091560572
:10DD2000992341F080915505890F8093550587FD12
:10DD30001092560580915605882309F4A2C02091BF
:10DD40005505E09133052E170CF49BC0022E000CF4
:10DD5000330B0E2E000CFF0BCF014D96821793074D
:10DD60000CF48FC010913205E0905405CE2C0E2C8F
:10DD7000000CDD08C601811B910917FD93956EE02B
:10DD800070E00F94B32EF62E653008F07AC02E1B8B
:10DD90003F0BC90102966AE070E00F94B32E062F84
:10DDA000633008F06EC0812C912C540183940F2CA9
:10DDB00004C0880C991CAA1CBB1C0A94D2F7A62F7D
:10DDC000660FBB0BBD016E5C7A4FFB0197A5892FD7
:10DDD000882109F456C0FD01EB5BFC4FE0814E2F1A
:10DDE00050E0812FFEE0FF9E800D11249A012E5BF2
:10DDF0003C4FF901F080F80EEF140CF442C0FA0128
:10DE0000E15CFC4F1081412F50E04F0D511DF7FC9C
:10DE10005A95C416D506ACF510925605282D2095B6
:10DE20002923FB0127A723E030E02A1B3B0B80912D
:10DE3000A1059091A205280F391F3093A2052093C8
:10DE4000A1056AE070E088E290E00F94A727209196
:10DE50003305FAE00F9F200D1124912F96958F2DF9
:10DE6000890F8550809357052093580584E080934F
:10DE7000590580915E05815080935E05882321F0CD
:10DE800039DD08E315E012C084E18093A005BBDD15
:10DE9000F8CF8291890F808380346CF0F801108272
:10DEA0000D5F1F4FF5E006351F07E9F0F80190817F
:10DEB0009923B1F3EECF87339CF3F8013297208199
:10DEC00080913505281764F3022E000C330B082EC1
:10DED000000C990B0A968217930714F368E780EAFF
:10DEE00095E0ABDDDDCF80917405811124C024EF76
:10DEF00031E040E050E060E070E0CB010E94583635
:10DF0000672B682B692BB9F422E030E040E050E049
:10DF100060E070E0CB010E945836672B682B692BBC
:10DF200009F099C18FEF80937405813009F495C190
:10DF30008FE780937305809156058823B1F1809116
:10DF40007405882391F180915505873074F52091EF
:10DF5000540580917305281744F1022E000C330BF1
:10DF6000082E000C990B0C9682179307F4F0109270
:10DF70007405109256058091A1059091A2050A960C
:10DF80009093A2058093A1056AE070E088E290E09A
:10DF90000F94A727809173058F5F8093570581E0C9
:10DFA0008093580584E08093590580911A0682FF7A
:10DFB00004C080915F05815001C08AE080935F05B5
:10DFC0000E94C67B8823C1F08091A005811103C007
:10DFD00010925F0511C0813079F48091560581114E
:10DFE0000BC0809135058B5F8093540584E380934B
:10DFF00055058CEF8093560580915F05811101C016
:10E00000EBD161E082EE93E00E94EF303091330576
:10E01000632F032E000C770B80915D05AB012AE086
:10E020008202400D511D1124425051098091160465
:10E0300090E0841795072CF08091740581116BC0D6
:10E040006FC08091180490E086179707ACF3F5E451
:10E050006F2EF3E07F2EC12CD12CF30121913F01D3
:10E06000432F032E000C550BBA01695F7F4F80913F
:10E07000160490E0681779074CF4365FFFEFCF1A6B
:10E08000DF0A23E0C216D10441F7D6CF80911804ED
:10E0900090E0841795078CF31091320546E4542ED6
:10E0A000510EA12CB12CC6018E5C9A4F4C01822FCF
:10E0B00090E01C01220C331CF40187A590E0A0E045
:10E0C000B0E00A2C04C0B695A795979587950A9459
:10E0D000D2F780FF19C0809175057101E80EF11C1F
:10E0E000C701E4E0880F991FEA95E1F7AC014256B9
:10E0F000514D7A0108E022E0432F612F82EE93E038
:10E1000039830E9419313981125F5FEFA51AB50A70
:10E110001511D2CFB2CF80911604883008F49FC079
:10E120008091A005882369F0909116049F3348F4EC
:10E1300090911804973328F0823008F49EC081FD36
:10E140009CC0809156058823B1F040915505242F3D
:10E15000042E000C330BB9016D5F7F4F80911604C4
:10E1600090E0681779073CF08091180490E08217DE
:10E1700093070CF090C000E010E0F801EE5CFA4F5D
:10E180008681882399F04581842F042E000C990BF9
:10E190002091160430E08217930744F002972091F3
:10E1A000180430E0281739070CF07DC00D5F1F4FB1
:10E1B0000E31110511F7809159058823B1F0409176
:10E1C0005805242F042E000C330BB9016A5F7F4FD2
:10E1D0008091160490E0681779073CF0809118044C
:10E1E00090E0821793070CF066C08091A005811122
:10E1F00001C0B5D0809116048A3008F06EC000913D
:10E20000A1051091A20569E080E00E94F737C801DE
:10E210000E94FC3780913405882309F45EC011E028
:10E2200060E1C62ED12C80913405811708F455C0C9
:10E23000B601611B7109660F660F660F79E8E72E5C
:10E240007EE2F72E05E021E041E082EE93E00E94BD
:10E2500019311F5FE8CF81E066CE83EF6ACE21E7F8
:10E26000E22E2EE2F22E05E022E042E060917305FC
:10E2700082EE93E00E94193153CF9EE8E92E9EE290
:10E28000F92E08E022E047E36091350582EE93E045
:10E290000E94193156CF24E06091540582EE93E03C
:10E2A0000E94203368CF425023E0648182EE93E0E5
:10E2B0000E9420337BCF8BE7E82E8EE2F82E07E01A
:10E2C00022E06091570582EE93E00E94193180911F
:10E2D000590581508093590588CF0F90DF91CF91D8
:10E2E0001F910F91FF90EF90DF90CF90BF90AF9074
:10E2F0009F908F907F906F905F903F902F900895A8
:10E30000CF93DF9369E47DE684E155D0C2E3D5E0A5
:10E3100083E08A838AE08DA71CA280DB1B82109297
:10E32000110610921006DF91CF9108958091120688
:10E33000882319F082E08093310584E080932202E3
:10E340008091A005882349F0909131058FEF890FC6
:10E350008093310581E019160CF080E008950F9349
:10E3600080911604853228F5809118048B3108F1CC
:10E3700060E082EE93E00E94EF3009E028E34BE199
:10E3800064E282EE93E00E94913361E082EE93E0DA
:10E390000E94EF300E940F7D882359F063E285E2EE
:10E3A0000E94F7376FEF7FEF8EEF9EE20F910C9494
:10E3B00050380F910895FB011092A2051092A1050B
:10E3C0008093A00520E040E060E070E0CF0137D509
:10E3D00081E08093180608951092180680E062C5C7
:10E3E000809137059091390589130DC080913805CA
:10E3F00090913A05891714F02FEF01C021E0820FA8
:10E400008093380508C0891714F02FEF01C021E070
:10E41000820F8093370589131BC020919F052150DF
:10E4200020939F0530E0832F90E0DC01AA0FBB1FF3
:10E43000AE5CBA4F880F991FFC01EC5CFA4F8581E6
:10E44000968116969C938E9315973F5F231758F7E6
:10E450000895EF92FF921F93CF93DF9310919F0542
:10E4600020913405E22E022E000CFF083091330576
:10E47000C32F032E000CDD0BEAE3F5E040E041176B
:10E4800009F446C0CF010397DC019C91BF016150A4
:10E490007109DB018C9198131DC0692F092E000CA6
:10E4A000770B61507109C617D70711F039132DC0CA
:10E4B0009081BF0162507109DB018C91582F981730
:10E4C0000CF4592F25170CF189170CF4892F82179A
:10E4D000E4F020C0BF0162507109DB015C91652F3F
:10E4E000052E000C770B61507109E616F70611F046
:10E4F00025130BC0582F98170CF4592F35172CF0F3
:10E5000089170CF4892F83172CF44F5F3296B7CFFD
:10E5100080E001C081E0DF91CF911F91FF90EF90EB
:10E52000089528E130E040E050E060E070E0CB0189
:10E530000E945836609333052AE030E040E050E016
:10E5400060E070E0CB010E9458366093340581DFB3
:10E550008111E7CF089590913205811102C08FEFAC
:10E5600001C081E0980F93709093320580919F05D0
:10E570008F5F80939F0590E0FC01EE0FFF1FEE5C24
:10E58000FA4F20919C052583880F991FFC01E85CB8
:10E59000FA4F80919E05808308951F93CF93DF9358
:10E5A000C2E3D5E080E091E090939C0580939B05C9
:10E5B00080E095E090939E0580939D0518821092CF
:10E5C0009F051D8215E01E8381E0C5DF1B8310922D
:10E5D0001106109210061C82DF91CF911F910895B1
:10E5E000EF92FF920F931F93CF93DF9380919F053C
:10E5F000843008F4DEC090E0FC01EE0FFF1FE05D08
:10E60000FA4F3581FC01EE0FFF1FEE5CFA4F65817A
:10E61000AC0142505109361739F0C0E0880F991FFC
:10E62000FC01EA5CFA4F82C0F12CDC01AA0FBB1F8F
:10E63000A85CBA4F880F991FFC01EA5CFA4F8F2D36
:10E6400090E0841795070CF0B4C0BC01660F771FEB
:10E650006E5C7A4FEB016D818C01000F111F0C5C19
:10E660001A4FE8012D816217F1F0722F62170CF436
:10E67000762F3717ECF126170CF4262F2317C4F149
:10E68000880F991F885C9A4FEC01288191E0808166
:10E6900028170CF090E081E06C9162170CF480E098
:10E6A000981731F188C0361323C07C9120818C01EA
:10E6B000000F111F065C1A4FE8016881880F991F2F
:10E6C000885C9A4FEC018881122F72170CF4172F77
:10E6D000982F86170CF4962F911754F0922F271726
:10E6E0000CF4972F68170CF4862F98170CF063C062
:10E6F000F394A5CF7C01DFEFED1AFD0A8C01000F2A
:10E70000111F085C1A4FD8017C918C01000F111F5A
:10E71000065C1A4FD8012C91721729F1A081B22FF3
:10E7200072170CF4B72FAB173CF4CF5F8C2F90E02F
:10E7300084179507FCF23DC027170CF4272F2A17E2
:10E74000A4F3880F991FDC01AE5CBA4F15962C918B
:10E7500091E023170CF090E081E062170CF480E068
:10E76000981719F328C020812713DFCFD701AA0FEC
:10E77000BB1FAE5CBA4F15962C91880F991FDC0118
:10E78000AE5CBA4F15968C91762F36170CF4732F1A
:10E79000982F82170CF4922F97173CF2962F63173D
:10E7A0000CF4932F28170CF4822F98170CF4BDCF7C
:10E7B00002C080E001C081E0DF91CF911F910F91F5
:10E7C000FF90EF900895BF92CF92DF92EF92FF9269
:10E7D0000F931F93CF93DF931F92CDB7DEB7A6DDC4
:10E7E000882309F486C080919B0590919C05392F60
:10E7F00040919D0550919E0520913205213061F098
:10E800002CF4211116C0CA01C3970AC0223031F07E
:10E81000233079F4C39709C0C39607C0CA01C396D1
:10E8200090939E0580939D0504C090939C058093D2
:10E830009B0510919C0500919E05311303C005179F
:10E8400009F457C0183110F40A3048F01092A005AE
:10E8500068E270E080E991E00F94A7274AC08091B8
:10E860009F0590E0FC01EE0FFF1FEE5CFA4F158351
:10E87000880F991FFC01E85CFA4F00838091100615
:10E8800090913605282F291B39F08093360581E0B9
:10E8900012160CF080E05FDE80913505882321F0B0
:10E8A00081508093350501C09BDD9ADE8111CECF6A
:10E8B0008091330518131DC080913405081319C0C9
:10E8C0006CED70E085E090E00F94A72768E171E0BF
:10E8D00085E090E00F94A7278091A1059091A20573
:10E8E00001969093A2058093A10582E0809335055F
:10E8F00018DE61E082EE93E00E94EF308091160412
:10E90000893058F4E090A105F090A20567E080E01E
:10E910000E94F737C7010E94FC3706E32CE749E065
:10E9200062E082EE93E00E94413310E080919F0507
:10E9300030911604181708F084C0412F50E0BA0136
:10E94000660F771FFB01EE5CFA4FA581FB01EC5CC3
:10E95000FA4F2581CA010396A21351C0FB01E65C60
:10E96000FA4F2081880F991FFC01EE5CFA4FC0809E
:10E97000DC2CC2160CF4D22E8D2D95E08902A0015C
:10E980001124425F5F4F832F90E0481759070CF422
:10E9900056C02C150CF4C22EEC2DF5E0EF029001C0
:10E9A0001124265F3F4F8091180490E02817390703
:10E9B0000CF045C08C2D880F880F8C0DEBE0BE2E1F
:10E9C000B80ECB01895C9A4F7C01DC14C4F12B2D6D
:10E9D0000B2C000C330BA9014D5F5F4F8091160487
:10E9E00090E0481759073CF08091180490E0821796
:10E9F00093070CF053C0C39495E0B90EE6CF880F8F
:10EA0000991FFC01EE5CFA4F8081982F990F990FA6
:10EA1000890F5BE0E52EE80E4E2D0E2C000C550BF9
:10EA2000BA016D5F7F4F832F90E0681779073CF044
:10EA30006091180470E0641775070CF03EC01F5F0A
:10EA400075CF40913405842F880F880F480F455F9C
:10EA5000642F042E000C770BFB013396832F90E07C
:10EA6000E817F9073CF08091180490E086179707A3
:10EA70000CF045C08091A005811101C070DC86D6E4
:10EA8000882309F44AC00F90DF91CF911F910F9115
:10EA9000FF90EF90DF90CF90BF909ECCF701608108
:10EAA000862F880F880F680F6C5F04E024E04B2DE1
:10EAB00082EE93E00E9491339ECFD22EA2170CF4E7
:10EAC000DA2EC22E2A170CF4CA2EFD2CFF0CFF0CD6
:10EAD0008F2D8D0D30E094E0F92EF80ECD140CF44E
:10EAE000AECF6F2D630F04E024E04E2D82EE93E055
:10EAF00039830E949133D39439813B5FEFCF60918A
:10EB00003305862F880F880F680F6C5F04E024E0C0
:10EB100082EE93E00E944133ADCF0F90DF91CF9111
:10EB20001F910F91FF90EF90DF90CF90BF900895CD
:10EB300063EE73E781E03FDC30DDF3CC0F931F938E
:10EB4000CF93DF9361E081E093D2D091EA05C0E0FA
:10EB5000D11115C08091E905811103C017D681112B
:10EB600081C080912202882321F181E09091E90502
:10EB7000911180E004E024E048E45FE217C0D13066
:10EB8000C1F48091E905813019F400D6811172C079
:10EB900080912202882369F081E09091E90591300B
:10EBA00009F080E003E02EE346E35FE26C2F0E9471
:10EBB00036412ED1182FD230D1F48091E905823020
:10EBC00019F4E4D5811164C080912202882309F4EC
:10EBD00071C081E09091E905923009F080E000E297
:10EBE0002EE347E25FE26C2F0E94364163C0811141
:10EBF00063C0D330B1F48091E905833019F4C6D5F0
:10EC000081114DC080912202882319F181E09091F9
:10EC1000E905933009F080E000E22EE349E15FE28C
:10EC200015C0D430B1F48091E905843009F43EC0B8
:10EC300080912202882369F081E09091E905943067
:10EC400009F080E000E22EE348E05FE26C2F0E94D2
:10EC5000364185E0CF5FDF5FC53009F079CF809323
:10EC6000E80535C081E01ED18091B605882309F4FE
:10EC700078CF2DC031D020E040E060E070E087EF39
:10EC80009CE4DDD08091B605882309F481CF1FC0B4
:10EC90005DD28091B605882309F496CF18C059D269
:10ECA0008091B605882309F4ADCF11C06FD58111CD
:10ECB00005C0BECF112369F283E0CCCF0E9404D0FF
:10ECC00081E028D28091B605882309F4B1CFDF9185
:10ECD000CF911F910F910895E091B705E63000F5AF
:10ECE00081E08E0F8093B7058091100690911106F8
:10ECF000A0E0B0E03091EA052091E80548E0E49F0B
:10ED0000F0011124E854FA4F40910B0650910C0683
:10ED10005183408382839383A483B583368327837F
:10ED200008950D942A1A2F923F924F925F926F92FC
:10ED30007F928F929F92AF92BF92CF92DF92EF928B
:10ED4000FF920F931F93CF93DF9300D000D0CDB7E6
:10ED5000DEB71C012B833C834D835E8369837A83FA
:10ED6000BBDF83E0809322023092B5052092B40588
:10ED700069817A817093B3056093B2052B813C81E0
:10ED80004D815E812093AE053093AF054093B00571
:10ED90005093B105E092AA05F092AB050093AC0543
:10EDA0001093AD05D0921106C0921006B0920C06D9
:10EDB000A0920B069092A9058092A8058C8D809355
:10EDC000A70526960FB6F894DEBF0FBECDBFDF9124
:10EDD000CF911F910F91FF90EF90DF90CF90BF9058
:10EDE000AF909F908F907F906F905F904F903F90EB
:10EDF0002F900895FB01908181E08927808383E033
:10EE0000809322024115510511F0FA0119940895D9
:10EE10008091150E9091120E891B8F7071F4909154
:10EE2000F60892FB882780F992FD08C081E0909156
:10EE30004116913019F080E0089581E00895E09145
:10EE40000B06F0910C06E817F90721F130911B062B
:10EE500037FD10921B0690930C0680930B0670935F
:10EE60001106609310064093EA052093E805865248
:10EE70009B4721F4109218061092B7050E946C402F
:10EE800082E08093220281E08093B60510921306FF
:10EE90001092A305089520E040E060E070E086E273
:10EEA0009BE7CDCFE091B705EE23F9F0E150E09379
:10EEB000B70598E0E99FF0011124DF01A854BA4F8B
:10EEC00017962C911797811108C016964C9116979A
:10EED00012966D917C91139703C040E060E070E062
:10EEE000E854FA4F80819181AACFD5CFCF93DF9399
:10EEF000FC01EB01809110069091110697FF04C070
:10EF000010921106109210064091AA055091AB057F
:10EF10006091AC057091AD0580911006909111063D
:10EF2000092E000CAA0BBB0B481759076A077B0771
:10EF300024F45093110640931006809122028823F6
:10EF4000D1F020911006309111068091AE0590917C
:10EF5000AF05A091B005B091B105BC01CD01620F24
:10EF6000731F811D911D1995BC018091B40590916D
:10EF7000B5050E94CF4180910506811108C080919E
:10EF8000A705882389F180912202882369F1809165
:10EF9000B2059091B305009791F020911006309141
:10EFA00011064091AE055091AF056091B00570918A
:10EFB000B105420F531F611D711DFE011995E091AE
:10EFC000A805F091A905309741F08091A70581111E
:10EFD00003C08091050681111995D8D3882321F0AB
:10EFE00080E0DF91CF915ECFDF91CF9108950F93B5
:10EFF0001F93CF93DF9380912202882359F0609171
:10F00000A4057091A50500E010E020E041E081E05A
:10F010000E94D3408091A60581111CC081E080939D
:10F02000A605C0910B06D0910C0620E040E060E000
:10F0300070E087EF97E703DF0E9402E81092A605D1
:10F0400020E040E060E070E0CE01DF91CF911F91C1
:10F050000F91F5CEDF91CF911F910F9108950097F9
:10F0600011F48DE49FE29093A5058093A405BFCF92
:10F07000282F10920A068091100690911106813077
:10F08000904820F0109211061092100680911206FE
:10F09000882331F0809110068093E9051092B6051F
:10F0A0008091E8051816BCF4082E000C990B821B01
:10F0B00091092091E905022E000C330B281739071E
:10F0C00054F097FF02C080E090E08093E9059093B0
:10F0D0001106809310068091E9056623C1F0909196
:10F0E000EA05891714F48093EA052091EA05022EB7
:10F0F000000C330B2C5F3F4F482F082E000C550B94
:10F100002417350734F484508093EA0508958093DA
:10F11000EA050895882361F063E972E084E690E0EF
:10F120000F94A7276AEB72E084E690E00D94A7277E
:10F1300068EB71E084E190E00D94A72721E0209333
:10F14000A6050F942F1A1092A60508950E943ECC92
:10F15000E1CF0E9442DADECF2091100630911106F5
:10F160002115310559F081E0121613060CF080E0EC
:10F170008093A30510921106109210068091A305AA
:10F1800008954F925F926F927F928F929F92AF926B
:10F19000BF92CF92DF92EF92FF920F931F93CF9384
:10F1A000DF931F921F92CDB7DEB75C014A01390190
:10F1B00028018701760169837A83CEDFD82EE6D2D3
:10F1C000C82E69817A81811104C08091220288232E
:10F1D000F9F092014D2DC5010E949E42CC20C1F054
:10F1E000DD2011F0F40101C0F3010F900F90DF91C9
:10F1F000CF911F910F91FF90EF90DF90CF90BF9034
:10F20000AF909F908F907F906F905F904F901994E8
:10F210000F900F90DF91CF911F910F91FF90EF9082
:10F22000DF90CF90BF90AF909F908F907F906F9026
:10F230005F904F900895FC0180810895FC018491B6
:10F2400008954F925F926F927F928F929F92AF92AA
:10F25000BF92CF92DF92EF92FF920F931F93CF93C3
:10F26000DF936C017B015A012901672B31F088245F
:10F270008394912CC0E0D0E019C0F8011182108273
:10F2800027C03701680C791C76946794E3012197B5
:10F29000A201BE01C601F50119951816190654F010
:10F2A000892BC9F04301FFEF8F1A9F0AE814F90474
:10F2B00040F702C07E01FACFCE15DF0530F4CE0153
:10F2C00002968816990620F02196F801D183C08312
:10F2D0008FEF9FEF05C0F801D183C08380E090E0FD
:10F2E000DF91CF911F910F91FF90EF90DF90CF9022
:10F2F000BF90AF909F908F907F906F905F904F9056
:10F3000008958F929F92AF92BF92CF92DF92EF9229
:10F31000FF920F931F93CF93DF93EC016B017A0160
:10F32000FB01199587FD06C0082F10E020E030E0B2
:10F33000219620C1982F907E903CC1F4082F0F7128
:10F3400010E020E030E04801590186E0880C991C6B
:10F35000AA1CBB1C8A95D1F7CE010196F60119951E
:10F360008F7395018401082B229604C1982F907FFA
:10F37000903E19F58F70882E912CA12CB12C16E09F
:10F38000880C991CAA1CBB1C1A95D1F7CE010196BA
:10F39000F60119958F73882A06E0880C991CAA1C1F
:10F3A000BB1C0A95D1F7CE010296F60119958F7311
:10F3B00095018401082B2396DDC0982F987F903FFC
:10F3C00081F58770882E912CA12CB12CF6E0880C49
:10F3D000991CAA1CBB1CFA95D1F7CE010196F60127
:10F3E00019958F73882AA6E0880C991CAA1CBB1C4F
:10F3F000AA95D1F7CE010296F60119958F73882A46
:10F40000B6E0880C991CAA1CBB1CBA95D1F7CE019A
:10F410000396F60119958F7395018401082B2496A4
:10F42000A9C0982F9C7F983FE9F58370882E912C76
:10F43000A12CB12C56E0880C991CAA1CBB1C5A9517
:10F44000D1F7CE010196F60119958F73882A66E0EF
:10F45000880C991CAA1CBB1C6A95D1F7CE01029698
:10F46000F60119958F73882A76E0880C991CAA1CDE
:10F47000BB1C7A95D1F7CE010396F60119958F73CF
:10F48000882AE6E0880C991CAA1CBB1CEA95D1F7D7
:10F49000CE010496F60119958F7395018401082B0E
:10F4A000259668C0982F9E7F9C3F09F04AC08170C6
:10F4B000882E912CA12CB12C86E0880C991CAA1CBA
:10F4C000BB1C8A95D1F7CE010196F60119958F7371
:10F4D000882A96E0880C991CAA1CBB1C9A95D1F727
:10F4E000CE010296F60119958F73882A26E0880CC2
:10F4F000991CAA1CBB1C2A95D1F7CE010396F601D4
:10F5000019958F73882A36E0880C991CAA1CBB1C9D
:10F510003A95D1F7CE010496F60119958F73882A92
:10F5200046E0880C991CAA1CBB1C4A95D1F7CE0159
:10F530000596F60119958F7395018401082B26967F
:10F5400019C0982F907C903849F4082F007C00381F
:10F5500071F42196CE01F6011995F7CF082F0E7F91
:10F560000D3F28F02196CE01F6011995F7CF00E066
:10F5700010E09801E114F10429F0F70100831183F0
:10F5800022833383CE01DF91CF911F910F91FF90A2
:10F59000EF90DF90CF90BF90AF909F908F900895A5
:10F5A0001F93CF93DF9300D01F92CDB7DEB710E04B
:10F5B000AE014F5F5F4F6BE179E7A3DE49815A816E
:10F5C0006B817C81452B462B472B11F01F5FF0CFC1
:10F5D000812F0F900F900F900F90DF91CF911F917F
:10F5E00008951F93CF93DF9300D01F92CDB7DEB75E
:10F5F00010E0AE014F5F5F4F6EE179E782DE498137
:10F600005A816B817C81452B462B472B11F01F5F64
:10F61000F0CF812F0F900F900F900F90DF91CF912F
:10F620001F910895FC01A081B1811C92A281B38138
:10F630008C918F5F8C930280F381E02D80816CE050
:10F64000689F600D112480E00C94F73710920A0631
:10F650008091050610920506882349F020E040E0DD
:10F6600060E070E089EB91E6EADB0C943C4020918D
:10F670005F02309160024091100650911106C9015D
:10F68000840F951F2436310551F44730510514F08D
:10F69000069720C04A3F5F4F64F506961BC024368C
:10F6A000310524F48536910524F504C0843691058E
:10F6B00024F41FC08A3091053CF0883E43E0940753
:10F6C0002CF087EE93E002C08AE090E0281739071B
:10F6D00031F40DC08A30910584F78AE090E0909370
:10F6E000600280935F0210921106109210060C9433
:10F6F000EC3884E690E0E1CFCF93DF931F92CDB753
:10F70000DEB78091A708811103C089EE98E02FC071
:10F71000211103C087EA98E02AC08DE0815048F0AB
:10F72000440F411DE82FF0E0E751F74F9081492742
:10F73000F5CF8091FC058417A9F04093FC0587EA7A
:10F7400098E069832DDF90E06981861B910997FF1E
:10F7500002C080E090E080930D0610920E0688E0D3
:10F760008093240280910E0690E08955974F0F9068
:10F77000DF91CF91089580930A06109206061092A9
:10F780000706109208061092090608958091050652
:10F790001092050608957F928F929F92AF92BF922A
:10F7A000CF92DF92EF92FF920F931F93CF93DF934D
:10F7B000CDB7DEB728970FB6F894DEBF0FBECDBF2A
:10F7C0007C014B016A015901FB0180816CE0689F5B
:10F7D000600D1124F7018081982F990F890F880FF0
:10F7E0000E94F737C114D10409F496C0FE82ED825D
:10F7F00098868F82011103C01C2D0D2D74C09D2C85
:10F800000C2D1D2DD12C88248394AE014F5F5F4FAA
:10F81000B5018C2D992D75DDC82E992E89819A817F
:10F82000AB81BC81772473940097A105B105C9F021
:10F83000712C80329105A105B10581F0AC01BD01AB
:10F840004D52510961097109423051056105710537
:10F8500040F08B97A105B10589F503C0DD2009F4BF
:10F8600055C0F70120818D2D90E0820F911D4697A4
:10F870002CF0253018F0CE010596D4DE372D382532
:10F88000D30EF70180818D0D8083DD2089F0DA941D
:10F89000AE014F5F5F4FB501C80133DD8C01698157
:10F8A0007A818B819C814FEF5FEF0E940238EDCF10
:10F8B000711032C00C2D192DD12CA7CFD394011566
:10F8C000110509F0A2CF0C2D192D9FCF4FEF5FEF3F
:10F8D0000E940238F70120812F5F2083253118F024
:10F8E000CE0105969FDEAE014F5F5F4FB501812FC0
:10F8F000902F07DD182F092F69817A818B819C81D8
:10F90000611571058105910509F706C001151105FD
:10F9100089F20F5F1F4FD3CF28960FB6F894DEBF42
:10F920000FBECDBFDF91CF911F910F91FF90EF9050
:10F93000DF90CF90BF90AF909F908F907F90089571
:10F94000AF92BF92CF92DF92EF92FF920F931F93ED
:10F95000CF93DF931F921F92CDB7DEB75C016B018F
:10F960007A013FDE182FE114F10419F0C70139DEE6
:10F9700001C080E01A821982C114D104C1F4412F60
:10F9800050E090E09A01280F391F263131057CF4B0
:10F9900025E130E0241B350B281B390B37FF02C053
:10F9A0002F5F3F4F359527952A8381E0898301E0BA
:10F9B0002EE139E7A501BE016F5F7F4FCE010296B0
:10F9C000EADEC114D10489F08A81882321F01A82E9
:10F9D00089818F5F898300E02BE139E7A601BE01B1
:10F9E0006F5F7F4FCE010296D6DEE114F10451F035
:10F9F00000E02EE139E7A701BE016F5F7F4FCE0126
:10FA00000296C9DE0F900F90DF91CF911F910F9159
:10FA1000FF90EF90DF90CF90BF90AF900895CF927E
:10FA2000DF92EF92FF920F931F930E94BC2B0091E5
:10FA3000F8051091F9052091FA053091FB056B014D
:10FA40007C01C01AD10AE20AF30AF7FC13C0209124
:10FA5000F70520952093F705DC01CB018A549C4FD4
:10FA6000AF4FBF4F8093F8059093F905A093FA0527
:10FA7000B093FB0581E09091F705911101C080E002
:10FA80001F910F91FF90EF90DF90CF900895CF934B
:10FA900093E090932202811110921A060E94BC2BCF
:10FAA000DC01CB018C509E4FAF4FBF4F80931406AB
:10FAB00090931506A0931606B093170668E873E1B5
:10FAC00082E090E00F94A727C6E0C15049F00F9460
:10FAD000462762E070E080E090E00E94ED2BF5CFD9
:10FAE000CF910895AF92BF92CF92DF92EF920F9392
:10FAF0001F93CF93DF9300D01F92CDB7DEB78091D5
:10FB000023028F3F09F444C00E94BC2B0091FD05E5
:10FB10001091FE052091FF0530910006DC01CB011C
:10FB2000801B910BA20BB30BB7FD32C09091120E4C
:10FB30008091150E8F5F8F70981751F1E09123021D
:10FB400084E0E802F0011124E85BFC4F20E030E0A3
:10FB500040E752E460817181828193810F94872B09
:10FB600069837A838B839C83A12CB12C6501E12C62
:10FB70008E010F5F1F4F21E732E04DE652E069E64C
:10FB800072E085E692E00E9474F58FEF8093230285
:10FB90000F900F900F900F90DF91CF911F910F91C9
:10FBA000EF90DF90CF90BF90AF9008950F931F9389
:10FBB0000E94BC2B00911406109115062091160688
:10FBC00030911706DC01CB01801B910BA20BB30B0C
:10FBD000B7FD0FC08091030185FB992790F981E063
:10FBE00089279091030196FF8260629B84608093D5
:10FBF0001A0680911A06817090911A0691FD826012
:10FC00009091EB05891741F18130A9F028F08230FD
:10FC100041F0833059F01EC0913089F09230A9F044
:10FC200019C0992361F0933081F014C0913069F0CC
:10FC3000923081F404C0992341F0933059F49091AB
:10FC40000F069F5F90930F0605C090910F0691508D
:10FC500090930F068093EB051F910F910895CF931A
:10FC6000DF930E943C40E4E0F1E080818F7D80835F
:10FC7000C5E0D1E0888180958072A3E0B1E08C93EB
:10FC800080818F7B80838881809580748C936A9833
:10FC9000729A54985C9A82E08093190687DF1092DA
:10FCA0000F06DF91CF910895CF93C09160068CE14C
:10FCB00096E076DCC81790F4809160068F5F21E0B3
:10FCC000280FE82FF0E0E45EF94F9081907C9038A7
:10FCD00011F4822FF4CF8093600602C01092600668
:10FCE000CF9108950F931F93CF93DF938C01C09111
:10FCF0006006D0E0C45ED94FCE0152DCF8018083AB
:10FD0000CE01DF91CF911F910F91089581E09091E5
:10FD10001C06911101C080E00895CF93DF932091DC
:10FD20005F06211120C0FC0101900020E9F7319706
:10FD3000EF01C81BD90BC334D10534F031972081B2
:10FD4000207C2038D9F3F4CFBC01DD27AE018CE153
:10FD500096E00F942334C45ED94F18821092600647
:10FD600083E080932202DF91CF910895CF93DF93B8
:10FD7000CDB7DEB78E8190915F06891790F08093A2
:10FD80005F069E01275F3F4F4F81588562E470E018
:10FD90008CE196E00F946C341092600683E08093BF
:10FDA0002202DF91CF9108950F931F93CF93DF939A
:10FDB0008C0167FF03C010925F0660E080915F06D0
:10FDC00090E0262F062E000C330B281739071CF164
:10FDD00060935F06C8010F948533F801E80FF91F9F
:10FDE000EF01C01BD10BC334D10534F0319784919E
:10FDF000807C8038D9F3F4CFDD27AE01B8018CE1E7
:10FE000096E00F94A633C45ED94F18821092600614
:10FE100083E080932202DF91CF911F910F9108958B
:10FE20004F925F926F927F928F929F92AF92BF920A
:10FE3000CF92DF92EF92FF920F931F93CF930E9486
:10FE4000BC2B6B017C014EDEB1DE80911A0682FF75
:10FE500015C08091F605811113C091E09093F605CD
:10FE600020914C16211103C08091A605892780930B
:10FE7000050610924C1681E00ADE02C01092F605CB
:10FE8000C9B1C295C17081E0C82780911906C81711
:10FE900079F10E94EA3F882359F110911906C09325
:10FEA0001906CC2309F4CAC164EF71E080E090E048
:10FEB0000E94AD9A0E94728B123009F0BAC10E9462
:10FEC000498C0E943C4083E0809322020E94BC2B1C
:10FED0006B017C01DC01CB018C599F4FAF4FBF4FB1
:10FEE0008093F2059093F305A093F405B093F50584
:10FEF0008091F2059091F305A091F405B091F5057C
:10FF0000A7019601281B390B4A0B5B0B57FF05C055
:10FF100080911306882309F41FC2D701C6018C59AA
:10FF20009F4FAF4FBF4F8093F2059093F305A0937F
:10FF3000F405B093F50560910F06062E000C770BC3
:10FF400077FF03C0719561957109062E000C770B40
:10FF5000880B990B0F94222C2B013C0120E030E000
:10FF600040E050E40F94832D87FF05C08091050683
:10FF700081117DC08DC080910A06882309F456C086
:10FF80008090060690900706A0900806B09009069B
:10FF900081149104A104B104E1F120E030E040E0DB
:10FFA0005FE3C301B2010F94BE2D2B013C01C701D9
:10FFB000B601681979098A099B090F94202C9B01C5
:10FFC000AC01C301B2010F94872B20E030E04AE777
:10FFD00054E40F94BE2D4B015C0120E030E040EA78
:10FFE00052E40F94832D87FF0FC020E030E040EFF4
:10FFF00051E4C501B4010F94832D87FD0AC02AE0A6
:020000021000EC
:1000000030E040E050E009C024E630E040E050E05D
:1000100004C021E030E040E050E0C0920606D092FB
:100020000706E0920806F092090604C021E030E0DD
:1000300040E050E0A0910F060091100610911106CB
:100040000A2E000CBB0B0F94252F22E030E040E07D
:1000500050E00F94E82EDA01C901800F911FA11D15
:10006000B11D909311068093100610920F06D701D0
:10007000C6018856954CAF4FBF4F8093EE059093C5
:10008000EF05A093F005B093F10581E08093220283
:1000900020910B0630910C064BE72632340741F4D1
:1000A00080912402882309F4D4C0815080932402D3
:1000B00024513D4551F580912402882321F081503F
:1000C0008093240222C084E08093240280910E0653
:1000D0008F5F80930E0690910D06981728F410926A
:1000E0000E068CE08093240281E080932202D701E7
:1000F000C6018856954CAF4FBF4F8093EE05909345
:10010000EF05A093F005B093F10580916F0081FB9E
:10011000222720F981FF05C080916F008D7F809399
:100120006F008091490D90914A0DA0914B0DB091B7
:100130004C0D222329F020916F00226020936F0044
:100140003AE0B695A795979587953A95D1F7009798
:1001500021E0A207B10520F08FEF9FEFA0E0B0E013
:100160009695879520912202211105C030911306A2
:100170003111EEC051C0009741F04091EC05509113
:10018000ED054817590708F047C080911306811103
:1001900017C0223008F06DC080911B04811107C088
:1001A00081E080931B0482EE93E00E948F3082EE08
:1001B00093E00E94C63081E080931206809313067C
:1001C00083E00E94CF3F61E082EE93E00E94EF3037
:1001D000E0910B06F0910C06199510921206809191
:1001E0001306811152C0109205060E94BC2BDC013F
:1001F000CB018C199D09AE09BF090091EC05109146
:10020000ED0520E030E0081719072A073B0720F426
:100210009093ED058093EC0580910B0690910C0670
:1002200086529B4709F457C080911806811153C02C
:100230007EC060E088EC9FE2B7DD43CEECD51230A3
:1002400009F43FCE60E08AEB9FE2AEDD0E944B777F
:1002500038CE8CE0809324028091EC059091ED05DE
:1002600001979093ED058093EC0581E08093220245
:100270001FCF243030F0243009F08ECF10922202AC
:100280008BCF81E08093220287CF82EE93E00E94A1
:10029000CA3091E0811101C090E090931306992338
:1002A00009F4A1CF0E94BC2BDC01CB018C199D0964
:1002B000AE09BF09C090EC05D090ED05E12CF12C02
:1002C000C816D906EA06FB0608F046C09093ED056D
:1002D0008093EC0541C048E9C40E4AE3D41EE11CFA
:1002E000F11CC092EE05D092EF05E092F005F0927D
:1002F000F1058091130681112FC080912202813077
:1003000099F0833049F5CF911F910F91FF90EF90B5
:10031000DF90CF90BF90AF909F908F907F906F9025
:100320005F904F900C946C401092220215C0809107
:10033000EE059091EF05A091F005B091F105C81A76
:10034000D90AEA0AFB0AF7FCD4CF0E944B77D1CF37
:10035000009709F435CF11CFCF911F910F91FF90E6
:10036000EF90DF90CF90BF90AF909F908F907F9055
:100370006F905F904F90089561E016DD0C944B777D
:10038000CF93DF931F921F92CDB7DEB789839A83F5
:1003900066DC89819A81F0DF0F900F90DF91CF9119
:1003A0000C9441408091F60882FD05C08091411671
:1003B000823061F410C08091A708811103C089EEDA
:1003C00098E002C087EA98E061E0A7CC813031F084
:1003D0008CE89FE205C08DEA9FE202C081EA9FE2BD
:1003E0006FEFE2CC10924C1610928C028091F608BE
:1003F00080648093F6080E944DA90F94E62760E080
:100400008EE79FE2D1DC0C944B7782E79FE20E945B
:100410002F7860E085E69FE2C7DC40E061E080E0A5
:100420000E9449618BE59FE20D942A1ABBDF10926E
:100430004C1610928C020E94AB61882321F08091AF
:10044000F60882FF04C00E9445A90D945E2887E546
:100450009FE20F942A1AF7CF8091F60882FF2AC0F4
:100460000E94AB61882319F18091B1069091B20688
:10047000A091B306B091B4060097A105B105B9F0FB
:10048000BC01CD016D597F4F8F4F9F4F24E630E067
:1004900040E050E00F94C62E6091AD067091AE061C
:1004A0008091AF069091B0060F94C62E01C020E057
:1004B00020931B0680911B068F77089586E29BE7A9
:1004C00090930C0680930B06089561E0FC018081F7
:1004D0000E94EC2D8FEF0C949C9BCF93DF93EC014B
:1004E0008A810E945E9B60E08881DF91CF910C94AD
:1004F000EC2D8F929F92AF92BF92EF92FF920F934B
:100500001F93CF93DF93EC018B017A010E94BC2BE8
:100510004B015C012CE2820E21E0921EA11CB11C59
:100520000E94769B8B838F3F61F40E94BC2BDC0181
:10053000CB0188199909AA09BB09B7FDF1CF81E15F
:100540000DC08E3F51F4B701C8010E947D9B0E94EF
:10055000769B0E94769B11E003C08FE0898310E0B8
:10056000CE01B3DF812FDF91CF911F910F91FF90CB
:10057000EF90BF90AF909F908F900895CF92DF92B1
:10058000EF92FF926A017B010E94BC2BC60ED71E20
:10059000E81EF91E0E94769B8F3F61F00E94BC2BE3
:1005A000DC01CB018C199D09AE09BF09B7FDF2CF63
:1005B00080E001C081E0FF90EF90DF90CF90089540
:1005C000EF92FF921F93CF93DF9300D01F92CDB78E
:1005D000DEB77C01162F29833A834B835C837DDF52
:1005E00048E552E060E070E0C701C8DF812F806419
:1005F0000E949C9B8C810E949C9B8B810E949C9B57
:100600008A810E949C9B89810E949C9B112311F0EE
:1006100087E801C085E90E949C9B1C3011F40E9470
:10062000769B10E00E94769BF701838387FF04C0CE
:100630001F3F11F01F5FF6CF0F900F900F900F909C
:10064000DF91CF911F91FF90EF9008958F929F922D
:10065000AF92BF92CF92DF92EF92FF920F931F93D0
:10066000CF93DF93EC01162F1C82198248830E94DE
:10067000BC2B6B017C0120EDC20E27E0D21EE11CD9
:10068000F11CA89561E088810E94EC2D61E08881D1
:100690000E94B02D0E946F9B85E08A830E945E9B22
:1006A0000AE08FEF0E949C9B0150D9F7A89520E0AB
:1006B00030E0A90160E0CE0183DF8B83813061F0FF
:1006C0000E94BC2BDC01CB018C199D09AE09BF092E
:1006D000B7FDEDCF81E055C0A8952AEA31E040E0B2
:1006E00050E068E0CE016CDF853011F481E009C094
:1006F00004E00E94769B8B830150D9F78A3A51F42B
:1007000082E08C83A8958C81823081F0812C912CA1
:10071000540111C00E94BC2BDC01CB018C199D0936
:10072000AE09BF09B7FDD9CF82E02BC0812C912C37
:10073000A12C80E4B82E20E030E0A90167E3CE01CF
:100740003FDFA501940169E2CE013ADF8B83882364
:1007500061F00E94BC2BDC01CB018C199D09AE0914
:10076000BF09B7FDE8CF8AE00CC08C818230D1F49C
:1007700020E030E0A9016AE3CE0122DF882329F0DE
:1007800088E08983CE01A1DE16C00E94769B807C22
:10079000803C11F483E08C830E94769B0E94769BC0
:1007A0000E94769BCE0191DE173018F41A8381E007
:1007B00003C088E1898380E0DF91CF911F910F9181
:1007C000FF90EF90DF90CF90BF90AF909F908F9071
:1007D00008950F931F93CF93DF93EC0189018C81D0
:1007E000833039F089E0440F551F661F771F8A95C3
:1007F000D1F79A01AB0161E1CE01E2DE811109C0BE
:1008000040E052E0B801CE01DF91CF911F910F91EE
:1008100070CE84E08983CE0158DE80E0DF91CF91F5
:100820001F910F910895CF93DF93EC01862FBA01AA
:100830000E94A19B8FEF0E949C9B8FEF0E949C9B2C
:100840000E94769B8B83982F9F71953031F083E1C6
:100850008983CE013ADE80E001C081E0DF91CF9153
:1008600008950F931F93CF93DF93EC0189018C813F
:10087000833039F089E0440F551F661F771F8A9532
:10088000D1F79A01AB0168E1CE019ADE81111EC059
:10089000A8016EEFCE01C7DF8823E1F048E552E002
:1008A00060E070E0CE016ADE882371F020E030E085
:1008B000A9016DE0CE0184DE81110AC00E94769B01
:1008C000811106C011E007C087E103C086E001C0C6
:1008D00086E1898310E0CE01F8DD812FDF91CF9191
:1008E0001F910F910895CF93DF931F92CDB7DEB77D
:1008F00020914E1630914F16CE01019621153105EB
:1009000019F0821B930B02C0845596410F90DF9122
:10091000CF910895FC01238121110C94B395089582
:1009200081E696E0F7CF8CE796E0F4CF80919706CA
:10093000811107C00E9442DA882319F081E0809378
:10094000970608958091F608847F8B7F8093F60840
:100950001092AD061092AE061092AF061092B0063D
:100960001092B1061092B2061092B3061092B4061D
:1009700010922207109261078EE091E0E2E6F7E024
:10098000DF019C011D9221503040E1F78FEF8093F1
:10099000A6080895FC0120E03EE2DB014C914032C4
:1009A00041F0283011F430833196DB014C914083C3
:1009B00031962F5F6F5F7F4F2B3079F7108208954C
:1009C0002F923F924F925F926F927F928F929F925F
:1009D000AF92BF92CF92DF92EF92FF920F931F934D
:1009E000CF93DF93CDB7DEB7C356D1090FB6F894D6
:1009F000DEBF0FBECDBF8C015B014A014DB65EB6B6
:100A0000312C7E0187E5E80EF11C9BE1292E47EA97
:100A100058E0BE016F5F7F4FC5010E9423941816F6
:100A20000CF005C18C85282F2871203109F074C085
:100A30009091AC069150923008F46EC06DB67EB6BF
:100A4000BE016F5F7F4FC701A5DF0115110521F0C2
:100A5000F8018081811173C021E081E090E0F7010D
:100A600001900020E9F73197EE19FF09E80FF91F0F
:100A700032968DB79EB78E1B9F0B0FB6F8949EBF14
:100A80000FBE8DBFEDB7FEB731966F01211102C0C9
:100A9000B80102C068E573E0C6010F940E34B701D7
:100AA000C6010F94F83368E573E0C6010F94F8337C
:100AB0001CAE1FAE21E0A701B501CE01CC960E946D
:100AC000AF9781110DC08091AC06811109C00E94C1
:100AD000DF9A8AEC91E30E94D19AC7010E94D4A0C8
:100AE000FE01FC96DE019196822D01900D928A9571
:100AF000E1F740E050E0BE016F5D7F4FC60160DF6F
:100B0000CE01819607DFCE01CC9604DF0FB6F894B4
:100B10007EBE0FBE6DBE7BCF9981992309F487C03D
:100B2000953E09F474CF9E3209F471CF9091A708D5
:100B30009E3209F46CCF8A7009F069CF0AC0F801BF
:100B400001900020E9F73197CF01801B910B20E045
:100B500086CF81E0203109F080E09091F60880FB9B
:100B600094F99093F608811108C08985873409F0BB
:100B70004ECF8A858E3709F44ACF8091AC068130FA
:100B800021F068F08230B9F142CF8091AA069091AD
:100B9000AB0601969093AB068093AA0638CFBE01B0
:100BA0006F5F7F4F89EE98E0F5DE0115110511F0BA
:100BB000680105C089EEC82E88E0D82E08C0F6016D
:100BC00081916F018823B1F30E947DA0F8CFF601D7
:100BD00081916F01882319F00E947DA0F8CF80E2F7
:100BE0000E947DA06D8D7E8D8F8D98A14AE050E092
:100BF0000E948AA10CCFBE016F5F7F4F89EE98E003
:100C0000C9DE8114910441F069EE78E0C4010F94CB
:100C1000E533892B51F40BC0832D90E02091A80679
:100C20003091A9068217930711F03394F0CE0FB6D6
:100C3000F8945EBE0FBE4DBECD59DF4F0FB6F8948F
:100C4000DEBF0FBECDBFDF91CF911F910F91FF90FF
:100C5000EF90DF90CF90BF90AF909F908F907F905C
:100C60006F905F904F903F902F900895CF93DF93B8
:100C7000CDB7DEB76B970FB6F894DEBF0FBECDBF12
:100C80001092AC0640E050E0BA018BE898E00E9478
:100C9000D2948BE1EBE8F8E0DE01119601900D9221
:100CA0008A95E1F740E050E0BE016F5F7F4F80E042
:100CB00090E086DECE0101962DDE6B960FB6F8949D
:100CC000DEBF0FBECDBFDF91CF9108950F931F936D
:100CD000CF93DF93CDB7DEB72D970FB6F894DEBF75
:100CE0000FBECDBF80912607882391F0BE016F5FB4
:100CF0007F4F83E297E00E9445928E010F5F1F4F66
:100D0000F80181918F01882339F00E947DA0F8CFEE
:100D100080EC91E30E94D19A8AE00E947DA02D96FA
:100D20000FB6F894DEBF0FBECDBFDF91CF911F91FC
:100D30000F910895CF92DF92EF92FF920F931F933E
:100D4000CF93DF93CDB7DEB7EDB6FEB6DC010D90E5
:100D50000020E9F79D01281B390B2C5F3F4F4DB751
:100D60005EB7421B530B0FB6F8945EBF0FBE4DBF6C
:100D70000DB71EB70F5F1F4F9F938F938AE791E3C5
:100D80009F938F931F930F930F943D34680154E00A
:100D9000C50ED11C0F900F900F900F900F900F90D9
:100DA000F6018081882349F0082E000C990B0F94DE
:100DB0006933F60181936F01F3CFC8010F942F1AA5
:100DC00086E791E30F943D1A0FB6F894FEBE0FBE6E
:100DD000EDBEDF91CF911F910F91FF90EF90DF90CB
:100DE000CF9008958091F60883FF03C084608093BC
:100DF000F60808951092C30B8091F6088F7B8B7FC5
:100E00008093F6080E94AB61882321F083E297E08B
:100E10000C94B3950895EEDF8091F608877F809358
:100E2000F60808950F931F93CF93DF938B01EA0188
:100E3000DB016D917C910E944592D801ED91FC916E
:100E40009081888191110EC08936B0F48FE2808341
:100E5000F8018081918101969183808388818F5FE1
:100E600088830AC0893680F73196D801ED93FC93C8
:100E700088818F5F8883E1CFDF91CF911F910F91A0
:100E800008950F931F93CF93DF9300D0CDB7DEB7B4
:100E90009C012F5F3F4F3B832A832FE2FC0120837D
:100EA00081E0898310E00BE180916107181770F4ED
:100EB000019FC0011124AE014F5F5F4FBE016E5F05
:100EC0007F4F8E59984FAEDF1F5FEECF89818B35F4
:100ED00070F4AE014F5F5F4FBE016E5F7F4F83E2E4
:100EE00097E0A0DF8A819B8101979B838A83EA81B7
:100EF000FB8110820F900F900F90DF91CF911F9187
:100F00000F9108958091F60882FF1FC08EE390E351
:100F10000E94D19A6091AD067091AE068091AF06A5
:100F20009091B0064AE050E00E947FA18FE20E94BB
:100F30007DA06091B1067091B2068091B306909148
:100F4000B4064AE050E00C948AA18DE290E30C9440
:100F5000D19AEF92FF920F931F93CF93DF938C015F
:100F6000FC0101900020E9F73197EF01C81BD90B74
:100F7000109223076EE470E00F9403347C01009715
:100F800029F4FE013197E00FF11F0EC060E270E01E
:100F90000F9403348C010F5F1F4F6AE270E0C701AA
:100FA0000F940334FC0131978DE081838AE08283C2
:100FB0001382B80183E297E00E94429A809123074E
:100FC000882361F00E94E29A86E190E3DF91CF915D
:100FD0001F910F91FF90EF900C94D19ADF91CF91D8
:100FE0001F910F91FF90EF90089583E297E00E9488
:100FF000689583E297E00E94B3958091F6088D7F13
:101000008E7F8093F6081092AD061092AE06109275
:10101000AF061092B00681E08093B40B08950F9351
:101020001F93CF93DF93CDB7DEB76B970FB6F894CE
:10103000DEBF0FBECDBF8B0122E02093AC069093A4
:10104000A9068093A80640E050E0BA0180E798E046
:101050000E94D2948BE1E0E7F8E0DE011196019066
:101060000D928A95E1F7A801BE016F5F7F4F80E086
:1010700090E0A6DCCE0101964DDC6B960FB6F8949D
:10108000DEBF0FBECDBFDF91CF911F910F910895AD
:10109000CF93DF93CDB7DEB76B970FB6F894DEBF73
:1010A0000FBECDBF81E08093AC061092AB061092CC
:1010B000AA0640E050E0BA0180E798E00E94D2948E
:1010C0008BE1E0E7F8E0DE01119601900D928A9540
:1010D000E1F740E050E0BE016F5F7F4F80E090E0BD
:1010E0006FDCCE01019616DC8091AA069091AB06CA
:1010F0006B960FB6F894DEBF0FBECDBFDF91CF91D8
:1011000008952F923F924F925F926F927F928F92AB
:101110009F92AF92BF92CF92DF92EF92FF920F9386
:101120001F93CF93DF9300D01F92CDB7DEB77C0122
:101130008B01342E2DB73EB73C832B838091A006C4
:1011400081110BC010927C0610927F0681E0809383
:10115000A00683E994E80E94E53780919806811102
:101160000BC0109261061092640681E0809398068D
:1011700080E994E80E94E537F80180818F3251F4CC
:101180008BE898E0F70191838083109261070F5FED
:101190001F4F05C080E798E0F70191838083F70136
:1011A0000190F081E02DFA83E9832CE7A22E26E05E
:1011B000B22E3BE1232E0115110509F47FC04DB677
:1011C0005EB66FE270E0C8010F9403343C0108176B
:1011D000190708F073C06C01C01AD10ADD24C601DA
:1011E00001962DB73EB7281B390B0FB6F8943EBFBA
:1011F0000FBE2DBF8DB79EB701964C01A601B80159
:101200000F942334F401EC0DFD1D1082332019F0EE
:10121000C4010E94D4A0F7016081718121E0A40182
:10122000C5010E94AF97811111C0B40189EF9FE2FF
:101230000E94E59A86EF9FE20E94D19A0FB6F89439
:101240005EBE0FBE4DBE80E090E039C0F7018081E8
:10125000918129813A818217930711F00E94B395F9
:10126000F701B182A082A0916107AA3078F481E0F1
:101270008A0F809361072A9ED0011124AE59B84F7E
:10128000F501822D01900D928A95E1F7F701808199
:1012900091818C57964029F491E6A92E96E0B92EBB
:1012A00004C08CE7A82E86E0B82E83010F5F1F4F85
:1012B0000FB6F8945EBE0FBE4DBE7DCFC8012B8128
:1012C0003C810FB6F8943EBF0FBE2DBF0F900F901C
:1012D0000F900F90DF91CF911F910F91FF90EF90A2
:1012E000DF90CF90BF90AF909F908F907F906F9046
:1012F0005F904F903F902F9008950F931F93CF933F
:10130000DF931F921F92CDB7DEB72091F60823FF1F
:1013100028C0BC0140E0CE010196F3DE8C010097AD
:1013200001F1BC0189819A810E948998B8018823C2
:1013300081F08BE690E30E94E59A8AE00E947DA00E
:101340001092AD061092AE061092AF061092B00643
:1013500008C083E590E30E94E59A80E590E30E944F
:10136000D19A0F900F90DF91CF911F910F91089517
:10137000EF92FF920F931F93CF93DF9300D0CDB7DF
:10138000DEB72091F60823FF0AC1F42EE62E8C0169
:101390000E94AB61882309F452C0FF2009F45CC0AD
:1013A00080912207882361F00E94E29A81E391E311
:1013B0000E94D19A60E080E090E00F94FE28EFC098
:1013C00085EB96E05EDDE091220784E0E89FF00186
:1013D0001124E25EF84F8091AD069091AE06A09187
:1013E000AF06B091B00680839183A283B3830E943D
:1013F000DF9AB80188E191E30E94E59A8091220783
:1014000099E6899FB00111246B54794F8DE091E3E7
:101410000E94E59A4091AD065091AE066091AF06EC
:101420007091B00687E091E30E94469B8AE00E949B
:101430007DA0809122078F5F8093220725C0FF2027
:1014400039F00E94DF9A87EF90E30E94D19A1CC086
:101450001092220722E001C021E02B830E94DF9A34
:1014600082EF90E30E94D19A2B81213009F494C03D
:1014700086EE90E30E94D19AB8018EED90E30E942F
:10148000E59A8AE00E947DA0B5DC40E0B801CE017B
:10149000019637DE8C01009709F481C069817A8159
:1014A000EE2009F44FC021E0AC0183E297E00E94F6
:1014B000AF97882309F43EC0809134079091350797
:1014C000A0913607B09137078093B1069093B2068A
:1014D000A093B306B093B4061092AD061092AE0678
:1014E0001092AF061092B006B80180ED90E30E9412
:1014F000E59A4091B1065091B2066091B3067091A1
:10150000B40688EC90E30E94469B8AE00E947DA08E
:1015100089EB90E30E94D19AB80180E090E07FDDF2
:101520008091A708811102C0C80102C087EA98E033
:1015300060E02FC0B80185EA90E30E94E59A82EA54
:1015400090E30FC026E5AC0183E297E00E94AF97DD
:1015500081110AC0B8018EE890E30E94E59A8BE8F9
:1015600090E30E94D19A1BC08091F608816080931D
:10157000F608B80180E090E052DD1092B40BB8019B
:1015800089E790E30E94E59A8AE00E947DA060E0EE
:10159000C8010E948D7E03C08CEE90E36BCF0F904C
:1015A0000F900F90DF91CF911F910F91FF90EF90CF
:1015B00008952091F60822602093F60840E060E04C
:1015C000D7CE0F931F93CF93DF93CDB7DEB76B9733
:1015D0000FB6F894DEBF0FBECDBF8C0119821C82FE
:1015E00080917308811103C06BE878E002C060E766
:1015F00078E021E0A801CE0101960E94AF978823F0
:1016000019F18BE1FE013196A0E7B8E001900D924F
:101610008A95E1F78091F6088F7D8093F608A09176
:101620006107AA30D8F481E08A0F809361078BE1CB
:101630008A9FD0011124AE59B84FE0E7F8E001903D
:101640000D928A95E1F70AC00E94DF9AB80180EEF8
:101650009FE20E94E59A8AE00E947DA0CE01019659
:1016600059D96B960FB6F894DEBF0FBECDBFDF9190
:10167000CF911F910F910895809161078823C9F040
:10168000815080936107882359F090E001972BE106
:10169000289FF001299FF00D1124EE59F84F02C048
:1016A000EBE8F8E08BE1A0E7B8E001900D928A95B5
:1016B000E1F780916107811105C09091F608906271
:1016C0009093F60808958BE1EBE8F8E0A0E7B8E026
:1016D00001900D928A95E1F78091F60880628093DF
:1016E000F60808958091F608877F8093F608809128
:1016F0008E08882321F08BE898E00E94B39545E39B
:1017000060E08CE597E00E942683811105C00E946D
:10171000DF9A82EB91E314C041E06CE577E08EE361
:1017200097E08AD481110FC040E06CE577E08EE34A
:1017300097E082D4811107C00E94E29A8EE991E37A
:101740000E94D19A18C06EE377E08BE898E0F9D652
:10175000811105C00E94E29A8DE891E3F1CF80915A
:10176000F60888608093F6080E94DF9A81E891E38A
:101770000E94D19ADBD8A7DF83E0809322020895EC
:10178000AF92BF92CF92DF92EF92FF921F93CF93CF
:10179000DF93CDB7DEB7A8970FB6F894DEBF0FBEC4
:1017A000CDBF8091A60887FD64C08091F60882FDB8
:1017B00060C083FD02C096DF01C0B8D88091F608F2
:1017C00083FF54C08091A608082E000C990BC09688
:1017D0009F938F938DE090E39F938F936E0181E2AF
:1017E000C80ED11CDF92CF920F943D3440E050E000
:1017F000BA018BE898E00E94D2940F900F900F905E
:101800000F900F900F90FE0131967F0140E050E065
:10181000B7018BE898E00E94239418163CF5F70175
:1018200001900020E9F731971E2F1E19115068F022
:101830005701A10EB11C17FDBA94F501808190E00B
:101840000F946933F5018083F1CF8A858E37F1F2E9
:1018500045E050E0B601C7010F941534892BB1F66D
:10186000C60168DA8091A6088F5F01C08FEF809370
:10187000A608A8960FB6F894DEBF0FBECDBFDF91C5
:10188000CF911F91FF90EF90DF90CF90BF90AF90DE
:1018900008951092A60817CFFBCB0E9402E883E2BE
:1018A00097E00E94B39580912207882329F1815007
:1018B0008093220729E6829FC001112441E061E064
:1018C0008B54994F55DDE091220784E0E89FF001A9
:1018D0001124E25EF84F408151816281738140930F
:1018E000AD065093AE066093AF067093B00683E2E8
:1018F00097E00E94D29476CA7DDA0E94DCE70F94CA
:10190000E6270F942B286D3371058105910518F496
:1019100087ED9FE202C08CED9FE20F943D1A84E6B2
:1019200080931B06089510928B0810928E081092D7
:1019300070081092730880E090E0FC01EE59F84FB7
:10194000108213824B968E3021E09207B1F789E125
:1019500080935D071092600710925507109223073D
:10196000109226070895CF93DF9383E297E00E94B9
:101970008A84C0E7D8E06B97CE010E948A8487E012
:10198000C236D807C1F780E798E00E948A848BE8C6
:1019900098E0DF91CF910C948A84CF938091FB08DB
:1019A0008823B9F14091FE0A5091FF0A6091000B23
:1019B0007091010B2EEF38E08091FC089091FD08AA
:1019C0000E943184C82F811102C0C0E023C0409121
:1019D000F7085091F8086091F9087091FA084115DC
:1019E00051056105710591F02EEF38E08091FC08FA
:1019F0009091FD080E943184882339F31092F708F2
:101A00001092F8081092F9081092FA081092FB0848
:101A100001C0C1E08C2FCF910895CF92DF92EF9259
:101A2000FF92CF936B017C01C42F8091FE0A9091AD
:101A3000FF0AA091000BB091010B8C159D05AE051E
:101A4000BF05C9F0AADF811102C080E018C02EEFE7
:101A500038E0B701A6018091FC089091FD080E9432
:101A6000E983882391F3C092FE0AD092FF0AE092A4
:101A7000000BF092010B81E0C1118093FB08CF9124
:101A8000FF90EF90DF90CF900895CF92DF92EF928A
:101A9000FF920F931F93CF93DF93FC018185928573
:101AA000A385B4850196A11DB11D84179507A607CE
:101AB000B70710F480E060C08789803149F4BB2704
:101AC000A72F962F852FC388D488E588F6880FC066
:101AD000803281F783899489A589B6896A017B015F
:101AE000C7E0F694E794D794C794CA95D1F78C0DC4
:101AF0009D1DAE1DBF1DE9016A017B018F01409153
:101B0000FE0A5091FF0A6091000B7091010B84173F
:101B10009507A607B70731F040E0BC01CD017DDF96
:101B2000882341F2F8018789803179F4B701A60151
:101B3000552766277727440F551FFA01E250F74FC4
:101B400080819181A0E0B0E012C0B701A6014F777B
:101B5000552766277727440F551F440F551FFA0155
:101B6000E250F74F80819181A281B381BF70888359
:101B70009983AA83BB8381E0DF91CF911F910F915D
:101B8000FF90EF90DF90CF9008954F925F926F9209
:101B90007F92AF92BF92CF92DF92EF92FF920F931C
:101BA0001F93CF93DF9300D01F92CDB7DEB78C0188
:101BB00049835A836B837C835901C12CD12C7601D4
:101BC000412C82E0582E612C712C49815A816B8105
:101BD0007C819E012F5F3F4FC80157DF882341F171
:101BE000D301C201F801058404C0880F991FAA1F00
:101BF000BB1F0A94D2F7C80ED91EEA1EFB1E4981EC
:101C00005A816B817C818789803139F481E0483F3A
